 textPlugin

 Timestamp is 614c8024 (Thu Sep 23 13:24:52 2021)

 Preferred load address is 10000000

 Start         Length     Name                   Class
 0001:00000000 00000063H .text$di                CODE
 0001:00000070 0000482cH .text$mn                CODE
 0001:0000489c 00000c84H .text$x                 CODE
 0001:00005520 00000021H .text$yd                CODE
 0002:00000000 000007d4H .idata$5                DATA
 0002:000007d4 00000004H .CRT$XCA                DATA
 0002:000007d8 0000000cH .CRT$XCU                DATA
 0002:000007e4 00000004H .CRT$XCZ                DATA
 0002:000007e8 00000004H .CRT$XIA                DATA
 0002:000007ec 00000004H .CRT$XIAA               DATA
 0002:000007f0 00000004H .CRT$XIC                DATA
 0002:000007f4 00000004H .CRT$XIZ                DATA
 0002:000007f8 00002198H .rdata                  DATA
 0002:00002990 00000b0cH .rdata$r                DATA
 0002:0000349c 00000004H .rtc$IAA                DATA
 0002:000034a0 00000004H .rtc$IZZ                DATA
 0002:000034a4 00000004H .rtc$TAA                DATA
 0002:000034a8 00000004H .rtc$TZZ                DATA
 0002:000034b0 00000cbcH .xdata$x                DATA
 0002:00004170 0000005eH .edata                  DATA
 0002:000041d0 0000003cH .idata$2                DATA
 0002:0000420c 00000014H .idata$3                DATA
 0002:00004220 000007d4H .idata$4                DATA
 0002:000049f4 00004ffaH .idata$6                DATA
 0003:00000000 00000054H .data                   DATA
 0003:00000054 000003fcH .data$r                 DATA
 0003:00000450 000003a4H .bss                    DATA
 0004:00000000 000000a0H .rsrc$01                DATA
 0004:000000a0 00000608H .rsrc$02                DATA

  Address         Publics by Value              Rva+Base       Lib:Object

 0000:00000000       ___guard_fids_table        00000000     <absolute>
 0000:00000000       ___safe_se_handler_table   00000000     <absolute>
 0000:00000000       ___guard_fids_count        00000000     <absolute>
 0000:00000000       ___safe_se_handler_count   00000000     <absolute>
 0000:00000000       ___guard_flags             00000000     <absolute>
 0000:00000000       ___ImageBase               10000000     <linker-defined>
 0001:00000070       ??0config@@QAE@ABVQString@@@Z 10001070 f   config.obj
 0001:000008d8       ??1config@@UAE@XZ          100018d8 f   config.obj
 0001:00000939       ??_Gconfig@@UAEPAXI@Z      10001939 f i config.obj
 0001:00000939       ??_Econfig@@UAEPAXI@Z      10001939 f i config.obj
 0001:00000958       ?getDescFromKey@config@@QAE?AVQString@@ABV2@@Z 10001958 f   config.obj
 0001:000009cc       ?getFilenameFromKey@config@@QAE?AVQString@@ABV2@@Z 100019cc f   config.obj
 0001:00000a40       ?getHelpFromKey@config@@QAE?AVQString@@ABV2@@Z 10001a40 f   config.obj
 0001:00000ab4       ?getKeys@config@@QAE?AVQStringList@@XZ 10001ab4 f   config.obj
 0001:00000cdb       ?getNamedAttribute@config@@AAE?AVQString@@ABV2@0@Z 10001cdb f   config.obj
 0001:00000f05       ??_Econfig_plugin_desc_base@@UAEPAXI@Z 10001f05 f i plugindesc.obj
 0001:00000f05       ??_Gplugindesc@@UAEPAXI@Z  10001f05 f i plugindesc.obj
 0001:00000f05       ??_Gconfig_plugin_desc_base@@UAEPAXI@Z 10001f05 f i plugindesc.obj
 0001:00000f05       ??_Eplugindesc@@UAEPAXI@Z  10001f05 f i plugindesc.obj
 0001:00000f25       ?create@plugindesc@@UAEPAVconfig_plugin_base@@ABVQString@@00@Z 10001f25 f   plugindesc.obj
 0001:00000f60       ?keys@plugindesc@@UAE?AVQStringList@@ABVQString@@0@Z 10001f60 f   plugindesc.obj
 0001:00000fa6       ?pixmap@plugindesc@@UAE?AVQPixmap@@ABVQString@@@Z 10001fa6 f   plugindesc.obj
 0001:00000fc5       _load_bncs_config_plugin_desc 10001fc5 f   plugindesc.obj
 0001:00000fdd       ??0text_highlighter@@QAE@PAVQTextEdit@@@Z 10001fdd f   text_highlighter.obj
 0001:0000104e       ??1text_highlighter@@UAE@XZ 1000204e f   text_highlighter.obj
 0001:000010a1       ??_Gtext_highlighter@@UAEPAXI@Z 100020a1 f i text_highlighter.obj
 0001:000010a1       ??_Etext_highlighter@@UAEPAXI@Z 100020a1 f i text_highlighter.obj
 0001:000010c0       ?highlightParagraph@text_highlighter@@UAEHABVQString@@H@Z 100020c0 f   text_highlighter.obj
 0001:000014cd       ??0?$QGuardedPtr@VQPopupMenu@@@@QAE@XZ 100024cd f i textPlugin.obj
 0001:000014cd       ??0?$QGuardedPtr@VQDockWindow@@@@QAE@XZ 100024cd f i textPlugin.obj
 0001:0000150e       ??0config_plugin_base@@QAE@ABVQString@@00@Z 1000250e f i textPlugin.obj
 0001:0000159b       ??0textPlugin@@QAE@ABVQString@@00@Z 1000259b f   textPlugin.obj
 0001:000017b5       ??1?$QDict@VQAction@@@@UAE@XZ 100027b5 f i textPlugin.obj
 0001:000017e8       ??1?$QGuardedPtr@VQDockWindow@@@@QAE@XZ 100027e8 f i textPlugin.obj
 0001:000017e8       ??1?$QGuardedPtr@VQPopupMenu@@@@QAE@XZ 100027e8 f i textPlugin.obj
 0001:000017ed       ??1?$QPtrList@VQPopupMenu@@@@UAE@XZ 100027ed f i textPlugin.obj
 0001:00001820       ??1QDockWindowList@@UAE@XZ 10002820 f i textPlugin.obj
 0001:00001869       ??1QPopupMenuList@@UAE@XZ  10002869 f i textPlugin.obj
 0001:0000189b       ??1config_plugin_base@@UAE@XZ 1000289b f i textPlugin.obj
 0001:000018f5       ??1textPlugin@@UAE@XZ      100028f5 f   textPlugin.obj
 0001:000019a5       ??_Econfig_plugin_base@@WCI@AEPAXI@Z 100029a5 f i textPlugin.obj
 0001:000019ad       ??_EtextPlugin@@WCI@AEPAXI@Z 100029ad f i textPlugin.obj
 0001:000019b5       ??_G?$QDict@VQAction@@@@UAEPAXI@Z 100029b5 f i textPlugin.obj
 0001:000019b5       ??_E?$QDict@VQAction@@@@UAEPAXI@Z 100029b5 f i textPlugin.obj
 0001:000019d4       ??_E?$QPtrList@VQPopupMenu@@@@UAEPAXI@Z 100029d4 f i textPlugin.obj
 0001:000019d4       ??_G?$QPtrList@VQPopupMenu@@@@UAEPAXI@Z 100029d4 f i textPlugin.obj
 0001:000019f3       ??_GQDockWindowList@@UAEPAXI@Z 100029f3 f i textPlugin.obj
 0001:000019f3       ??_EQDockWindowList@@UAEPAXI@Z 100029f3 f i textPlugin.obj
 0001:00001a12       ??_GQGuardedPtrPrivate@@UAEPAXI@Z 10002a12 f i textPlugin.obj
 0001:00001a12       ??_EQGuardedPtrPrivate@@UAEPAXI@Z 10002a12 f i textPlugin.obj
 0001:00001a32       ??_EQPopupMenuList@@UAEPAXI@Z 10002a32 f i textPlugin.obj
 0001:00001a32       ??_GQPopupMenuList@@UAEPAXI@Z 10002a32 f i textPlugin.obj
 0001:00001a51       ??_Gconfig_plugin_base@@UAEPAXI@Z 10002a51 f i textPlugin.obj
 0001:00001a51       ??_Econfig_plugin_base@@UAEPAXI@Z 10002a51 f i textPlugin.obj
 0001:00001a70       ??_GtextPlugin@@UAEPAXI@Z  10002a70 f i textPlugin.obj
 0001:00001a70       ??_EtextPlugin@@UAEPAXI@Z  10002a70 f i textPlugin.obj
 0001:00001a8f       ?about@config_plugin_base@@UAE?AVQString@@XZ 10002a8f f i textPlugin.obj
 0001:00001ae5       ?about@textPlugin@@UAE?AVQString@@XZ 10002ae5 f   textPlugin.obj
 0001:00001b8d       ?activate@config_plugin_base@@UAEX_N@Z 10002b8d f i textPlugin.obj
 0001:00001b8d       ?reply@config_plugin_base@@UAEXPAVresponse@@@Z 10002b8d f i textPlugin.obj
 0001:00001b90       ?activate@textPlugin@@UAEX_N@Z 10002b90 f   textPlugin.obj
 0001:00001d9f       ?apply@config_plugin_base@@UAEXXZ 10002d9f f i textPlugin.obj
 0001:00001da1       ?apply@textPlugin@@UAEXXZ  10002da1 f   textPlugin.obj
 0001:00002053       ?clear@?$QDict@VQAction@@@@UAEXXZ 10003053 f i textPlugin.obj
 0001:00002059       ?clear@?$QPtrList@VQPopupMenu@@@@UAEXXZ 10003059 f i textPlugin.obj
 0001:0000205f       ?closeEvent@config_plugin_base@@UAEXPAVQCloseEvent@@@Z 1000305f f i textPlugin.obj
 0001:0000206d       ?closeEvent@textPlugin@@UAEXPAVQCloseEvent@@@Z 1000306d f   textPlugin.obj
 0001:000020c9       ?count@?$QDict@VQAction@@@@UBEIXZ 100030c9 f i textPlugin.obj
 0001:000020cd       ?count@?$QPtrList@VQPopupMenu@@@@UBEIXZ 100030cd f i textPlugin.obj
 0001:000020d1       ?db@@YAXABVQString@@@Z     100030d1 f   textPlugin.obj
 0001:00002119       ?deleteItem@?$QPtrList@VQPopupMenu@@@@EAEXPAX@Z 10003119 f i textPlugin.obj
 0001:00002119       ?deleteItem@?$QDict@VQAction@@@@EAEXPAX@Z 10003119 f i textPlugin.obj
 0001:00002134       ?deref@?$QGuardedPtr@VQPopupMenu@@@@AAEXXZ 10003134 f i textPlugin.obj
 0001:00002134       ?deref@?$QGuardedPtr@VQDockWindow@@@@AAEXXZ 10003134 f i textPlugin.obj
 0001:00002149       ?isDirty@textPlugin@@UAE_NXZ 10003149 f   textPlugin.obj
 0001:00002156       ?menus@config_plugin_base@@UAE?AVQPopupMenuList@@XZ 10003156 f i textPlugin.obj
 0001:00002179       ?menus@textPlugin@@UAE?AVQPopupMenuList@@XZ 10003179 f   textPlugin.obj
 0001:000021c3       ?metaObject@textPlugin@@UBEPAVQMetaObject@@XZ 100031c3 f i textPlugin.obj
 0001:000021c8       ?navigate@config_plugin_base@@UAEXABVQString@@0@Z 100031c8 f i textPlugin.obj
 0001:000021cb       ?navigate@textPlugin@@UAEXABVQString@@0@Z 100031cb f   textPlugin.obj
 0001:00002247       ?reply@textPlugin@@UAEXPAVresponse@@@Z 10003247 f   textPlugin.obj
 0001:00002626       ?resizeEvent@textPlugin@@UAEXPAVQResizeEvent@@@Z 10003626 f   textPlugin.obj
 0001:0000265b       ?textStatus@response@@QAE?AVQString@@W4status@1@@Z 1000365b f i textPlugin.obj
 0001:000026aa       ?toolbars@config_plugin_base@@UAE?AVQDockWindowList@@XZ 100036aa f i textPlugin.obj
 0001:000026cd       ?toolbars@textPlugin@@UAE?AVQDockWindowList@@XZ 100036cd f   textPlugin.obj
 0001:00002725       ?validate@config_plugin_base@@UAE_NXZ 10003725 f i textPlugin.obj
 0001:00002725       ?isDirty@config_plugin_base@@UAE_NXZ 10003725 f i textPlugin.obj
 0001:00002728       ??0textPluginDlg@@QAE@ABVQString@@PAVQWidget@@PBDI@Z 10003728 f   textPlugindlgimpl.obj
 0001:000027a0       ??1textPluginDlg@@UAE@XZ   100037a0 f   textPlugindlgimpl.obj
 0001:000027f2       ??_EtextPluginDlg@@WCI@AEPAXI@Z 100037f2 f i textPlugindlgimpl.obj
 0001:000027fa       ??_GtextPluginDlg@@UAEPAXI@Z 100037fa f i textPlugindlgimpl.obj
 0001:000027fa       ??_EtextPluginDlg@@UAEPAXI@Z 100037fa f i textPlugindlgimpl.obj
 0001:00002819       ?load@textPluginDlg@@QAE_NABVQString@@@Z 10003819 f   textPlugindlgimpl.obj
 0001:000028d8       ?metaObject@textPluginDlg@@UBEPAVQMetaObject@@XZ 100038d8 f i textPlugindlgimpl.obj
 0001:000028dd       ?save@textPluginDlg@@QAEXABVQString@@@Z 100038dd f   textPlugindlgimpl.obj
 0001:00002965       ?setClean@textPluginDlg@@QAEXXZ 10003965 f   textPlugindlgimpl.obj
 0001:0000296d       ?setReadOnly@textPluginDlg@@QAEX_N@Z 1000396d f   textPlugindlgimpl.obj
 0001:000029a2       ?textChanged@textPluginDlg@@QAEXXZ 100039a2 f   textPlugindlgimpl.obj
 0001:000029eb       ??0xml_highlighter@@QAE@PAVQTextEdit@@@Z 100039eb f   xml_highlighter.obj
 0001:00002b01       ??1xml_highlighter@@UAE@XZ 10003b01 f   xml_highlighter.obj
 0001:00002b39       ??_Gxml_highlighter@@UAEPAXI@Z 10003b39 f i xml_highlighter.obj
 0001:00002b39       ??_Exml_highlighter@@UAEPAXI@Z 10003b39 f i xml_highlighter.obj
 0001:00002b58       ?setDefaultColours@xml_highlighter@@QAEXXZ 10003b58 f   xml_highlighter.obj
 0001:00002bae       ?className@textPlugin@@UBEPBDXZ 10003bae f   moc_textPlugin.obj
 0001:00002bb4       ?command@textPlugin@@IAEXVQString@@0@Z 10003bb4 f   moc_textPlugin.obj
 0001:00002c74       ?qt_cast@textPlugin@@UAEPAXPBD@Z 10003c74 f   moc_textPlugin.obj
 0001:00002ca2       ?qt_emit@textPlugin@@UAE_NHPAUQUObject@@@Z 10003ca2 f   moc_textPlugin.obj
 0001:00002d06       ?qt_invoke@textPlugin@@UAE_NHPAUQUObject@@@Z 10003d06 f   moc_textPlugin.obj
 0001:00002d10       ?qt_property@textPluginDlgBase@@UAE_NHHPAVQVariant@@@Z 10003d10 f   moc_textPlugindlg.obj
 0001:00002d10       ?qt_property@textPlugin@@UAE_NHHPAVQVariant@@@Z 10003d10 f   moc_textPlugin.obj
 0001:00002d1a       ?staticMetaObject@textPlugin@@SAPAVQMetaObject@@XZ 10003d1a f   moc_textPlugin.obj
 0001:00002daf       ?className@textPluginDlgBase@@UBEPBDXZ 10003daf f   moc_textPlugindlg.obj
 0001:00002db5       ?qt_cast@textPluginDlgBase@@UAEPAXPBD@Z 10003db5 f   moc_textPlugindlg.obj
 0001:00002de3       ?qt_emit@textPluginDlgBase@@UAE_NHPAUQUObject@@@Z 10003de3 f   moc_textPlugindlg.obj
 0001:00002ded       ?qt_invoke@textPluginDlgBase@@UAE_NHPAUQUObject@@@Z 10003ded f   moc_textPlugindlg.obj
 0001:00002e1f       ?staticMetaObject@textPluginDlgBase@@SAPAVQMetaObject@@XZ 10003e1f f   moc_textPlugindlg.obj
 0001:00002e69       ?tr@textPluginDlgBase@@SA?AVQString@@PBD0@Z 10003e69 f   moc_textPlugindlg.obj
 0001:00002eac       ?className@textPluginDlg@@UBEPBDXZ 10003eac f   moc_textPlugindlgimpl.obj
 0001:00002eb2       ?command@textPluginDlg@@IAEXVQString@@0@Z 10003eb2 f   moc_textPlugindlgimpl.obj
 0001:00002f72       ?qt_cast@textPluginDlg@@UAEPAXPBD@Z 10003f72 f   moc_textPlugindlgimpl.obj
 0001:00002f9f       ?qt_emit@textPluginDlg@@UAE_NHPAUQUObject@@@Z 10003f9f f   moc_textPlugindlgimpl.obj
 0001:00003002       ?qt_invoke@textPluginDlg@@UAE_NHPAUQUObject@@@Z 10004002 f   moc_textPlugindlgimpl.obj
 0001:00003030       ?qt_property@textPluginDlg@@UAE_NHHPAVQVariant@@@Z 10004030 f   moc_textPlugindlgimpl.obj
 0001:00003039       ?staticMetaObject@textPluginDlg@@SAPAVQMetaObject@@XZ 10004039 f   moc_textPlugindlgimpl.obj
 0001:000030d1       ??0textPluginDlgBase@@QAE@PAVQWidget@@PBDI@Z 100040d1 f   textPlugindlg.obj
 0001:000033a8       ??1textPluginDlgBase@@UAE@XZ 100043a8 f   textPlugindlg.obj
 0001:000033bb       ??_EQHBoxLayout@@WCI@AEPAXI@Z 100043bb f i textPlugindlg.obj
 0001:000033c3       ??_EQLabel@@WCI@AEPAXI@Z   100043c3 f i textPlugindlg.obj
 0001:000033cb       ??_EQTextEdit@@WCI@AEPAXI@Z 100043cb f i textPlugindlg.obj
 0001:000033d3       ??_EQVBoxLayout@@WCI@AEPAXI@Z 100043d3 f i textPlugindlg.obj
 0001:000033db       ??_EtextPluginDlgBase@@WCI@AEPAXI@Z 100043db f i textPlugindlg.obj
 0001:000033e3       ??_GQHBoxLayout@@UAEPAXI@Z 100043e3 f i textPlugindlg.obj
 0001:000033e3       ??_EQHBoxLayout@@UAEPAXI@Z 100043e3 f i textPlugindlg.obj
 0001:00003403       ??_EQLabel@@UAEPAXI@Z      10004403 f i textPlugindlg.obj
 0001:00003403       ??_GQLabel@@UAEPAXI@Z      10004403 f i textPlugindlg.obj
 0001:00003423       ??_GQSpacerItem@@UAEPAXI@Z 10004423 f i textPlugindlg.obj
 0001:00003423       ??_EQSpacerItem@@UAEPAXI@Z 10004423 f i textPlugindlg.obj
 0001:00003443       ??_GQTextEdit@@UAEPAXI@Z   10004443 f i textPlugindlg.obj
 0001:00003443       ??_EQTextEdit@@UAEPAXI@Z   10004443 f i textPlugindlg.obj
 0001:00003463       ??_EQVBoxLayout@@UAEPAXI@Z 10004463 f i textPlugindlg.obj
 0001:00003463       ??_GQVBoxLayout@@UAEPAXI@Z 10004463 f i textPlugindlg.obj
 0001:00003483       ??_EtextPluginDlgBase@@UAEPAXI@Z 10004483 f i textPlugindlg.obj
 0001:00003483       ??_GtextPluginDlgBase@@UAEPAXI@Z 10004483 f i textPlugindlg.obj
 0001:000034a2       ?languageChange@textPluginDlgBase@@MAEXXZ 100044a2 f   textPlugindlg.obj
 0001:0000353a       ?metaObject@textPluginDlgBase@@UBEPAVQMetaObject@@XZ 1000453a f i textPlugindlg.obj
 0001:00003540       ?setName@QWidget@@UAEXPBD@Z 10004540 f   qt-mt323:qt-mt323.dll
 0001:00003546       ?closeEvent@QWidget@@MAEXPAVQCloseEvent@@@Z 10004546 f   qt-mt323:qt-mt323.dll
 0001:0000354c       ?adjustSize@QWidget@@UAEXXZ 1000454c f   qt-mt323:qt-mt323.dll
 0001:00003552       ?checkConnectArgs@QObject@@MAE_NPBDPBV1@0@Z 10004552 f   qt-mt323:qt-mt323.dll
 0001:00003558       ?childEvent@QObject@@MAEXPAVQChildEvent@@@Z 10004558 f   qt-mt323:qt-mt323.dll
 0001:0000355e       ?className@QGuardedPtrPrivate@@UBEPBDXZ 1000455e f   qt-mt323:qt-mt323.dll
 0001:00003564       ?className@QWidget@@UBEPBDXZ 10004564 f   qt-mt323:qt-mt323.dll
 0001:0000356a       ?clear@?$QPtrList@VQDockWindow@@@@UAEXXZ 1000456a f   qt-mt323:qt-mt323.dll
 0001:00003570       ?close@QWidget@@UAE_N_N@Z  10004570 f   qt-mt323:qt-mt323.dll
 0001:00003576       ?cmd@QPaintDevice@@MAE_NHPAVQPainter@@PATQPDevCmdParam@@@Z 10004576 f   qt-mt323:qt-mt323.dll
 0001:0000357c       ?compareItems@QGList@@MAEHPAX0@Z 1000457c f   qt-mt323:qt-mt323.dll
 0001:00003582       ?connectNotify@QObject@@MAEXPBD@Z 10004582 f   qt-mt323:qt-mt323.dll
 0001:00003588       ?contextMenuEvent@QWidget@@MAEXPAVQContextMenuEvent@@@Z 10004588 f   qt-mt323:qt-mt323.dll
 0001:0000358e       ?count@?$QPtrList@VQDockWindow@@@@UBEIXZ 1000458e f   qt-mt323:qt-mt323.dll
 0001:00003594       ?create@QWidget@@MAEXPAUHWND__@@_N1@Z 10004594 f   qt-mt323:qt-mt323.dll
 0001:0000359a       ?customEvent@QObject@@MAEXPAVQCustomEvent@@@Z 1000459a f   qt-mt323:qt-mt323.dll
 0001:000035a0       ?customWhatsThis@QWidget@@UBE_NXZ 100045a0 f   qt-mt323:qt-mt323.dll
 0001:000035a6       ?deleteItem@?$QPtrList@VQDockWindow@@@@EAEXPAX@Z 100045a6 f   qt-mt323:qt-mt323.dll
 0001:000035ac       ?destroy@QWidget@@MAEX_N0@Z 100045ac f   qt-mt323:qt-mt323.dll
 0001:000035b2       ?disconnectNotify@QObject@@MAEXPBD@Z 100045b2 f   qt-mt323:qt-mt323.dll
 0001:000035b8       ?dragEnterEvent@QWidget@@MAEXPAVQDragEnterEvent@@@Z 100045b8 f   qt-mt323:qt-mt323.dll
 0001:000035be       ?dragLeaveEvent@QWidget@@MAEXPAVQDragLeaveEvent@@@Z 100045be f   qt-mt323:qt-mt323.dll
 0001:000035c4       ?dragMoveEvent@QWidget@@MAEXPAVQDragMoveEvent@@@Z 100045c4 f   qt-mt323:qt-mt323.dll
 0001:000035ca       ?dropEvent@QWidget@@MAEXPAVQDropEvent@@@Z 100045ca f   qt-mt323:qt-mt323.dll
 0001:000035d0       ?enabledChange@QWidget@@MAEX_N@Z 100045d0 f   qt-mt323:qt-mt323.dll
 0001:000035d6       ?enterEvent@QWidget@@MAEXPAVQEvent@@@Z 100045d6 f   qt-mt323:qt-mt323.dll
 0001:000035dc       ?event@QObject@@UAE_NPAVQEvent@@@Z 100045dc f   qt-mt323:qt-mt323.dll
 0001:000035e2       ?event@QWidget@@MAE_NPAVQEvent@@@Z 100045e2 f   qt-mt323:qt-mt323.dll
 0001:000035e8       ?eventFilter@QObject@@UAE_NPAV1@PAVQEvent@@@Z 100045e8 f   qt-mt323:qt-mt323.dll
 0001:000035ee       ?focusInEvent@QWidget@@MAEXPAVQFocusEvent@@@Z 100045ee f   qt-mt323:qt-mt323.dll
 0001:000035f4       ?focusNextPrevChild@QWidget@@MAE_N_N@Z 100045f4 f   qt-mt323:qt-mt323.dll
 0001:000035fa       ?focusOutEvent@QWidget@@MAEXPAVQFocusEvent@@@Z 100045fa f   qt-mt323:qt-mt323.dll
 0001:00003600       ?fontChange@QWidget@@MAEXABVQFont@@@Z 10004600 f   qt-mt323:qt-mt323.dll
 0001:00003606       ?fontInf@QPaintDevice@@MBEHPAVQFont@@H@Z 10004606 f   qt-mt323:qt-mt323.dll
 0001:0000360c       ?fontMet@QPaintDevice@@MBEHPAVQFont@@HPBDH@Z 1000460c f   qt-mt323:qt-mt323.dll
 0001:00003612       ?handle@QPaintDevice@@UBEPAUHDC__@@XZ 10004612 f   qt-mt323:qt-mt323.dll
 0001:00003618       ?heightForWidth@QWidget@@UBEHH@Z 10004618 f   qt-mt323:qt-mt323.dll
 0001:0000361e       ?hide@QWidget@@UAEXXZ      1000461e f   qt-mt323:qt-mt323.dll
 0001:00003624       ?hideEvent@QWidget@@MAEXPAVQHideEvent@@@Z 10004624 f   qt-mt323:qt-mt323.dll
 0001:0000362a       ?imComposeEvent@QWidget@@MAEXPAVQIMEvent@@@Z 1000462a f   qt-mt323:qt-mt323.dll
 0001:00003630       ?imEndEvent@QWidget@@MAEXPAVQIMEvent@@@Z 10004630 f   qt-mt323:qt-mt323.dll
 0001:00003636       ?imStartEvent@QWidget@@MAEXPAVQIMEvent@@@Z 10004636 f   qt-mt323:qt-mt323.dll
 0001:0000363c       ?insertChild@QObject@@UAEXPAV1@@Z 1000463c f   qt-mt323:qt-mt323.dll
 0001:00003642       ?keyPressEvent@QWidget@@MAEXPAVQKeyEvent@@@Z 10004642 f   qt-mt323:qt-mt323.dll
 0001:00003648       ?keyReleaseEvent@QWidget@@MAEXPAVQKeyEvent@@@Z 10004648 f   qt-mt323:qt-mt323.dll
 0001:0000364e       ?leaveEvent@QWidget@@MAEXPAVQEvent@@@Z 1000464e f   qt-mt323:qt-mt323.dll
 0001:00003654       ?metaObject@QGuardedPtrPrivate@@UBEPAVQMetaObject@@XZ 10004654 f   qt-mt323:qt-mt323.dll
 0001:0000365a       ?metaObject@QWidget@@UBEPAVQMetaObject@@XZ 1000465a f   qt-mt323:qt-mt323.dll
 0001:00003660       ?metric@QWidget@@MBEHH@Z   10004660 f   qt-mt323:qt-mt323.dll
 0001:00003666       ?minimumSizeHint@QWidget@@UBE?AVQSize@@XZ 10004666 f   qt-mt323:qt-mt323.dll
 0001:0000366c       ?mouseDoubleClickEvent@QWidget@@MAEXPAVQMouseEvent@@@Z 1000466c f   qt-mt323:qt-mt323.dll
 0001:00003672       ?mouseMoveEvent@QWidget@@MAEXPAVQMouseEvent@@@Z 10004672 f   qt-mt323:qt-mt323.dll
 0001:00003678       ?mousePressEvent@QWidget@@MAEXPAVQMouseEvent@@@Z 10004678 f   qt-mt323:qt-mt323.dll
 0001:0000367e       ?mouseReleaseEvent@QWidget@@MAEXPAVQMouseEvent@@@Z 1000467e f   qt-mt323:qt-mt323.dll
 0001:00003684       ?move@QWidget@@UAEXHH@Z    10004684 f   qt-mt323:qt-mt323.dll
 0001:0000368a       ?moveEvent@QWidget@@MAEXPAVQMoveEvent@@@Z 1000468a f   qt-mt323:qt-mt323.dll
 0001:00003690       ?newItem@QPtrCollection@@MAEPAXPAX@Z 10004690 f   qt-mt323:qt-mt323.dll
 0001:00003696       ?paintEvent@QWidget@@MAEXPAVQPaintEvent@@@Z 10004696 f   qt-mt323:qt-mt323.dll
 0001:0000369c       ?paletteChange@QWidget@@MAEXABVQPalette@@@Z 1000469c f   qt-mt323:qt-mt323.dll
 0001:000036a2       ?polish@QWidget@@UAEXXZ    100046a2 f   qt-mt323:qt-mt323.dll
 0001:000036a8       ?property@QObject@@UBE?AVQVariant@@PBD@Z 100046a8 f   qt-mt323:qt-mt323.dll
 0001:000036ae       ?qt_cast@QGuardedPtrPrivate@@UAEPAXPBD@Z 100046ae f   qt-mt323:qt-mt323.dll
 0001:000036b4       ?qt_cast@QWidget@@UAEPAXPBD@Z 100046b4 f   qt-mt323:qt-mt323.dll
 0001:000036ba       ?qt_emit@QGuardedPtrPrivate@@UAE_NHPAUQUObject@@@Z 100046ba f   qt-mt323:qt-mt323.dll
 0001:000036c0       ?qt_emit@QWidget@@UAE_NHPAUQUObject@@@Z 100046c0 f   qt-mt323:qt-mt323.dll
 0001:000036c6       ?qt_invoke@QGuardedPtrPrivate@@UAE_NHPAUQUObject@@@Z 100046c6 f   qt-mt323:qt-mt323.dll
 0001:000036cc       ?qt_invoke@QWidget@@UAE_NHPAUQUObject@@@Z 100046cc f   qt-mt323:qt-mt323.dll
 0001:000036d2       ?qt_property@QGuardedPtrPrivate@@UAE_NHHPAVQVariant@@@Z 100046d2 f   qt-mt323:qt-mt323.dll
 0001:000036d8       ?qt_property@QWidget@@UAE_NHHPAVQVariant@@@Z 100046d8 f   qt-mt323:qt-mt323.dll
 0001:000036de       ?read@QGDict@@MAEAAVQDataStream@@AAV2@AAPAX@Z 100046de f   qt-mt323:qt-mt323.dll
 0001:000036e4       ?read@QGList@@MAEAAVQDataStream@@AAV2@AAPAX@Z 100046e4 f   qt-mt323:qt-mt323.dll
 0001:000036ea       ?removeChild@QObject@@UAEXPAV1@@Z 100046ea f   qt-mt323:qt-mt323.dll
 0001:000036f0       ?reparent@QWidget@@UAEXPAV1@IABVQPoint@@_N@Z 100046f0 f   qt-mt323:qt-mt323.dll
 0001:000036f6       ?resize@QWidget@@UAEXHH@Z  100046f6 f   qt-mt323:qt-mt323.dll
 0001:000036fc       ?resizeEvent@QWidget@@MAEXPAVQResizeEvent@@@Z 100046fc f   qt-mt323:qt-mt323.dll
 0001:00003702       ?resolution@QPaintDevice@@UBEHXZ 10004702 f   qt-mt323:qt-mt323.dll
 0001:00003708       ?setAcceptDrops@QWidget@@UAEX_N@Z 10004708 f   qt-mt323:qt-mt323.dll
 0001:0000370e       ?setActiveWindow@QWidget@@UAEXXZ 1000470e f   qt-mt323:qt-mt323.dll
 0001:00003714       ?setAutoMask@QWidget@@UAEX_N@Z 10004714 f   qt-mt323:qt-mt323.dll
 0001:0000371a       ?setBackgroundColor@QWidget@@UAEXABVQColor@@@Z 1000471a f   qt-mt323:qt-mt323.dll
 0001:00003720       ?setBackgroundMode@QWidget@@UAEXW4BackgroundMode@Qt@@@Z 10004720 f   qt-mt323:qt-mt323.dll
 0001:00003726       ?setBackgroundOrigin@QWidget@@UAEXW4BackgroundOrigin@1@@Z 10004726 f   qt-mt323:qt-mt323.dll
 0001:0000372c       ?setBackgroundPixmap@QWidget@@UAEXABVQPixmap@@@Z 1000472c f   qt-mt323:qt-mt323.dll
 0001:00003732       ?setCaption@QWidget@@UAEXABVQString@@@Z 10004732 f   qt-mt323:qt-mt323.dll
 0001:00003738       ?setCursor@QWidget@@UAEXABVQCursor@@@Z 10004738 f   qt-mt323:qt-mt323.dll
 0001:0000373e       ?setEnabled@QWidget@@UAEX_N@Z 1000473e f   qt-mt323:qt-mt323.dll
 0001:00003744       ?setEraseColor@QWidget@@UAEXABVQColor@@@Z 10004744 f   qt-mt323:qt-mt323.dll
 0001:0000374a       ?setErasePixmap@QWidget@@UAEXABVQPixmap@@@Z 1000474a f   qt-mt323:qt-mt323.dll
 0001:00003750       ?setFocus@QWidget@@UAEXXZ  10004750 f   qt-mt323:qt-mt323.dll
 0001:00003756       ?setFocusPolicy@QWidget@@UAEXW4FocusPolicy@1@@Z 10004756 f   qt-mt323:qt-mt323.dll
 0001:0000375c       ?setFocusProxy@QWidget@@UAEXPAV1@@Z 1000475c f   qt-mt323:qt-mt323.dll
 0001:00003762       ?setFont@QWidget@@UAEXABVQFont@@@Z 10004762 f   qt-mt323:qt-mt323.dll
 0001:00003768       ?setGeometry@QWidget@@UAEXABVQRect@@@Z 10004768 f   qt-mt323:qt-mt323.dll
 0001:0000376e       ?setGeometry@QWidget@@UAEXHHHH@Z 1000476e f   qt-mt323:qt-mt323.dll
 0001:00003774       ?setIcon@QWidget@@UAEXABVQPixmap@@@Z 10004774 f   qt-mt323:qt-mt323.dll
 0001:0000377a       ?setIconText@QWidget@@UAEXABVQString@@@Z 1000477a f   qt-mt323:qt-mt323.dll
 0001:00003780       ?setKeyCompression@QWidget@@MAEX_N@Z 10004780 f   qt-mt323:qt-mt323.dll
 0001:00003786       ?setMask@QWidget@@UAEXABVQBitmap@@@Z 10004786 f   qt-mt323:qt-mt323.dll
 0001:0000378c       ?setMask@QWidget@@UAEXABVQRegion@@@Z 1000478c f   qt-mt323:qt-mt323.dll
 0001:00003792       ?setMaximumSize@QWidget@@UAEXHH@Z 10004792 f   qt-mt323:qt-mt323.dll
 0001:00003798       ?setMicroFocusHint@QWidget@@MAEXHHHH_NPAVQFont@@@Z 10004798 f   qt-mt323:qt-mt323.dll
 0001:0000379e       ?setMinimumSize@QWidget@@UAEXHH@Z 1000479e f   qt-mt323:qt-mt323.dll
 0001:000037a4       ?setMouseTracking@QWidget@@UAEX_N@Z 100047a4 f   qt-mt323:qt-mt323.dll
 0001:000037aa       ?setName@QObject@@UAEXPBD@Z 100047aa f   qt-mt323:qt-mt323.dll
 0001:000037b0       ?setPalette@QWidget@@UAEXABVQPalette@@@Z 100047b0 f   qt-mt323:qt-mt323.dll
 0001:000037b6       ?setPaletteBackgroundColor@QWidget@@UAEXABVQColor@@@Z 100047b6 f   qt-mt323:qt-mt323.dll
 0001:000037bc       ?setPaletteBackgroundPixmap@QWidget@@UAEXABVQPixmap@@@Z 100047bc f   qt-mt323:qt-mt323.dll
 0001:000037c2       ?setProperty@QObject@@UAE_NPBDABVQVariant@@@Z 100047c2 f   qt-mt323:qt-mt323.dll
 0001:000037c8       ?setResolution@QPaintDevice@@UAEXH@Z 100047c8 f   qt-mt323:qt-mt323.dll
 0001:000037ce       ?setSizeIncrement@QWidget@@UAEXHH@Z 100047ce f   qt-mt323:qt-mt323.dll
 0001:000037d4       ?setSizePolicy@QWidget@@UAEXVQSizePolicy@@@Z 100047d4 f   qt-mt323:qt-mt323.dll
 0001:000037da       ?setUpdatesEnabled@QWidget@@UAEX_N@Z 100047da f   qt-mt323:qt-mt323.dll
 0001:000037e0       ?setWFlags@QWidget@@MAEXI@Z 100047e0 f   qt-mt323:qt-mt323.dll
 0001:000037e6       ?setWState@QWidget@@MAEXI@Z 100047e6 f   qt-mt323:qt-mt323.dll
 0001:000037ec       ?show@QWidget@@UAEXXZ      100047ec f   qt-mt323:qt-mt323.dll
 0001:000037f2       ?showEvent@QWidget@@MAEXPAVQShowEvent@@@Z 100047f2 f   qt-mt323:qt-mt323.dll
 0001:000037f8       ?showMaximized@QWidget@@UAEXXZ 100047f8 f   qt-mt323:qt-mt323.dll
 0001:000037fe       ?showMinimized@QWidget@@UAEXXZ 100047fe f   qt-mt323:qt-mt323.dll
 0001:00003804       ?showNormal@QWidget@@UAEXXZ 10004804 f   qt-mt323:qt-mt323.dll
 0001:0000380a       ?sizeHint@QWidget@@UBE?AVQSize@@XZ 1000480a f   qt-mt323:qt-mt323.dll
 0001:00003810       ?sizePolicy@QWidget@@UBE?AVQSizePolicy@@XZ 10004810 f   qt-mt323:qt-mt323.dll
 0001:00003816       ?styleChange@QWidget@@MAEXAAVQStyle@@@Z 10004816 f   qt-mt323:qt-mt323.dll
 0001:0000381c       ?tabletEvent@QWidget@@MAEXPAVQTabletEvent@@@Z 1000481c f   qt-mt323:qt-mt323.dll
 0001:00003822       ?timerEvent@QObject@@MAEXPAVQTimerEvent@@@Z 10004822 f   qt-mt323:qt-mt323.dll
 0001:00003828       ?unsetCursor@QWidget@@UAEXXZ 10004828 f   qt-mt323:qt-mt323.dll
 0001:0000382e       ?updateMask@QWidget@@MAEXXZ 1000482e f   qt-mt323:qt-mt323.dll
 0001:00003834       ?wheelEvent@QWidget@@MAEXPAVQWheelEvent@@@Z 10004834 f   qt-mt323:qt-mt323.dll
 0001:0000383a       ?winEvent@QWidget@@MAE_NPAUtagMSG@@@Z 1000483a f   qt-mt323:qt-mt323.dll
 0001:00003840       ?windowActivationChange@QWidget@@MAEX_N@Z 10004840 f   qt-mt323:qt-mt323.dll
 0001:00003846       ?write@QGDict@@MBEAAVQDataStream@@AAV2@PAX@Z 10004846 f   qt-mt323:qt-mt323.dll
 0001:0000384c       ?write@QGList@@MBEAAVQDataStream@@AAV2@PAX@Z 1000484c f   qt-mt323:qt-mt323.dll
 0001:00003852       ?addChild@QScrollView@@UAEXPAVQWidget@@HH@Z 10004852 f   qt-mt323:qt-mt323.dll
 0001:00003858       ?addItem@QBoxLayout@@UAEXPAVQLayoutItem@@@Z 10004858 f   qt-mt323:qt-mt323.dll
 0001:0000385e       ?append@QTextEdit@@UAEXABVQString@@@Z 1000485e f   qt-mt323:qt-mt323.dll
 0001:00003864       ?childEvent@QLayout@@MAEXPAVQChildEvent@@@Z 10004864 f   qt-mt323:qt-mt323.dll
 0001:0000386a       ?className@QHBoxLayout@@UBEPBDXZ 1000486a f   qt-mt323:qt-mt323.dll
 0001:00003870       ?className@QLabel@@UBEPBDXZ 10004870 f   qt-mt323:qt-mt323.dll
 0001:00003876       ?className@QTextEdit@@UBEPBDXZ 10004876 f   qt-mt323:qt-mt323.dll
 0001:0000387c       ?className@QVBoxLayout@@UBEPBDXZ 1000487c f   qt-mt323:qt-mt323.dll
 0001:00003882       ?clear@QTextEdit@@UAEXXZ   10004882 f   qt-mt323:qt-mt323.dll
 0001:00003888       ?clearParagraphBackground@QTextEdit@@UAEXH@Z 10004888 f   qt-mt323:qt-mt323.dll
 0001:0000388e       ?contentsContextMenuEvent@QTextEdit@@MAEXPAVQContextMenuEvent@@@Z 1000488e f   qt-mt323:qt-mt323.dll
 0001:00003894       ?contentsDragEnterEvent@QTextEdit@@MAEXPAVQDragEnterEvent@@@Z 10004894 f   qt-mt323:qt-mt323.dll
 0001:0000389a       ?contentsDragLeaveEvent@QTextEdit@@MAEXPAVQDragLeaveEvent@@@Z 1000489a f   qt-mt323:qt-mt323.dll
 0001:000038a0       ?contentsDragMoveEvent@QTextEdit@@MAEXPAVQDragMoveEvent@@@Z 100048a0 f   qt-mt323:qt-mt323.dll
 0001:000038a6       ?contentsDropEvent@QTextEdit@@MAEXPAVQDropEvent@@@Z 100048a6 f   qt-mt323:qt-mt323.dll
 0001:000038ac       ?contentsMouseDoubleClickEvent@QTextEdit@@MAEXPAVQMouseEvent@@@Z 100048ac f   qt-mt323:qt-mt323.dll
 0001:000038b2       ?contentsMouseMoveEvent@QTextEdit@@MAEXPAVQMouseEvent@@@Z 100048b2 f   qt-mt323:qt-mt323.dll
 0001:000038b8       ?contentsMousePressEvent@QTextEdit@@MAEXPAVQMouseEvent@@@Z 100048b8 f   qt-mt323:qt-mt323.dll
 0001:000038be       ?contentsMouseReleaseEvent@QTextEdit@@MAEXPAVQMouseEvent@@@Z 100048be f   qt-mt323:qt-mt323.dll
 0001:000038c4       ?contentsWheelEvent@QTextEdit@@MAEXPAVQWheelEvent@@@Z 100048c4 f   qt-mt323:qt-mt323.dll
 0001:000038ca       ?contextMenuEvent@QScrollView@@MAEXPAVQContextMenuEvent@@@Z 100048ca f   qt-mt323:qt-mt323.dll
 0001:000038d0       ?copy@QTextEdit@@UAEXXZ    100048d0 f   qt-mt323:qt-mt323.dll
 0001:000038d6       ?createPopupMenu@QTextEdit@@MAEPAVQPopupMenu@@ABVQPoint@@@Z 100048d6 f   qt-mt323:qt-mt323.dll
 0001:000038dc       ?createPopupMenu@QTextEdit@@MAEPAVQPopupMenu@@XZ 100048dc f   qt-mt323:qt-mt323.dll
 0001:000038e2       ?cut@QTextEdit@@UAEXXZ     100048e2 f   qt-mt323:qt-mt323.dll
 0001:000038e8       ?del@QTextEdit@@UAEXXZ     100048e8 f   qt-mt323:qt-mt323.dll
 0001:000038ee       ?doChangeInterval@QTextEdit@@MAEXXZ 100048ee f   qt-mt323:qt-mt323.dll
 0001:000038f4       ?doKeyboardAction@QTextEdit@@UAEXW4KeyboardAction@1@@Z 100048f4 f   qt-mt323:qt-mt323.dll
 0001:000038fa       ?drawContents@QLabel@@MAEXPAVQPainter@@@Z 100048fa f   qt-mt323:qt-mt323.dll
 0001:00003900       ?drawContents@QTextEdit@@EAEXPAVQPainter@@@Z 10004900 f   qt-mt323:qt-mt323.dll
 0001:00003906       ?drawContents@QTextEdit@@MAEXPAVQPainter@@HHHH@Z 10004906 f   qt-mt323:qt-mt323.dll
 0001:0000390c       ?drawContentsOffset@QScrollView@@MAEXPAVQPainter@@HHHHHH@Z 1000490c f   qt-mt323:qt-mt323.dll
 0001:00003912       ?drawFrame@QFrame@@MAEXPAVQPainter@@@Z 10004912 f   qt-mt323:qt-mt323.dll
 0001:00003918       ?emitHighlighted@QTextEdit@@EAEXABVQString@@@Z 10004918 f   qt-mt323:qt-mt323.dll
 0001:0000391e       ?emitLinkClicked@QTextEdit@@EAEXABVQString@@@Z 1000491e f   qt-mt323:qt-mt323.dll
 0001:00003924       ?ensureCursorVisible@QTextEdit@@UAEXXZ 10004924 f   qt-mt323:qt-mt323.dll
 0001:0000392a       ?event@QTextEdit@@MAE_NPAVQEvent@@@Z 1000492a f   qt-mt323:qt-mt323.dll
 0001:00003930       ?eventFilter@QLayout@@MAE_NPAVQObject@@PAVQEvent@@@Z 10004930 f   qt-mt323:qt-mt323.dll
 0001:00003936       ?eventFilter@QTextEdit@@UAE_NPAVQObject@@PAVQEvent@@@Z 10004936 f   qt-mt323:qt-mt323.dll
 0001:0000393c       ?expanding@QBoxLayout@@UBE?AW4ExpandData@QSizePolicy@@XZ 1000493c f   qt-mt323:qt-mt323.dll
 0001:00003942       ?expanding@QSpacerItem@@UBE?AW4ExpandData@QSizePolicy@@XZ 10004942 f   qt-mt323:qt-mt323.dll
 0001:00003948       ?find@QTextEdit@@UAE_NABVQString@@_N11PAH2@Z 10004948 f   qt-mt323:qt-mt323.dll
 0001:0000394e       ?focusNextPrevChild@QTextEdit@@MAE_N_N@Z 1000494e f   qt-mt323:qt-mt323.dll
 0001:00003954       ?fontChange@QLabel@@MAEXABVQFont@@@Z 10004954 f   qt-mt323:qt-mt323.dll
 0001:0000395a       ?fontChange@QScrollView@@MAEXABVQFont@@@Z 1000495a f   qt-mt323:qt-mt323.dll
 0001:00003960       ?frameChanged@QFrame@@MAEXXZ 10004960 f   qt-mt323:qt-mt323.dll
 0001:00003966       ?frameChanged@QScrollView@@MAEXXZ 10004966 f   qt-mt323:qt-mt323.dll
 0001:0000396c       ?geometry@QLayout@@UBE?AVQRect@@XZ 1000496c f   qt-mt323:qt-mt323.dll
 0001:00003972       ?geometry@QSpacerItem@@UBE?AVQRect@@XZ 10004972 f   qt-mt323:qt-mt323.dll
 0001:00003978       ?getFormat@QTextEdit@@UAE_NHHPAVQFont@@PAVQColor@@PAW4VerticalAlignment@1@@Z 10004978 f   qt-mt323:qt-mt323.dll
 0001:0000397e       ?getParagraphFormat@QTextEdit@@UAE_NHPAVQFont@@PAVQColor@@PAW4VerticalAlignment@1@PAHPAW4DisplayMode@QStyleSheetItem@@PAW4ListStyle@6@3@Z 1000497e f   qt-mt323:qt-mt323.dll
 0001:00003984       ?hasHeightForWidth@QBoxLayout@@UBE_NXZ 10004984 f   qt-mt323:qt-mt323.dll
 0001:0000398a       ?hasHeightForWidth@QLayoutItem@@UBE_NXZ 1000498a f   qt-mt323:qt-mt323.dll
 0001:00003990       ?heightForWidth@QBoxLayout@@UBEHH@Z 10004990 f   qt-mt323:qt-mt323.dll
 0001:00003996       ?heightForWidth@QLabel@@UBEHH@Z 10004996 f   qt-mt323:qt-mt323.dll
 0001:0000399c       ?heightForWidth@QLayoutItem@@UBEHH@Z 1000499c f   qt-mt323:qt-mt323.dll
 0001:000039a2       ?heightForWidth@QTextEdit@@UBEHH@Z 100049a2 f   qt-mt323:qt-mt323.dll
 0001:000039a8       ?imComposeEvent@QTextEdit@@MAEXPAVQIMEvent@@@Z 100049a8 f   qt-mt323:qt-mt323.dll
 0001:000039ae       ?imEndEvent@QTextEdit@@MAEXPAVQIMEvent@@@Z 100049ae f   qt-mt323:qt-mt323.dll
 0001:000039b4       ?imStartEvent@QTextEdit@@MAEXPAVQIMEvent@@@Z 100049b4 f   qt-mt323:qt-mt323.dll
 0001:000039ba       ?indent@QTextEdit@@UAEXXZ  100049ba f   qt-mt323:qt-mt323.dll
 0001:000039c0       ?insert@QTextEdit@@UAEXABVQString@@_N11@Z 100049c0 f   qt-mt323:qt-mt323.dll
 0001:000039c6       ?insertAt@QTextEdit@@UAEXABVQString@@HH@Z 100049c6 f   qt-mt323:qt-mt323.dll
 0001:000039cc       ?insertParagraph@QTextEdit@@UAEXABVQString@@H@Z 100049cc f   qt-mt323:qt-mt323.dll
 0001:000039d2       ?invalidate@QBoxLayout@@UAEXXZ 100049d2 f   qt-mt323:qt-mt323.dll
 0001:000039d8       ?invalidate@QLayoutItem@@UAEXXZ 100049d8 f   qt-mt323:qt-mt323.dll
 0001:000039de       ?isEmpty@QLayout@@UBE_NXZ  100049de f   qt-mt323:qt-mt323.dll
 0001:000039e4       ?isEmpty@QSpacerItem@@UBE_NXZ 100049e4 f   qt-mt323:qt-mt323.dll
 0001:000039ea       ?iterator@QBoxLayout@@UAE?AVQLayoutIterator@@XZ 100049ea f   qt-mt323:qt-mt323.dll
 0001:000039f0       ?iterator@QLayoutItem@@UAE?AVQLayoutIterator@@XZ 100049f0 f   qt-mt323:qt-mt323.dll
 0001:000039f6       ?keyPressEvent@QTextEdit@@MAEXPAVQKeyEvent@@@Z 100049f6 f   qt-mt323:qt-mt323.dll
 0001:000039fc       ?layout@QLayout@@UAEPAV1@XZ 100049fc f   qt-mt323:qt-mt323.dll
 0001:00003a02       ?layout@QLayoutItem@@UAEPAVQLayout@@XZ 10004a02 f   qt-mt323:qt-mt323.dll
 0001:00003a08       ?linksEnabled@QTextEdit@@EBE_NXZ 10004a08 f   qt-mt323:qt-mt323.dll
 0001:00003a0e       ?maximumSize@QBoxLayout@@UBE?AVQSize@@XZ 10004a0e f   qt-mt323:qt-mt323.dll
 0001:00003a14       ?maximumSize@QSpacerItem@@UBE?AVQSize@@XZ 10004a14 f   qt-mt323:qt-mt323.dll
 0001:00003a1a       ?metaObject@QHBoxLayout@@UBEPAVQMetaObject@@XZ 10004a1a f   qt-mt323:qt-mt323.dll
 0001:00003a20       ?metaObject@QLabel@@UBEPAVQMetaObject@@XZ 10004a20 f   qt-mt323:qt-mt323.dll
 0001:00003a26       ?metaObject@QTextEdit@@UBEPAVQMetaObject@@XZ 10004a26 f   qt-mt323:qt-mt323.dll
 0001:00003a2c       ?metaObject@QVBoxLayout@@UBEPAVQMetaObject@@XZ 10004a2c f   qt-mt323:qt-mt323.dll
 0001:00003a32       ?minimumSize@QBoxLayout@@UBE?AVQSize@@XZ 10004a32 f   qt-mt323:qt-mt323.dll
 0001:00003a38       ?minimumSize@QSpacerItem@@UBE?AVQSize@@XZ 10004a38 f   qt-mt323:qt-mt323.dll
 0001:00003a3e       ?minimumSizeHint@QLabel@@UBE?AVQSize@@XZ 10004a3e f   qt-mt323:qt-mt323.dll
 0001:00003a44       ?minimumSizeHint@QScrollView@@UBE?AVQSize@@XZ 10004a44 f   qt-mt323:qt-mt323.dll
 0001:00003a4a       ?mouseDoubleClickEvent@QScrollView@@MAEXPAVQMouseEvent@@@Z 10004a4a f   qt-mt323:qt-mt323.dll
 0001:00003a50       ?mouseMoveEvent@QScrollView@@MAEXPAVQMouseEvent@@@Z 10004a50 f   qt-mt323:qt-mt323.dll
 0001:00003a56       ?mousePressEvent@QScrollView@@MAEXPAVQMouseEvent@@@Z 10004a56 f   qt-mt323:qt-mt323.dll
 0001:00003a5c       ?mouseReleaseEvent@QScrollView@@MAEXPAVQMouseEvent@@@Z 10004a5c f   qt-mt323:qt-mt323.dll
 0001:00003a62       ?moveChild@QScrollView@@UAEXPAVQWidget@@HH@Z 10004a62 f   qt-mt323:qt-mt323.dll
 0001:00003a68       ?moveCursor@QTextEdit@@UAEXW4CursorAction@1@_N@Z 10004a68 f   qt-mt323:qt-mt323.dll
 0001:00003a6e       ?paintEvent@QFrame@@MAEXPAVQPaintEvent@@@Z 10004a6e f   qt-mt323:qt-mt323.dll
 0001:00003a74       ?paste@QTextEdit@@UAEXXZ   10004a74 f   qt-mt323:qt-mt323.dll
 0001:00003a7a       ?pasteSubType@QTextEdit@@UAEXABVQCString@@@Z 10004a7a f   qt-mt323:qt-mt323.dll
 0001:00003a80       ?placeCursor@QTextEdit@@UAEXABVQPoint@@PAVQTextCursor@@@Z 10004a80 f   qt-mt323:qt-mt323.dll
 0001:00003a86       ?polish@QTextEdit@@UAEXXZ  10004a86 f   qt-mt323:qt-mt323.dll
 0001:00003a8c       ?qt_cast@QHBoxLayout@@UAEPAXPBD@Z 10004a8c f   qt-mt323:qt-mt323.dll
 0001:00003a92       ?qt_cast@QLabel@@UAEPAXPBD@Z 10004a92 f   qt-mt323:qt-mt323.dll
 0001:00003a98       ?qt_cast@QTextEdit@@UAEPAXPBD@Z 10004a98 f   qt-mt323:qt-mt323.dll
 0001:00003a9e       ?qt_cast@QVBoxLayout@@UAEPAXPBD@Z 10004a9e f   qt-mt323:qt-mt323.dll
 0001:00003aa4       ?qt_emit@QHBoxLayout@@UAE_NHPAUQUObject@@@Z 10004aa4 f   qt-mt323:qt-mt323.dll
 0001:00003aaa       ?qt_emit@QLabel@@UAE_NHPAUQUObject@@@Z 10004aaa f   qt-mt323:qt-mt323.dll
 0001:00003ab0       ?qt_emit@QTextEdit@@UAE_NHPAUQUObject@@@Z 10004ab0 f   qt-mt323:qt-mt323.dll
 0001:00003ab6       ?qt_emit@QVBoxLayout@@UAE_NHPAUQUObject@@@Z 10004ab6 f   qt-mt323:qt-mt323.dll
 0001:00003abc       ?qt_invoke@QHBoxLayout@@UAE_NHPAUQUObject@@@Z 10004abc f   qt-mt323:qt-mt323.dll
 0001:00003ac2       ?qt_invoke@QLabel@@UAE_NHPAUQUObject@@@Z 10004ac2 f   qt-mt323:qt-mt323.dll
 0001:00003ac8       ?qt_invoke@QTextEdit@@UAE_NHPAUQUObject@@@Z 10004ac8 f   qt-mt323:qt-mt323.dll
 0001:00003ace       ?qt_invoke@QVBoxLayout@@UAE_NHPAUQUObject@@@Z 10004ace f   qt-mt323:qt-mt323.dll
 0001:00003ad4       ?qt_property@QHBoxLayout@@UAE_NHHPAVQVariant@@@Z 10004ad4 f   qt-mt323:qt-mt323.dll
 0001:00003ada       ?qt_property@QLabel@@UAE_NHHPAVQVariant@@@Z 10004ada f   qt-mt323:qt-mt323.dll
 0001:00003ae0       ?qt_property@QTextEdit@@UAE_NHHPAVQVariant@@@Z 10004ae0 f   qt-mt323:qt-mt323.dll
 0001:00003ae6       ?qt_property@QVBoxLayout@@UAE_NHHPAVQVariant@@@Z 10004ae6 f   qt-mt323:qt-mt323.dll
 0001:00003aec       ?redo@QTextEdit@@UAEXXZ    10004aec f   qt-mt323:qt-mt323.dll
 0001:00003af2       ?removeChild@QScrollView@@UAEXPAVQObject@@@Z 10004af2 f   qt-mt323:qt-mt323.dll
 0001:00003af8       ?removeParagraph@QTextEdit@@UAEXH@Z 10004af8 f   qt-mt323:qt-mt323.dll
 0001:00003afe       ?removeSelectedText@QTextEdit@@UAEXH@Z 10004afe f   qt-mt323:qt-mt323.dll
 0001:00003b04       ?removeSelection@QTextEdit@@UAEXH@Z 10004b04 f   qt-mt323:qt-mt323.dll
 0001:00003b0a       ?resetFormat@QTextEdit@@UAEXXZ 10004b0a f   qt-mt323:qt-mt323.dll
 0001:00003b10       ?resize@QScrollView@@UAEXHH@Z 10004b10 f   qt-mt323:qt-mt323.dll
 0001:00003b16       ?resizeContents@QScrollView@@UAEXHH@Z 10004b16 f   qt-mt323:qt-mt323.dll
 0001:00003b1c       ?resizeEvent@QLabel@@MAEXPAVQResizeEvent@@@Z 10004b1c f   qt-mt323:qt-mt323.dll
 0001:00003b22       ?resizeEvent@QTextEdit@@MAEXPAVQResizeEvent@@@Z 10004b22 f   qt-mt323:qt-mt323.dll
 0001:00003b28       ?scrollToAnchor@QTextEdit@@UAEXABVQString@@@Z 10004b28 f   qt-mt323:qt-mt323.dll
 0001:00003b2e       ?scrollToBottom@QTextEdit@@UAEXXZ 10004b2e f   qt-mt323:qt-mt323.dll
 0001:00003b34       ?selectAll@QTextEdit@@UAEX_N@Z 10004b34 f   qt-mt323:qt-mt323.dll
 0001:00003b3a       ?setAlignment@QLabel@@UAEXH@Z 10004b3a f   qt-mt323:qt-mt323.dll
 0001:00003b40       ?setAlignment@QLayoutItem@@UAEXH@Z 10004b40 f   qt-mt323:qt-mt323.dll
 0001:00003b46       ?setAlignment@QTextEdit@@UAEXH@Z 10004b46 f   qt-mt323:qt-mt323.dll
 0001:00003b4c       ?setAutoAdd@QLayout@@UAEX_N@Z 10004b4c f   qt-mt323:qt-mt323.dll
 0001:00003b52       ?setAutoResize@QLabel@@UAEX_N@Z 10004b52 f   qt-mt323:qt-mt323.dll
 0001:00003b58       ?setBold@QTextEdit@@UAEX_N@Z 10004b58 f   qt-mt323:qt-mt323.dll
 0001:00003b5e       ?setBuddy@QLabel@@UAEXPAVQWidget@@@Z 10004b5e f   qt-mt323:qt-mt323.dll
 0001:00003b64       ?setColor@QTextEdit@@UAEXABVQColor@@@Z 10004b64 f   qt-mt323:qt-mt323.dll
 0001:00003b6a       ?setContentsPos@QScrollView@@UAEXHH@Z 10004b6a f   qt-mt323:qt-mt323.dll
 0001:00003b70       ?setCornerWidget@QScrollView@@UAEXPAVQWidget@@@Z 10004b70 f   qt-mt323:qt-mt323.dll
 0001:00003b76       ?setCurrentFont@QTextEdit@@UAEXABVQFont@@@Z 10004b76 f   qt-mt323:qt-mt323.dll
 0001:00003b7c       ?setCursorPosition@QTextEdit@@UAEXHH@Z 10004b7c f   qt-mt323:qt-mt323.dll
 0001:00003b82       ?setDragAutoScroll@QScrollView@@UAEX_N@Z 10004b82 f   qt-mt323:qt-mt323.dll
 0001:00003b88       ?setEnabled@QTextEdit@@UAEX_N@Z 10004b88 f   qt-mt323:qt-mt323.dll
 0001:00003b8e       ?setFamily@QTextEdit@@UAEXABVQString@@@Z 10004b8e f   qt-mt323:qt-mt323.dll
 0001:00003b94       ?setFont@QLabel@@UAEXABVQFont@@@Z 10004b94 f   qt-mt323:qt-mt323.dll
 0001:00003b9a       ?setFont@QTextEdit@@UAEXABVQFont@@@Z 10004b9a f   qt-mt323:qt-mt323.dll
 0001:00003ba0       ?setFormat@QTextEdit@@UAEXPAVQTextFormat@@H@Z 10004ba0 f   qt-mt323:qt-mt323.dll
 0001:00003ba6       ?setFrameRect@QFrame@@UAEXABVQRect@@@Z 10004ba6 f   qt-mt323:qt-mt323.dll
 0001:00003bac       ?setFrameStyle@QFrame@@UAEXH@Z 10004bac f   qt-mt323:qt-mt323.dll
 0001:00003bb2       ?setGeometry@QBoxLayout@@UAEXABVQRect@@@Z 10004bb2 f   qt-mt323:qt-mt323.dll
 0001:00003bb8       ?setGeometry@QSpacerItem@@UAEXABVQRect@@@Z 10004bb8 f   qt-mt323:qt-mt323.dll
 0001:00003bbe       ?setHBarGeometry@QScrollView@@MAEXAAVQScrollBar@@HHHH@Z 10004bbe f   qt-mt323:qt-mt323.dll
 0001:00003bc4       ?setHScrollBarMode@QScrollView@@UAEXW4ScrollBarMode@1@@Z 10004bc4 f   qt-mt323:qt-mt323.dll
 0001:00003bca       ?setItalic@QTextEdit@@UAEX_N@Z 10004bca f   qt-mt323:qt-mt323.dll
 0001:00003bd0       ?setLineWidth@QFrame@@UAEXH@Z 10004bd0 f   qt-mt323:qt-mt323.dll
 0001:00003bd6       ?setLinkUnderline@QTextEdit@@UAEX_N@Z 10004bd6 f   qt-mt323:qt-mt323.dll
 0001:00003bdc       ?setMargin@QFrame@@UAEXH@Z 10004bdc f   qt-mt323:qt-mt323.dll
 0001:00003be2       ?setMargin@QLayout@@UAEXH@Z 10004be2 f   qt-mt323:qt-mt323.dll
 0001:00003be8       ?setMargins@QScrollView@@MAEXHHHH@Z 10004be8 f   qt-mt323:qt-mt323.dll
 0001:00003bee       ?setMenuBar@QLayout@@UAEXPAVQMenuBar@@@Z 10004bee f   qt-mt323:qt-mt323.dll
 0001:00003bf4       ?setMidLineWidth@QFrame@@UAEXH@Z 10004bf4 f   qt-mt323:qt-mt323.dll
 0001:00003bfa       ?setMimeSourceFactory@QTextEdit@@UAEXPAVQMimeSourceFactory@@@Z 10004bfa f   qt-mt323:qt-mt323.dll
 0001:00003c00       ?setModified@QTextEdit@@UAEX_N@Z 10004c00 f   qt-mt323:qt-mt323.dll
 0001:00003c06       ?setMovie@QLabel@@UAEXABVQMovie@@@Z 10004c06 f   qt-mt323:qt-mt323.dll
 0001:00003c0c       ?setNum@QLabel@@UAEXH@Z    10004c0c f   qt-mt323:qt-mt323.dll
 0001:00003c12       ?setNum@QLabel@@UAEXN@Z    10004c12 f   qt-mt323:qt-mt323.dll
 0001:00003c18       ?setOverwriteMode@QTextEdit@@UAEX_N@Z 10004c18 f   qt-mt323:qt-mt323.dll
 0001:00003c1e       ?setPalette@QTextEdit@@UAEXABVQPalette@@@Z 10004c1e f   qt-mt323:qt-mt323.dll
 0001:00003c24       ?setPaper@QTextEdit@@UAEXABVQBrush@@@Z 10004c24 f   qt-mt323:qt-mt323.dll
 0001:00003c2a       ?setParagType@QTextEdit@@UAEXW4DisplayMode@QStyleSheetItem@@W4ListStyle@3@@Z 10004c2a f   qt-mt323:qt-mt323.dll
 0001:00003c30       ?setParagraphBackgroundColor@QTextEdit@@UAEXHABVQColor@@@Z 10004c30 f   qt-mt323:qt-mt323.dll
 0001:00003c36       ?setPicture@QLabel@@UAEXABVQPicture@@@Z 10004c36 f   qt-mt323:qt-mt323.dll
 0001:00003c3c       ?setPixmap@QLabel@@UAEXABVQPixmap@@@Z 10004c3c f   qt-mt323:qt-mt323.dll
 0001:00003c42       ?setPointSize@QTextEdit@@UAEXH@Z 10004c42 f   qt-mt323:qt-mt323.dll
 0001:00003c48       ?setReadOnly@QTextEdit@@UAEX_N@Z 10004c48 f   qt-mt323:qt-mt323.dll
 0001:00003c4e       ?setResizePolicy@QScrollView@@UAEXW4ResizePolicy@1@@Z 10004c4e f   qt-mt323:qt-mt323.dll
 0001:00003c54       ?setSelection@QTextEdit@@UAEXHHHHH@Z 10004c54 f   qt-mt323:qt-mt323.dll
 0001:00003c5a       ?setSelectionAttributes@QTextEdit@@UAEXHABVQColor@@_N@Z 10004c5a f   qt-mt323:qt-mt323.dll
 0001:00003c60       ?setSpacing@QLayout@@UAEXH@Z 10004c60 f   qt-mt323:qt-mt323.dll
 0001:00003c66       ?setStyleSheet@QTextEdit@@UAEXPAVQStyleSheet@@@Z 10004c66 f   qt-mt323:qt-mt323.dll
 0001:00003c6c       ?setTabStopWidth@QTextEdit@@UAEXH@Z 10004c6c f   qt-mt323:qt-mt323.dll
 0001:00003c72       ?setText@QLabel@@UAEXABVQString@@@Z 10004c72 f   qt-mt323:qt-mt323.dll
 0001:00003c78       ?setText@QTextEdit@@UAEXABVQString@@0@Z 10004c78 f   qt-mt323:qt-mt323.dll
 0001:00003c7e       ?setTextFormat@QTextEdit@@UAEXW4TextFormat@Qt@@@Z 10004c7e f   qt-mt323:qt-mt323.dll
 0001:00003c84       ?setUnderline@QTextEdit@@UAEX_N@Z 10004c84 f   qt-mt323:qt-mt323.dll
 0001:00003c8a       ?setUndoDepth@QTextEdit@@UAEXH@Z 10004c8a f   qt-mt323:qt-mt323.dll
 0001:00003c90       ?setUndoRedoEnabled@QTextEdit@@UAEX_N@Z 10004c90 f   qt-mt323:qt-mt323.dll
 0001:00003c96       ?setVBarGeometry@QScrollView@@MAEXAAVQScrollBar@@HHHH@Z 10004c96 f   qt-mt323:qt-mt323.dll
 0001:00003c9c       ?setVScrollBarMode@QScrollView@@UAEXW4ScrollBarMode@1@@Z 10004c9c f   qt-mt323:qt-mt323.dll
 0001:00003ca2       ?setVerticalAlignment@QTextEdit@@UAEXW4VerticalAlignment@1@@Z 10004ca2 f   qt-mt323:qt-mt323.dll
 0001:00003ca8       ?setWordWrap@QTextEdit@@UAEXW4WordWrap@1@@Z 10004ca8 f   qt-mt323:qt-mt323.dll
 0001:00003cae       ?setWrapColumnOrWidth@QTextEdit@@UAEXH@Z 10004cae f   qt-mt323:qt-mt323.dll
 0001:00003cb4       ?setWrapPolicy@QTextEdit@@UAEXW4WrapPolicy@1@@Z 10004cb4 f   qt-mt323:qt-mt323.dll
 0001:00003cba       ?show@QScrollView@@UAEXXZ  10004cba f   qt-mt323:qt-mt323.dll
 0001:00003cc0       ?sizeHint@QBoxLayout@@UBE?AVQSize@@XZ 10004cc0 f   qt-mt323:qt-mt323.dll
 0001:00003cc6       ?sizeHint@QLabel@@UBE?AVQSize@@XZ 10004cc6 f   qt-mt323:qt-mt323.dll
 0001:00003ccc       ?sizeHint@QSpacerItem@@UBE?AVQSize@@XZ 10004ccc f   qt-mt323:qt-mt323.dll
 0001:00003cd2       ?sizeHint@QTextEdit@@UBE?AVQSize@@XZ 10004cd2 f   qt-mt323:qt-mt323.dll
 0001:00003cd8       ?spacerItem@QLayoutItem@@UAEPAVQSpacerItem@@XZ 10004cd8 f   qt-mt323:qt-mt323.dll
 0001:00003cde       ?spacerItem@QSpacerItem@@UAEPAV1@XZ 10004cde f   qt-mt323:qt-mt323.dll
 0001:00003ce4       ?styleChange@QFrame@@MAEXAAVQStyle@@@Z 10004ce4 f   qt-mt323:qt-mt323.dll
 0001:00003cea       ?styleChange@QScrollView@@UAEXAAVQStyle@@@Z 10004cea f   qt-mt323:qt-mt323.dll
 0001:00003cf0       ?sync@QTextEdit@@UAEXXZ    10004cf0 f   qt-mt323:qt-mt323.dll
 0001:00003cf6       ?undo@QTextEdit@@UAEXXZ    10004cf6 f   qt-mt323:qt-mt323.dll
 0001:00003cfc       ?viewportContextMenuEvent@QScrollView@@MAEXPAVQContextMenuEvent@@@Z 10004cfc f   qt-mt323:qt-mt323.dll
 0001:00003d02       ?viewportDragEnterEvent@QScrollView@@MAEXPAVQDragEnterEvent@@@Z 10004d02 f   qt-mt323:qt-mt323.dll
 0001:00003d08       ?viewportDragLeaveEvent@QScrollView@@MAEXPAVQDragLeaveEvent@@@Z 10004d08 f   qt-mt323:qt-mt323.dll
 0001:00003d0e       ?viewportDragMoveEvent@QScrollView@@MAEXPAVQDragMoveEvent@@@Z 10004d0e f   qt-mt323:qt-mt323.dll
 0001:00003d14       ?viewportDropEvent@QScrollView@@MAEXPAVQDropEvent@@@Z 10004d14 f   qt-mt323:qt-mt323.dll
 0001:00003d1a       ?viewportMouseDoubleClickEvent@QScrollView@@MAEXPAVQMouseEvent@@@Z 10004d1a f   qt-mt323:qt-mt323.dll
 0001:00003d20       ?viewportMouseMoveEvent@QScrollView@@MAEXPAVQMouseEvent@@@Z 10004d20 f   qt-mt323:qt-mt323.dll
 0001:00003d26       ?viewportMousePressEvent@QScrollView@@MAEXPAVQMouseEvent@@@Z 10004d26 f   qt-mt323:qt-mt323.dll
 0001:00003d2c       ?viewportMouseReleaseEvent@QScrollView@@MAEXPAVQMouseEvent@@@Z 10004d2c f   qt-mt323:qt-mt323.dll
 0001:00003d32       ?viewportPaintEvent@QScrollView@@MAEXPAVQPaintEvent@@@Z 10004d32 f   qt-mt323:qt-mt323.dll
 0001:00003d38       ?viewportResizeEvent@QTextEdit@@MAEXPAVQResizeEvent@@@Z 10004d38 f   qt-mt323:qt-mt323.dll
 0001:00003d3e       ?viewportWheelEvent@QScrollView@@MAEXPAVQWheelEvent@@@Z 10004d3e f   qt-mt323:qt-mt323.dll
 0001:00003d44       ?wheelEvent@QScrollView@@MAEXPAVQWheelEvent@@@Z 10004d44 f   qt-mt323:qt-mt323.dll
 0001:00003d4a       ?widget@QLayoutItem@@UAEPAVQWidget@@XZ 10004d4a f   qt-mt323:qt-mt323.dll
 0001:00003d50       ?windowActivationChange@QTextEdit@@MAEX_N@Z 10004d50 f   qt-mt323:qt-mt323.dll
 0001:00003d56       ?zoomIn@QTextEdit@@UAEXH@Z 10004d56 f   qt-mt323:qt-mt323.dll
 0001:00003d5c       ?zoomIn@QTextEdit@@UAEXXZ  10004d5c f   qt-mt323:qt-mt323.dll
 0001:00003d62       ?zoomOut@QTextEdit@@UAEXH@Z 10004d62 f   qt-mt323:qt-mt323.dll
 0001:00003d68       ?zoomOut@QTextEdit@@UAEXXZ 10004d68 f   qt-mt323:qt-mt323.dll
 0001:00003d6e       ?zoomTo@QTextEdit@@UAEXH@Z 10004d6e f   qt-mt323:qt-mt323.dll
 0001:00003d74       ??3@YAXPAX@Z               10004d74 f   MSVCRT:MSVCR120.dll
 0001:00003d7a       @__security_check_cookie@4 10004d7a f   MSVCRT:secchk.obj
 0001:00003d89       __EH_epilog3               10004d89 f   MSVCRT:ehprolg3.obj
 0001:00003d9d       __EH_epilog3_GS            10004d9d f   MSVCRT:ehprolg3.obj
 0001:00003dac       __EH_prolog3               10004dac f   MSVCRT:ehprolg3.obj
 0001:00003ddf       __EH_prolog3_GS            10004ddf f   MSVCRT:ehprolg3.obj
 0001:00003e16       ___CxxFrameHandler3        10004e16 f   MSVCRT:MSVCR120.dll
 0001:00003e1c       ??_Etype_info@@UAEPAXI@Z   10004e1c f i MSVCRT:ti_inst.obj
 0001:00003e66       __purecall                 10004e66 f   MSVCRT:MSVCR120.dll
 0001:00003e6c       ??2@YAPAXI@Z               10004e6c f   MSVCRT:MSVCR120.dll
 0001:00003e72       ??_L@YGXPAXIHP6EX0@Z1@Z    10004e72 f   MSVCRT:ehvecctr.obj
 0001:00003ed4       ??_M@YGXPAXIHP6EX0@Z@Z     10004ed4 f   MSVCRT:ehvecdtr.obj
 0001:00003f43       ?__ArrayUnwind@@YGXPAXIHP6EX0@Z@Z 10004f43 f   MSVCRT:ehvecdtr.obj
 0001:00003fa1       ___atonexitinit            10004fa1 f   MSVCRT:atonexit.obj
 0001:00003fdd       __onexit                   10004fdd f   MSVCRT:atonexit.obj
 0001:00004086       _atexit                    10005086 f   MSVCRT:atonexit.obj
 0001:000040e7       __CRT_INIT@12              100050e7 f   MSVCRT:crtdll.obj
 0001:000042de       __DllMainCRTStartup@12     100052de f   MSVCRT:crtdll.obj
 0001:00004434       ___raise_securityfailure   10005434 f   MSVCRT:gs_report.obj
 0001:00004471       ___report_gsfailure        10005471 f   MSVCRT:gs_report.obj
 0001:0000456c       ??1type_info@@UAE@XZ       1000556c f   MSVCRT:MSVCR120.dll
 0001:00004580       __SEH_prolog4              10005580 f   MSVCRT:sehprolg4.obj
 0001:000045c5       __SEH_epilog4              100055c5 f   MSVCRT:sehprolg4.obj
 0001:000045d9       __except_handler4          100055d9 f   MSVCRT:chandler4gs.obj
 0001:000045fc       ?terminate@@YAXXZ          100055fc f   MSVCRT:MSVCR120.dll
 0001:00004602       __lock                     10005602 f   MSVCRT:MSVCR120.dll
 0001:00004608       __unlock                   10005608 f   MSVCRT:MSVCR120.dll
 0001:0000460e       ___dllonexit               1000560e f   MSVCRT:MSVCR120.dll
 0001:00004614       ___CppXcptFilter           10005614 f   MSVCRT:MSVCR120.dll
 0001:0000461a       __amsg_exit                1000561a f   MSVCRT:MSVCR120.dll
 0001:00004620       __FindPESection            10005620 f   MSVCRT:pesect.obj
 0001:00004670       __IsNonwritableInCurrentImage 10005670 f   MSVCRT:pesect.obj
 0001:00004730       __ValidateImageBase        10005730 f   MSVCRT:pesect.obj
 0001:00004761       ___security_init_cookie    10005761 f   MSVCRT:gs_support.obj
 0001:000047fd       _DllMain@12                100057fd f   MSVCRT:dllmain.obj
 0001:0000481f       __RTC_Initialize           1000581f f   MSVCRT:initsect.obj
 0001:0000483f       __RTC_Terminate            1000583f f   MSVCRT:initsect.obj
 0001:00004860       __initterm                 10005860 f   MSVCRT:MSVCR120.dll
 0001:00004866       __initterm_e               10005866 f   MSVCRT:MSVCR120.dll
 0001:0000486c       ___clean_type_info_names   1000586c f   MSVCRT:tncleanup.obj
 0001:00004878       __crt_debugger_hook        10005878 f   MSVCRT:MSVCR120.dll
 0001:0000487e       ___crtUnhandledException   1000587e f   MSVCRT:MSVCR120.dll
 0001:00004884       ___crtTerminateProcess     10005884 f   MSVCRT:MSVCR120.dll
 0001:0000488a       __except_handler4_common   1000588a f   MSVCRT:MSVCR120.dll
 0001:00004890       ___clean_type_info_names_internal 10005890 f   MSVCRT:MSVCR120.dll
 0001:00004896       _IsProcessorFeaturePresent@4 10005896 f   kernel32:KERNEL32.dll
 0002:00000000       __imp__GetSystemTimeAsFileTime@4 10007000     kernel32:KERNEL32.dll
 0002:00000004       __imp__GetCurrentThreadId@0 10007004     kernel32:KERNEL32.dll
 0002:00000008       __imp__GetCurrentProcessId@0 10007008     kernel32:KERNEL32.dll
 0002:0000000c       __imp__QueryPerformanceCounter@4 1000700c     kernel32:KERNEL32.dll
 0002:00000010       __imp__IsProcessorFeaturePresent@4 10007010     kernel32:KERNEL32.dll
 0002:00000014       __imp__IsDebuggerPresent@0 10007014     kernel32:KERNEL32.dll
 0002:00000018       __imp__DecodePointer@4     10007018     kernel32:KERNEL32.dll
 0002:0000001c       __imp__EncodePointer@4     1000701c     kernel32:KERNEL32.dll
 0002:00000020       __imp__DisableThreadLibraryCalls@4 10007020     kernel32:KERNEL32.dll
 0002:00000024       \177KERNEL32_NULL_THUNK_DATA 10007024     kernel32:KERNEL32.dll
 0002:00000028       __imp____clean_type_info_names_internal 10007028     MSVCRT:MSVCR120.dll
 0002:0000002c       __imp____crtTerminateProcess 1000702c     MSVCRT:MSVCR120.dll
 0002:00000030       __imp____crtUnhandledException 10007030     MSVCRT:MSVCR120.dll
 0002:00000034       __imp___crt_debugger_hook  10007034     MSVCRT:MSVCR120.dll
 0002:00000038       __imp___initterm_e         10007038     MSVCRT:MSVCR120.dll
 0002:0000003c       __imp___initterm           1000703c     MSVCRT:MSVCR120.dll
 0002:00000040       __imp___malloc_crt         10007040     MSVCRT:MSVCR120.dll
 0002:00000044       __imp__free                10007044     MSVCRT:MSVCR120.dll
 0002:00000048       __imp___amsg_exit          10007048     MSVCRT:MSVCR120.dll
 0002:0000004c       __imp____CppXcptFilter     1000704c     MSVCRT:MSVCR120.dll
 0002:00000050       __imp___onexit             10007050     MSVCRT:MSVCR120.dll
 0002:00000054       __imp____dllonexit         10007054     MSVCRT:MSVCR120.dll
 0002:00000058       __imp___calloc_crt         10007058     MSVCRT:MSVCR120.dll
 0002:0000005c       __imp___unlock             1000705c     MSVCRT:MSVCR120.dll
 0002:00000060       __imp___lock               10007060     MSVCRT:MSVCR120.dll
 0002:00000064       __imp_?terminate@@YAXXZ    10007064     MSVCRT:MSVCR120.dll
 0002:00000068       __imp_??1type_info@@UAE@XZ 10007068     MSVCRT:MSVCR120.dll
 0002:0000006c       __imp_??2@YAPAXI@Z         1000706c     MSVCRT:MSVCR120.dll
 0002:00000070       __imp___purecall           10007070     MSVCRT:MSVCR120.dll
 0002:00000074       __imp____CxxFrameHandler3  10007074     MSVCRT:MSVCR120.dll
 0002:00000078       __imp_??3@YAXPAX@Z         10007078     MSVCRT:MSVCR120.dll
 0002:0000007c       __imp___except_handler4_common 1000707c     MSVCRT:MSVCR120.dll
 0002:00000080       \177MSVCR120_NULL_THUNK_DATA 10007080     MSVCRT:MSVCR120.dll
 0002:00000084       __imp_??4QString@@QAEAAV0@PBD@Z 10007084     qt-mt323:qt-mt323.dll
 0002:00000088       __imp_?upper@QString@@QBE?AV1@XZ 10007088     qt-mt323:qt-mt323.dll
 0002:0000008c       __imp_?stripWhiteSpace@QString@@QBE?AV1@XZ 1000708c     qt-mt323:qt-mt323.dll
 0002:00000090       __imp_??YQString@@QAEAAV0@VQChar@@@Z 10007090     qt-mt323:qt-mt323.dll
 0002:00000094       __imp_?startsWith@QString@@QBE_NABV1@@Z 10007094     qt-mt323:qt-mt323.dll
 0002:00000098       __imp_?begin@?$QValueList@VQString@@@@QAE?AV?$QValueListIterator@VQString@@@@XZ 10007098     qt-mt323:qt-mt323.dll
 0002:0000009c       __imp_?find@?$QValueList@VQString@@@@QAE?AV?$QValueListIterator@VQString@@@@ABVQString@@@Z 1000709c     qt-mt323:qt-mt323.dll
 0002:000000a0       __imp_?detachInternal@?$QValueList@VQString@@@@AAEXXZ 100070a0     qt-mt323:qt-mt323.dll
 0002:000000a4       __imp_??0QColor@@QAE@PBD@Z 100070a4     qt-mt323:qt-mt323.dll
 0002:000000a8       __imp_??0QSyntaxHighlighter@@QAE@PAVQTextEdit@@@Z 100070a8     qt-mt323:qt-mt323.dll
 0002:000000ac       __imp_??1QSyntaxHighlighter@@UAE@XZ 100070ac     qt-mt323:qt-mt323.dll
 0002:000000b0       __imp_?setFormat@QSyntaxHighlighter@@QAEXHHABVQColor@@@Z 100070b0     qt-mt323:qt-mt323.dll
 0002:000000b4       __imp_?null@QChar@@2V1@A   100070b4     qt-mt323:qt-mt323.dll
 0002:000000b8       __imp_?qDebug@@YAXPBDZZ    100070b8     qt-mt323:qt-mt323.dll
 0002:000000bc       __imp_?arg@QString@@QBE?AV1@HHH@Z 100070bc     qt-mt323:qt-mt323.dll
 0002:000000c0       __imp_?arg@QString@@QBE?AV1@ABV1@H@Z 100070c0     qt-mt323:qt-mt323.dll
 0002:000000c4       __imp_?ascii@QString@@QBEPBDXZ 100070c4     qt-mt323:qt-mt323.dll
 0002:000000c8       __imp_?endsWith@QString@@QBE_NABV1@@Z 100070c8     qt-mt323:qt-mt323.dll
 0002:000000cc       __imp_??8@YA_NABVQString@@PBD@Z 100070cc     qt-mt323:qt-mt323.dll
 0002:000000d0       __imp_??H@YA?BVQString@@ABV0@0@Z 100070d0     qt-mt323:qt-mt323.dll
 0002:000000d4       __imp_??H@YA?BVQString@@PBDABV0@@Z 100070d4     qt-mt323:qt-mt323.dll
 0002:000000d8       __imp_??0QGList@@IAE@XZ    100070d8     qt-mt323:qt-mt323.dll
 0002:000000dc       __imp_??1QGList@@MAE@XZ    100070dc     qt-mt323:qt-mt323.dll
 0002:000000e0       __imp_?append@QGList@@IAEXPAX@Z 100070e0     qt-mt323:qt-mt323.dll
 0002:000000e4       __imp_?clear@QGList@@MAEXXZ 100070e4     qt-mt323:qt-mt323.dll
 0002:000000e8       __imp_?connect@QObject@@SA_NPBV1@PBD01@Z 100070e8     qt-mt323:qt-mt323.dll
 0002:000000ec       __imp_??0QWidget@@QAE@PAV0@PBDI@Z 100070ec     qt-mt323:qt-mt323.dll
 0002:000000f0       __imp_??1QWidget@@UAE@XZ   100070f0     qt-mt323:qt-mt323.dll
 0002:000000f4       __imp_?setName@QWidget@@UAEXPBD@Z 100070f4     qt-mt323:qt-mt323.dll
 0002:000000f8       __imp_?rect@QWidget@@QBE?AVQRect@@XZ 100070f8     qt-mt323:qt-mt323.dll
 0002:000000fc       __imp_?closeEvent@QWidget@@MAEXPAVQCloseEvent@@@Z 100070fc     qt-mt323:qt-mt323.dll
 0002:00000100       __imp_?information@QMessageBox@@SAHPAVQWidget@@ABVQString@@1111HH@Z 10007100     qt-mt323:qt-mt323.dll
 0002:00000104       __imp_??1?$QPtrList@VQDockWindow@@@@UAE@XZ 10007104     qt-mt323:qt-mt323.dll
 0002:00000108       __imp_??9QDateTime@@QBE_NABV0@@Z 10007108     qt-mt323:qt-mt323.dll
 0002:0000010c       __imp_??0QFileInfo@@QAE@ABVQString@@@Z 1000710c     qt-mt323:qt-mt323.dll
 0002:00000110       __imp_??1QFileInfo@@QAE@XZ 10007110     qt-mt323:qt-mt323.dll
 0002:00000114       __imp_?lastModified@QFileInfo@@QBE?AVQDateTime@@XZ 10007114     qt-mt323:qt-mt323.dll
 0002:00000118       __imp_?add@QWhatsThis@@SAXPAVQWidget@@ABVQString@@@Z 10007118     qt-mt323:qt-mt323.dll
 0002:0000011c       __imp_??0QGuardedPtrPrivate@@QAE@PAVQObject@@@Z 1000711c     qt-mt323:qt-mt323.dll
 0002:00000120       __imp_??1QGuardedPtrPrivate@@UAE@XZ 10007120     qt-mt323:qt-mt323.dll
 0002:00000124       __imp_??0QGDict@@IAE@IW4KeyType@0@_N1@Z 10007124     qt-mt323:qt-mt323.dll
 0002:00000128       __imp_??1QGDict@@MAE@XZ    10007128     qt-mt323:qt-mt323.dll
 0002:0000012c       __imp_?clear@QGDict@@MAEXXZ 1000712c     qt-mt323:qt-mt323.dll
 0002:00000130       __imp_?adjustSize@QWidget@@UAEXXZ 10007130     qt-mt323:qt-mt323.dll
 0002:00000134       __imp_?checkConnectArgs@QObject@@MAE_NPBDPBV1@0@Z 10007134     qt-mt323:qt-mt323.dll
 0002:00000138       __imp_?childEvent@QObject@@MAEXPAVQChildEvent@@@Z 10007138     qt-mt323:qt-mt323.dll
 0002:0000013c       __imp_?className@QGuardedPtrPrivate@@UBEPBDXZ 1000713c     qt-mt323:qt-mt323.dll
 0002:00000140       __imp_?className@QWidget@@UBEPBDXZ 10007140     qt-mt323:qt-mt323.dll
 0002:00000144       __imp_?clear@?$QPtrList@VQDockWindow@@@@UAEXXZ 10007144     qt-mt323:qt-mt323.dll
 0002:00000148       __imp_?close@QWidget@@UAE_N_N@Z 10007148     qt-mt323:qt-mt323.dll
 0002:0000014c       __imp_?cmd@QPaintDevice@@MAE_NHPAVQPainter@@PATQPDevCmdParam@@@Z 1000714c     qt-mt323:qt-mt323.dll
 0002:00000150       __imp_?compareItems@QGList@@MAEHPAX0@Z 10007150     qt-mt323:qt-mt323.dll
 0002:00000154       __imp_?connectNotify@QObject@@MAEXPBD@Z 10007154     qt-mt323:qt-mt323.dll
 0002:00000158       __imp_?contextMenuEvent@QWidget@@MAEXPAVQContextMenuEvent@@@Z 10007158     qt-mt323:qt-mt323.dll
 0002:0000015c       __imp_?count@?$QPtrList@VQDockWindow@@@@UBEIXZ 1000715c     qt-mt323:qt-mt323.dll
 0002:00000160       __imp_?create@QWidget@@MAEXPAUHWND__@@_N1@Z 10007160     qt-mt323:qt-mt323.dll
 0002:00000164       __imp_?customEvent@QObject@@MAEXPAVQCustomEvent@@@Z 10007164     qt-mt323:qt-mt323.dll
 0002:00000168       __imp_?customWhatsThis@QWidget@@UBE_NXZ 10007168     qt-mt323:qt-mt323.dll
 0002:0000016c       __imp_?deleteItem@?$QPtrList@VQDockWindow@@@@EAEXPAX@Z 1000716c     qt-mt323:qt-mt323.dll
 0002:00000170       __imp_?destroy@QWidget@@MAEX_N0@Z 10007170     qt-mt323:qt-mt323.dll
 0002:00000174       __imp_?disconnectNotify@QObject@@MAEXPBD@Z 10007174     qt-mt323:qt-mt323.dll
 0002:00000178       __imp_?dragEnterEvent@QWidget@@MAEXPAVQDragEnterEvent@@@Z 10007178     qt-mt323:qt-mt323.dll
 0002:0000017c       __imp_?dragLeaveEvent@QWidget@@MAEXPAVQDragLeaveEvent@@@Z 1000717c     qt-mt323:qt-mt323.dll
 0002:00000180       __imp_?dragMoveEvent@QWidget@@MAEXPAVQDragMoveEvent@@@Z 10007180     qt-mt323:qt-mt323.dll
 0002:00000184       __imp_?dropEvent@QWidget@@MAEXPAVQDropEvent@@@Z 10007184     qt-mt323:qt-mt323.dll
 0002:00000188       __imp_?enabledChange@QWidget@@MAEX_N@Z 10007188     qt-mt323:qt-mt323.dll
 0002:0000018c       __imp_?enterEvent@QWidget@@MAEXPAVQEvent@@@Z 1000718c     qt-mt323:qt-mt323.dll
 0002:00000190       __imp_?event@QObject@@UAE_NPAVQEvent@@@Z 10007190     qt-mt323:qt-mt323.dll
 0002:00000194       __imp_?event@QWidget@@MAE_NPAVQEvent@@@Z 10007194     qt-mt323:qt-mt323.dll
 0002:00000198       __imp_?eventFilter@QObject@@UAE_NPAV1@PAVQEvent@@@Z 10007198     qt-mt323:qt-mt323.dll
 0002:0000019c       __imp_?focusInEvent@QWidget@@MAEXPAVQFocusEvent@@@Z 1000719c     qt-mt323:qt-mt323.dll
 0002:000001a0       __imp_?focusNextPrevChild@QWidget@@MAE_N_N@Z 100071a0     qt-mt323:qt-mt323.dll
 0002:000001a4       __imp_?focusOutEvent@QWidget@@MAEXPAVQFocusEvent@@@Z 100071a4     qt-mt323:qt-mt323.dll
 0002:000001a8       __imp_?fontChange@QWidget@@MAEXABVQFont@@@Z 100071a8     qt-mt323:qt-mt323.dll
 0002:000001ac       __imp_?fontInf@QPaintDevice@@MBEHPAVQFont@@H@Z 100071ac     qt-mt323:qt-mt323.dll
 0002:000001b0       __imp_?fontMet@QPaintDevice@@MBEHPAVQFont@@HPBDH@Z 100071b0     qt-mt323:qt-mt323.dll
 0002:000001b4       __imp_?handle@QPaintDevice@@UBEPAUHDC__@@XZ 100071b4     qt-mt323:qt-mt323.dll
 0002:000001b8       __imp_?heightForWidth@QWidget@@UBEHH@Z 100071b8     qt-mt323:qt-mt323.dll
 0002:000001bc       __imp_?hide@QWidget@@UAEXXZ 100071bc     qt-mt323:qt-mt323.dll
 0002:000001c0       __imp_?hideEvent@QWidget@@MAEXPAVQHideEvent@@@Z 100071c0     qt-mt323:qt-mt323.dll
 0002:000001c4       __imp_?imComposeEvent@QWidget@@MAEXPAVQIMEvent@@@Z 100071c4     qt-mt323:qt-mt323.dll
 0002:000001c8       __imp_?imEndEvent@QWidget@@MAEXPAVQIMEvent@@@Z 100071c8     qt-mt323:qt-mt323.dll
 0002:000001cc       __imp_?imStartEvent@QWidget@@MAEXPAVQIMEvent@@@Z 100071cc     qt-mt323:qt-mt323.dll
 0002:000001d0       __imp_?insertChild@QObject@@UAEXPAV1@@Z 100071d0     qt-mt323:qt-mt323.dll
 0002:000001d4       __imp_?keyPressEvent@QWidget@@MAEXPAVQKeyEvent@@@Z 100071d4     qt-mt323:qt-mt323.dll
 0002:000001d8       __imp_?keyReleaseEvent@QWidget@@MAEXPAVQKeyEvent@@@Z 100071d8     qt-mt323:qt-mt323.dll
 0002:000001dc       __imp_?leaveEvent@QWidget@@MAEXPAVQEvent@@@Z 100071dc     qt-mt323:qt-mt323.dll
 0002:000001e0       __imp_?metaObject@QGuardedPtrPrivate@@UBEPAVQMetaObject@@XZ 100071e0     qt-mt323:qt-mt323.dll
 0002:000001e4       __imp_?metaObject@QWidget@@UBEPAVQMetaObject@@XZ 100071e4     qt-mt323:qt-mt323.dll
 0002:000001e8       __imp_?metric@QWidget@@MBEHH@Z 100071e8     qt-mt323:qt-mt323.dll
 0002:000001ec       __imp_?minimumSizeHint@QWidget@@UBE?AVQSize@@XZ 100071ec     qt-mt323:qt-mt323.dll
 0002:000001f0       __imp_?mouseDoubleClickEvent@QWidget@@MAEXPAVQMouseEvent@@@Z 100071f0     qt-mt323:qt-mt323.dll
 0002:000001f4       __imp_?mouseMoveEvent@QWidget@@MAEXPAVQMouseEvent@@@Z 100071f4     qt-mt323:qt-mt323.dll
 0002:000001f8       __imp_?mousePressEvent@QWidget@@MAEXPAVQMouseEvent@@@Z 100071f8     qt-mt323:qt-mt323.dll
 0002:000001fc       __imp_?mouseReleaseEvent@QWidget@@MAEXPAVQMouseEvent@@@Z 100071fc     qt-mt323:qt-mt323.dll
 0002:00000200       __imp_?move@QWidget@@UAEXHH@Z 10007200     qt-mt323:qt-mt323.dll
 0002:00000204       __imp_?moveEvent@QWidget@@MAEXPAVQMoveEvent@@@Z 10007204     qt-mt323:qt-mt323.dll
 0002:00000208       __imp_?newItem@QPtrCollection@@MAEPAXPAX@Z 10007208     qt-mt323:qt-mt323.dll
 0002:0000020c       __imp_?paintEvent@QWidget@@MAEXPAVQPaintEvent@@@Z 1000720c     qt-mt323:qt-mt323.dll
 0002:00000210       __imp_?paletteChange@QWidget@@MAEXABVQPalette@@@Z 10007210     qt-mt323:qt-mt323.dll
 0002:00000214       __imp_?polish@QWidget@@UAEXXZ 10007214     qt-mt323:qt-mt323.dll
 0002:00000218       __imp_?property@QObject@@UBE?AVQVariant@@PBD@Z 10007218     qt-mt323:qt-mt323.dll
 0002:0000021c       __imp_?qt_cast@QGuardedPtrPrivate@@UAEPAXPBD@Z 1000721c     qt-mt323:qt-mt323.dll
 0002:00000220       __imp_?qt_cast@QWidget@@UAEPAXPBD@Z 10007220     qt-mt323:qt-mt323.dll
 0002:00000224       __imp_?qt_emit@QGuardedPtrPrivate@@UAE_NHPAUQUObject@@@Z 10007224     qt-mt323:qt-mt323.dll
 0002:00000228       __imp_?qt_emit@QWidget@@UAE_NHPAUQUObject@@@Z 10007228     qt-mt323:qt-mt323.dll
 0002:0000022c       __imp_?qt_invoke@QGuardedPtrPrivate@@UAE_NHPAUQUObject@@@Z 1000722c     qt-mt323:qt-mt323.dll
 0002:00000230       __imp_?qt_invoke@QWidget@@UAE_NHPAUQUObject@@@Z 10007230     qt-mt323:qt-mt323.dll
 0002:00000234       __imp_?qt_property@QGuardedPtrPrivate@@UAE_NHHPAVQVariant@@@Z 10007234     qt-mt323:qt-mt323.dll
 0002:00000238       __imp_?qt_property@QWidget@@UAE_NHHPAVQVariant@@@Z 10007238     qt-mt323:qt-mt323.dll
 0002:0000023c       __imp_?read@QGDict@@MAEAAVQDataStream@@AAV2@AAPAX@Z 1000723c     qt-mt323:qt-mt323.dll
 0002:00000240       __imp_?read@QGList@@MAEAAVQDataStream@@AAV2@AAPAX@Z 10007240     qt-mt323:qt-mt323.dll
 0002:00000244       __imp_?removeChild@QObject@@UAEXPAV1@@Z 10007244     qt-mt323:qt-mt323.dll
 0002:00000248       __imp_?reparent@QWidget@@UAEXPAV1@IABVQPoint@@_N@Z 10007248     qt-mt323:qt-mt323.dll
 0002:0000024c       __imp_?resize@QWidget@@UAEXHH@Z 1000724c     qt-mt323:qt-mt323.dll
 0002:00000250       __imp_?resizeEvent@QWidget@@MAEXPAVQResizeEvent@@@Z 10007250     qt-mt323:qt-mt323.dll
 0002:00000254       __imp_?resolution@QPaintDevice@@UBEHXZ 10007254     qt-mt323:qt-mt323.dll
 0002:00000258       __imp_?setAcceptDrops@QWidget@@UAEX_N@Z 10007258     qt-mt323:qt-mt323.dll
 0002:0000025c       __imp_?setActiveWindow@QWidget@@UAEXXZ 1000725c     qt-mt323:qt-mt323.dll
 0002:00000260       __imp_?setAutoMask@QWidget@@UAEX_N@Z 10007260     qt-mt323:qt-mt323.dll
 0002:00000264       __imp_?setBackgroundColor@QWidget@@UAEXABVQColor@@@Z 10007264     qt-mt323:qt-mt323.dll
 0002:00000268       __imp_?setBackgroundMode@QWidget@@UAEXW4BackgroundMode@Qt@@@Z 10007268     qt-mt323:qt-mt323.dll
 0002:0000026c       __imp_?setBackgroundOrigin@QWidget@@UAEXW4BackgroundOrigin@1@@Z 1000726c     qt-mt323:qt-mt323.dll
 0002:00000270       __imp_?setBackgroundPixmap@QWidget@@UAEXABVQPixmap@@@Z 10007270     qt-mt323:qt-mt323.dll
 0002:00000274       __imp_?setCaption@QWidget@@UAEXABVQString@@@Z 10007274     qt-mt323:qt-mt323.dll
 0002:00000278       __imp_?setCursor@QWidget@@UAEXABVQCursor@@@Z 10007278     qt-mt323:qt-mt323.dll
 0002:0000027c       __imp_?setEnabled@QWidget@@UAEX_N@Z 1000727c     qt-mt323:qt-mt323.dll
 0002:00000280       __imp_?setEraseColor@QWidget@@UAEXABVQColor@@@Z 10007280     qt-mt323:qt-mt323.dll
 0002:00000284       __imp_?setErasePixmap@QWidget@@UAEXABVQPixmap@@@Z 10007284     qt-mt323:qt-mt323.dll
 0002:00000288       __imp_?setFocus@QWidget@@UAEXXZ 10007288     qt-mt323:qt-mt323.dll
 0002:0000028c       __imp_?setFocusPolicy@QWidget@@UAEXW4FocusPolicy@1@@Z 1000728c     qt-mt323:qt-mt323.dll
 0002:00000290       __imp_?setFocusProxy@QWidget@@UAEXPAV1@@Z 10007290     qt-mt323:qt-mt323.dll
 0002:00000294       __imp_?setFont@QWidget@@UAEXABVQFont@@@Z 10007294     qt-mt323:qt-mt323.dll
 0002:00000298       __imp_?setGeometry@QWidget@@UAEXABVQRect@@@Z 10007298     qt-mt323:qt-mt323.dll
 0002:0000029c       __imp_?setGeometry@QWidget@@UAEXHHHH@Z 1000729c     qt-mt323:qt-mt323.dll
 0002:000002a0       __imp_?setIcon@QWidget@@UAEXABVQPixmap@@@Z 100072a0     qt-mt323:qt-mt323.dll
 0002:000002a4       __imp_?setIconText@QWidget@@UAEXABVQString@@@Z 100072a4     qt-mt323:qt-mt323.dll
 0002:000002a8       __imp_?setKeyCompression@QWidget@@MAEX_N@Z 100072a8     qt-mt323:qt-mt323.dll
 0002:000002ac       __imp_?setMask@QWidget@@UAEXABVQBitmap@@@Z 100072ac     qt-mt323:qt-mt323.dll
 0002:000002b0       __imp_?setMask@QWidget@@UAEXABVQRegion@@@Z 100072b0     qt-mt323:qt-mt323.dll
 0002:000002b4       __imp_?setMaximumSize@QWidget@@UAEXHH@Z 100072b4     qt-mt323:qt-mt323.dll
 0002:000002b8       __imp_?setMicroFocusHint@QWidget@@MAEXHHHH_NPAVQFont@@@Z 100072b8     qt-mt323:qt-mt323.dll
 0002:000002bc       __imp_?setMinimumSize@QWidget@@UAEXHH@Z 100072bc     qt-mt323:qt-mt323.dll
 0002:000002c0       __imp_?setMouseTracking@QWidget@@UAEX_N@Z 100072c0     qt-mt323:qt-mt323.dll
 0002:000002c4       __imp_?setName@QObject@@UAEXPBD@Z 100072c4     qt-mt323:qt-mt323.dll
 0002:000002c8       __imp_?setPalette@QWidget@@UAEXABVQPalette@@@Z 100072c8     qt-mt323:qt-mt323.dll
 0002:000002cc       __imp_?setPaletteBackgroundColor@QWidget@@UAEXABVQColor@@@Z 100072cc     qt-mt323:qt-mt323.dll
 0002:000002d0       __imp_?setPaletteBackgroundPixmap@QWidget@@UAEXABVQPixmap@@@Z 100072d0     qt-mt323:qt-mt323.dll
 0002:000002d4       __imp_?setProperty@QObject@@UAE_NPBDABVQVariant@@@Z 100072d4     qt-mt323:qt-mt323.dll
 0002:000002d8       __imp_?setResolution@QPaintDevice@@UAEXH@Z 100072d8     qt-mt323:qt-mt323.dll
 0002:000002dc       __imp_?setSizeIncrement@QWidget@@UAEXHH@Z 100072dc     qt-mt323:qt-mt323.dll
 0002:000002e0       __imp_?setSizePolicy@QWidget@@UAEXVQSizePolicy@@@Z 100072e0     qt-mt323:qt-mt323.dll
 0002:000002e4       __imp_?setUpdatesEnabled@QWidget@@UAEX_N@Z 100072e4     qt-mt323:qt-mt323.dll
 0002:000002e8       __imp_?setWFlags@QWidget@@MAEXI@Z 100072e8     qt-mt323:qt-mt323.dll
 0002:000002ec       __imp_?setWState@QWidget@@MAEXI@Z 100072ec     qt-mt323:qt-mt323.dll
 0002:000002f0       __imp_?show@QWidget@@UAEXXZ 100072f0     qt-mt323:qt-mt323.dll
 0002:000002f4       __imp_?showEvent@QWidget@@MAEXPAVQShowEvent@@@Z 100072f4     qt-mt323:qt-mt323.dll
 0002:000002f8       __imp_?showMaximized@QWidget@@UAEXXZ 100072f8     qt-mt323:qt-mt323.dll
 0002:000002fc       __imp_?showMinimized@QWidget@@UAEXXZ 100072fc     qt-mt323:qt-mt323.dll
 0002:00000300       __imp_?showNormal@QWidget@@UAEXXZ 10007300     qt-mt323:qt-mt323.dll
 0002:00000304       __imp_?sizeHint@QWidget@@UBE?AVQSize@@XZ 10007304     qt-mt323:qt-mt323.dll
 0002:00000308       __imp_?sizePolicy@QWidget@@UBE?AVQSizePolicy@@XZ 10007308     qt-mt323:qt-mt323.dll
 0002:0000030c       __imp_?styleChange@QWidget@@MAEXAAVQStyle@@@Z 1000730c     qt-mt323:qt-mt323.dll
 0002:00000310       __imp_?tabletEvent@QWidget@@MAEXPAVQTabletEvent@@@Z 10007310     qt-mt323:qt-mt323.dll
 0002:00000314       __imp_?timerEvent@QObject@@MAEXPAVQTimerEvent@@@Z 10007314     qt-mt323:qt-mt323.dll
 0002:00000318       __imp_?unsetCursor@QWidget@@UAEXXZ 10007318     qt-mt323:qt-mt323.dll
 0002:0000031c       __imp_?updateMask@QWidget@@MAEXXZ 1000731c     qt-mt323:qt-mt323.dll
 0002:00000320       __imp_?wheelEvent@QWidget@@MAEXPAVQWheelEvent@@@Z 10007320     qt-mt323:qt-mt323.dll
 0002:00000324       __imp_?winEvent@QWidget@@MAE_NPAUtagMSG@@@Z 10007324     qt-mt323:qt-mt323.dll
 0002:00000328       __imp_?windowActivationChange@QWidget@@MAEX_N@Z 10007328     qt-mt323:qt-mt323.dll
 0002:0000032c       __imp_?write@QGDict@@MBEAAVQDataStream@@AAV2@PAX@Z 1000732c     qt-mt323:qt-mt323.dll
 0002:00000330       __imp_?write@QGList@@MBEAAVQDataStream@@AAV2@PAX@Z 10007330     qt-mt323:qt-mt323.dll
 0002:00000334       __imp_??_7?$QPtrList@VQDockWindow@@@@6B@ 10007334     qt-mt323:qt-mt323.dll
 0002:00000338       __imp_??0QTextStream@@QAE@PAVQIODevice@@@Z 10007338     qt-mt323:qt-mt323.dll
 0002:0000033c       __imp_??1QTextStream@@UAE@XZ 1000733c     qt-mt323:qt-mt323.dll
 0002:00000340       __imp_??6QTextStream@@QAEAAV0@ABVQString@@@Z 10007340     qt-mt323:qt-mt323.dll
 0002:00000344       __imp_?read@QTextStream@@QAE?AVQString@@XZ 10007344     qt-mt323:qt-mt323.dll
 0002:00000348       __imp_?blockSignals@QObject@@QAEX_N@Z 10007348     qt-mt323:qt-mt323.dll
 0002:0000034c       __imp_?setPaletteForegroundColor@QWidget@@QAEXABVQColor@@@Z 1000734c     qt-mt323:qt-mt323.dll
 0002:00000350       __imp_?text@QTextEdit@@QBE?AVQString@@XZ 10007350     qt-mt323:qt-mt323.dll
 0002:00000354       __imp_?setText@QTextEdit@@QAEXABVQString@@@Z 10007354     qt-mt323:qt-mt323.dll
 0002:00000358       __imp_?black@Qt@@2AAVQColor@@A 10007358     qt-mt323:qt-mt323.dll
 0002:0000035c       __imp_?gray@Qt@@2AAVQColor@@A 1000735c     qt-mt323:qt-mt323.dll
 0002:00000360       __imp_?append@?$QValueList@VQString@@@@QAE?AV?$QValueListIterator@VQString@@@@ABVQString@@@Z 10007360     qt-mt323:qt-mt323.dll
 0002:00000364       __imp_??4QColor@@QAEAAV0@ABV0@@Z 10007364     qt-mt323:qt-mt323.dll
 0002:00000368       __imp_?qstrcmp@@YAHPBD0@Z  10007368     qt-mt323:qt-mt323.dll
 0002:0000036c       __imp_?fromLatin1@QString@@SA?AV1@PBDH@Z 1000736c     qt-mt323:qt-mt323.dll
 0002:00000370       __imp_?receivers@QObject@@IBEPAVQConnectionList@@H@Z 10007370     qt-mt323:qt-mt323.dll
 0002:00000374       __imp_?activate_signal@QObject@@IAEXPAVQConnectionList@@PAUQUObject@@@Z 10007374     qt-mt323:qt-mt323.dll
 0002:00000378       __imp_?staticMetaObject@QWidget@@SAPAVQMetaObject@@XZ 10007378     qt-mt323:qt-mt323.dll
 0002:0000037c       __imp_?new_metaobject@QMetaObject@@SAPAV1@PBDPAV1@QBUQMetaData@@H2HQBVQMetaProperty@@HQBUQMetaEnum@@HQBUQClassInfo@@H@Z 1000737c     qt-mt323:qt-mt323.dll
 0002:00000380       __imp_??0QMetaObjectCleanUp@@QAE@PBDP6APAVQMetaObject@@XZ@Z 10007380     qt-mt323:qt-mt323.dll
 0002:00000384       __imp_??1QMetaObjectCleanUp@@QAE@XZ 10007384     qt-mt323:qt-mt323.dll
 0002:00000388       __imp_?setMetaObject@QMetaObjectCleanUp@@QAEXAAPAVQMetaObject@@@Z 10007388     qt-mt323:qt-mt323.dll
 0002:0000038c       __imp_?translate@QApplication@@QBE?AVQString@@PBD00W4Encoding@1@@Z 1000738c     qt-mt323:qt-mt323.dll
 0002:00000390       __imp_??0QUObject@@QAE@XZ  10007390     qt-mt323:qt-mt323.dll
 0002:00000394       __imp_??1QUObject@@QAE@XZ  10007394     qt-mt323:qt-mt323.dll
 0002:00000398       __imp_?set@QUType_QString@@QAEXPAUQUObject@@ABVQString@@@Z 10007398     qt-mt323:qt-mt323.dll
 0002:0000039c       __imp_?qApp@@3PAVQApplication@@A 1000739c     qt-mt323:qt-mt323.dll
 0002:000003a0       __imp_?static_QUType_QString@@3UQUType_QString@@A 100073a0     qt-mt323:qt-mt323.dll
 0002:000003a4       __imp_?resize@QWidget@@QAEXABVQSize@@@Z 100073a4     qt-mt323:qt-mt323.dll
 0002:000003a8       __imp_?setFrameShape@QFrame@@QAEXW4Shape@1@@Z 100073a8     qt-mt323:qt-mt323.dll
 0002:000003ac       __imp_?setFrameShadow@QFrame@@QAEXW4Shadow@1@@Z 100073ac     qt-mt323:qt-mt323.dll
 0002:000003b0       __imp_??0QLabel@@QAE@PAVQWidget@@PBDI@Z 100073b0     qt-mt323:qt-mt323.dll
 0002:000003b4       __imp_??1QLabel@@UAE@XZ    100073b4     qt-mt323:qt-mt323.dll
 0002:000003b8       __imp_??0QTextEdit@@QAE@PAVQWidget@@PBD@Z 100073b8     qt-mt323:qt-mt323.dll
 0002:000003bc       __imp_??1QTextEdit@@UAE@XZ 100073bc     qt-mt323:qt-mt323.dll
 0002:000003c0       __imp_??1QLayoutItem@@UAE@XZ 100073c0     qt-mt323:qt-mt323.dll
 0002:000003c4       __imp_??0QSpacerItem@@QAE@HHW4SizeType@QSizePolicy@@0@Z 100073c4     qt-mt323:qt-mt323.dll
 0002:000003c8       __imp_?addWidget@QBoxLayout@@QAEXPAVQWidget@@HH@Z 100073c8     qt-mt323:qt-mt323.dll
 0002:000003cc       __imp_?addLayout@QBoxLayout@@QAEXPAVQLayout@@H@Z 100073cc     qt-mt323:qt-mt323.dll
 0002:000003d0       __imp_??0QHBoxLayout@@QAE@PAVQWidget@@HHPBD@Z 100073d0     qt-mt323:qt-mt323.dll
 0002:000003d4       __imp_??1QHBoxLayout@@UAE@XZ 100073d4     qt-mt323:qt-mt323.dll
 0002:000003d8       __imp_??0QVBoxLayout@@QAE@PAVQWidget@@HHPBD@Z 100073d8     qt-mt323:qt-mt323.dll
 0002:000003dc       __imp_??1QVBoxLayout@@UAE@XZ 100073dc     qt-mt323:qt-mt323.dll
 0002:000003e0       __imp_?addChild@QScrollView@@UAEXPAVQWidget@@HH@Z 100073e0     qt-mt323:qt-mt323.dll
 0002:000003e4       __imp_??0QString@@QAE@VQChar@@@Z 100073e4     qt-mt323:qt-mt323.dll
 0002:000003e8       __imp_?append@QTextEdit@@UAEXABVQString@@@Z 100073e8     qt-mt323:qt-mt323.dll
 0002:000003ec       __imp_?childEvent@QLayout@@MAEXPAVQChildEvent@@@Z 100073ec     qt-mt323:qt-mt323.dll
 0002:000003f0       __imp_?className@QHBoxLayout@@UBEPBDXZ 100073f0     qt-mt323:qt-mt323.dll
 0002:000003f4       __imp_?className@QLabel@@UBEPBDXZ 100073f4     qt-mt323:qt-mt323.dll
 0002:000003f8       __imp_?className@QTextEdit@@UBEPBDXZ 100073f8     qt-mt323:qt-mt323.dll
 0002:000003fc       __imp_?className@QVBoxLayout@@UBEPBDXZ 100073fc     qt-mt323:qt-mt323.dll
 0002:00000400       __imp_?clear@QTextEdit@@UAEXXZ 10007400     qt-mt323:qt-mt323.dll
 0002:00000404       __imp_?clearParagraphBackground@QTextEdit@@UAEXH@Z 10007404     qt-mt323:qt-mt323.dll
 0002:00000408       __imp_?contentsContextMenuEvent@QTextEdit@@MAEXPAVQContextMenuEvent@@@Z 10007408     qt-mt323:qt-mt323.dll
 0002:0000040c       __imp_?contentsDragEnterEvent@QTextEdit@@MAEXPAVQDragEnterEvent@@@Z 1000740c     qt-mt323:qt-mt323.dll
 0002:00000410       __imp_?contentsDragLeaveEvent@QTextEdit@@MAEXPAVQDragLeaveEvent@@@Z 10007410     qt-mt323:qt-mt323.dll
 0002:00000414       __imp_?contentsDragMoveEvent@QTextEdit@@MAEXPAVQDragMoveEvent@@@Z 10007414     qt-mt323:qt-mt323.dll
 0002:00000418       __imp_?contentsDropEvent@QTextEdit@@MAEXPAVQDropEvent@@@Z 10007418     qt-mt323:qt-mt323.dll
 0002:0000041c       __imp_?contentsMouseDoubleClickEvent@QTextEdit@@MAEXPAVQMouseEvent@@@Z 1000741c     qt-mt323:qt-mt323.dll
 0002:00000420       __imp_?contentsMouseMoveEvent@QTextEdit@@MAEXPAVQMouseEvent@@@Z 10007420     qt-mt323:qt-mt323.dll
 0002:00000424       __imp_?contentsMousePressEvent@QTextEdit@@MAEXPAVQMouseEvent@@@Z 10007424     qt-mt323:qt-mt323.dll
 0002:00000428       __imp_?contentsMouseReleaseEvent@QTextEdit@@MAEXPAVQMouseEvent@@@Z 10007428     qt-mt323:qt-mt323.dll
 0002:0000042c       __imp_?contentsWheelEvent@QTextEdit@@MAEXPAVQWheelEvent@@@Z 1000742c     qt-mt323:qt-mt323.dll
 0002:00000430       __imp_?contextMenuEvent@QScrollView@@MAEXPAVQContextMenuEvent@@@Z 10007430     qt-mt323:qt-mt323.dll
 0002:00000434       __imp_?copy@QTextEdit@@UAEXXZ 10007434     qt-mt323:qt-mt323.dll
 0002:00000438       __imp_?createPopupMenu@QTextEdit@@MAEPAVQPopupMenu@@ABVQPoint@@@Z 10007438     qt-mt323:qt-mt323.dll
 0002:0000043c       __imp_?createPopupMenu@QTextEdit@@MAEPAVQPopupMenu@@XZ 1000743c     qt-mt323:qt-mt323.dll
 0002:00000440       __imp_?cut@QTextEdit@@UAEXXZ 10007440     qt-mt323:qt-mt323.dll
 0002:00000444       __imp_?del@QTextEdit@@UAEXXZ 10007444     qt-mt323:qt-mt323.dll
 0002:00000448       __imp_?doChangeInterval@QTextEdit@@MAEXXZ 10007448     qt-mt323:qt-mt323.dll
 0002:0000044c       __imp_?doKeyboardAction@QTextEdit@@UAEXW4KeyboardAction@1@@Z 1000744c     qt-mt323:qt-mt323.dll
 0002:00000450       __imp_?drawContents@QLabel@@MAEXPAVQPainter@@@Z 10007450     qt-mt323:qt-mt323.dll
 0002:00000454       __imp_?drawContents@QTextEdit@@EAEXPAVQPainter@@@Z 10007454     qt-mt323:qt-mt323.dll
 0002:00000458       __imp_?drawContents@QTextEdit@@MAEXPAVQPainter@@HHHH@Z 10007458     qt-mt323:qt-mt323.dll
 0002:0000045c       __imp_?drawContentsOffset@QScrollView@@MAEXPAVQPainter@@HHHHHH@Z 1000745c     qt-mt323:qt-mt323.dll
 0002:00000460       __imp_?drawFrame@QFrame@@MAEXPAVQPainter@@@Z 10007460     qt-mt323:qt-mt323.dll
 0002:00000464       __imp_?emitHighlighted@QTextEdit@@EAEXABVQString@@@Z 10007464     qt-mt323:qt-mt323.dll
 0002:00000468       __imp_?emitLinkClicked@QTextEdit@@EAEXABVQString@@@Z 10007468     qt-mt323:qt-mt323.dll
 0002:0000046c       __imp_?ensureCursorVisible@QTextEdit@@UAEXXZ 1000746c     qt-mt323:qt-mt323.dll
 0002:00000470       __imp_?event@QTextEdit@@MAE_NPAVQEvent@@@Z 10007470     qt-mt323:qt-mt323.dll
 0002:00000474       __imp_?eventFilter@QLayout@@MAE_NPAVQObject@@PAVQEvent@@@Z 10007474     qt-mt323:qt-mt323.dll
 0002:00000478       __imp_?eventFilter@QTextEdit@@UAE_NPAVQObject@@PAVQEvent@@@Z 10007478     qt-mt323:qt-mt323.dll
 0002:0000047c       __imp_?expanding@QBoxLayout@@UBE?AW4ExpandData@QSizePolicy@@XZ 1000747c     qt-mt323:qt-mt323.dll
 0002:00000480       __imp_?expanding@QSpacerItem@@UBE?AW4ExpandData@QSizePolicy@@XZ 10007480     qt-mt323:qt-mt323.dll
 0002:00000484       __imp_?find@QTextEdit@@UAE_NABVQString@@_N11PAH2@Z 10007484     qt-mt323:qt-mt323.dll
 0002:00000488       __imp_?focusNextPrevChild@QTextEdit@@MAE_N_N@Z 10007488     qt-mt323:qt-mt323.dll
 0002:0000048c       __imp_?fontChange@QLabel@@MAEXABVQFont@@@Z 1000748c     qt-mt323:qt-mt323.dll
 0002:00000490       __imp_?fontChange@QScrollView@@MAEXABVQFont@@@Z 10007490     qt-mt323:qt-mt323.dll
 0002:00000494       __imp_?frameChanged@QFrame@@MAEXXZ 10007494     qt-mt323:qt-mt323.dll
 0002:00000498       __imp_?frameChanged@QScrollView@@MAEXXZ 10007498     qt-mt323:qt-mt323.dll
 0002:0000049c       __imp_?geometry@QLayout@@UBE?AVQRect@@XZ 1000749c     qt-mt323:qt-mt323.dll
 0002:000004a0       __imp_?geometry@QSpacerItem@@UBE?AVQRect@@XZ 100074a0     qt-mt323:qt-mt323.dll
 0002:000004a4       __imp_?getFormat@QTextEdit@@UAE_NHHPAVQFont@@PAVQColor@@PAW4VerticalAlignment@1@@Z 100074a4     qt-mt323:qt-mt323.dll
 0002:000004a8       __imp_?getParagraphFormat@QTextEdit@@UAE_NHPAVQFont@@PAVQColor@@PAW4VerticalAlignment@1@PAHPAW4DisplayMode@QStyleSheetItem@@PAW4ListStyle@6@3@Z 100074a8     qt-mt323:qt-mt323.dll
 0002:000004ac       __imp_?hasHeightForWidth@QBoxLayout@@UBE_NXZ 100074ac     qt-mt323:qt-mt323.dll
 0002:000004b0       __imp_?hasHeightForWidth@QLayoutItem@@UBE_NXZ 100074b0     qt-mt323:qt-mt323.dll
 0002:000004b4       __imp_?heightForWidth@QBoxLayout@@UBEHH@Z 100074b4     qt-mt323:qt-mt323.dll
 0002:000004b8       __imp_?heightForWidth@QLabel@@UBEHH@Z 100074b8     qt-mt323:qt-mt323.dll
 0002:000004bc       __imp_?heightForWidth@QLayoutItem@@UBEHH@Z 100074bc     qt-mt323:qt-mt323.dll
 0002:000004c0       __imp_?heightForWidth@QTextEdit@@UBEHH@Z 100074c0     qt-mt323:qt-mt323.dll
 0002:000004c4       __imp_?imComposeEvent@QTextEdit@@MAEXPAVQIMEvent@@@Z 100074c4     qt-mt323:qt-mt323.dll
 0002:000004c8       __imp_?imEndEvent@QTextEdit@@MAEXPAVQIMEvent@@@Z 100074c8     qt-mt323:qt-mt323.dll
 0002:000004cc       __imp_?imStartEvent@QTextEdit@@MAEXPAVQIMEvent@@@Z 100074cc     qt-mt323:qt-mt323.dll
 0002:000004d0       __imp_?indent@QTextEdit@@UAEXXZ 100074d0     qt-mt323:qt-mt323.dll
 0002:000004d4       __imp_?insert@QTextEdit@@UAEXABVQString@@_N11@Z 100074d4     qt-mt323:qt-mt323.dll
 0002:000004d8       __imp_?insertAt@QTextEdit@@UAEXABVQString@@HH@Z 100074d8     qt-mt323:qt-mt323.dll
 0002:000004dc       __imp_?insertParagraph@QTextEdit@@UAEXABVQString@@H@Z 100074dc     qt-mt323:qt-mt323.dll
 0002:000004e0       __imp_?invalidate@QBoxLayout@@UAEXXZ 100074e0     qt-mt323:qt-mt323.dll
 0002:000004e4       __imp_?invalidate@QLayoutItem@@UAEXXZ 100074e4     qt-mt323:qt-mt323.dll
 0002:000004e8       __imp_?isEmpty@QLayout@@UBE_NXZ 100074e8     qt-mt323:qt-mt323.dll
 0002:000004ec       __imp_?isEmpty@QSpacerItem@@UBE_NXZ 100074ec     qt-mt323:qt-mt323.dll
 0002:000004f0       __imp_?iterator@QBoxLayout@@UAE?AVQLayoutIterator@@XZ 100074f0     qt-mt323:qt-mt323.dll
 0002:000004f4       __imp_?iterator@QLayoutItem@@UAE?AVQLayoutIterator@@XZ 100074f4     qt-mt323:qt-mt323.dll
 0002:000004f8       __imp_?keyPressEvent@QTextEdit@@MAEXPAVQKeyEvent@@@Z 100074f8     qt-mt323:qt-mt323.dll
 0002:000004fc       __imp_?layout@QLayout@@UAEPAV1@XZ 100074fc     qt-mt323:qt-mt323.dll
 0002:00000500       __imp_?layout@QLayoutItem@@UAEPAVQLayout@@XZ 10007500     qt-mt323:qt-mt323.dll
 0002:00000504       __imp_?linksEnabled@QTextEdit@@EBE_NXZ 10007504     qt-mt323:qt-mt323.dll
 0002:00000508       __imp_?maximumSize@QBoxLayout@@UBE?AVQSize@@XZ 10007508     qt-mt323:qt-mt323.dll
 0002:0000050c       __imp_?maximumSize@QSpacerItem@@UBE?AVQSize@@XZ 1000750c     qt-mt323:qt-mt323.dll
 0002:00000510       __imp_?metaObject@QHBoxLayout@@UBEPAVQMetaObject@@XZ 10007510     qt-mt323:qt-mt323.dll
 0002:00000514       __imp_?metaObject@QLabel@@UBEPAVQMetaObject@@XZ 10007514     qt-mt323:qt-mt323.dll
 0002:00000518       __imp_?metaObject@QTextEdit@@UBEPAVQMetaObject@@XZ 10007518     qt-mt323:qt-mt323.dll
 0002:0000051c       __imp_?metaObject@QVBoxLayout@@UBEPAVQMetaObject@@XZ 1000751c     qt-mt323:qt-mt323.dll
 0002:00000520       __imp_?minimumSize@QBoxLayout@@UBE?AVQSize@@XZ 10007520     qt-mt323:qt-mt323.dll
 0002:00000524       __imp_?minimumSize@QSpacerItem@@UBE?AVQSize@@XZ 10007524     qt-mt323:qt-mt323.dll
 0002:00000528       __imp_?minimumSizeHint@QLabel@@UBE?AVQSize@@XZ 10007528     qt-mt323:qt-mt323.dll
 0002:0000052c       __imp_?minimumSizeHint@QScrollView@@UBE?AVQSize@@XZ 1000752c     qt-mt323:qt-mt323.dll
 0002:00000530       __imp_?mouseDoubleClickEvent@QScrollView@@MAEXPAVQMouseEvent@@@Z 10007530     qt-mt323:qt-mt323.dll
 0002:00000534       __imp_?mouseMoveEvent@QScrollView@@MAEXPAVQMouseEvent@@@Z 10007534     qt-mt323:qt-mt323.dll
 0002:00000538       __imp_?mousePressEvent@QScrollView@@MAEXPAVQMouseEvent@@@Z 10007538     qt-mt323:qt-mt323.dll
 0002:0000053c       __imp_?mouseReleaseEvent@QScrollView@@MAEXPAVQMouseEvent@@@Z 1000753c     qt-mt323:qt-mt323.dll
 0002:00000540       __imp_?moveChild@QScrollView@@UAEXPAVQWidget@@HH@Z 10007540     qt-mt323:qt-mt323.dll
 0002:00000544       __imp_?moveCursor@QTextEdit@@UAEXW4CursorAction@1@_N@Z 10007544     qt-mt323:qt-mt323.dll
 0002:00000548       __imp_?paintEvent@QFrame@@MAEXPAVQPaintEvent@@@Z 10007548     qt-mt323:qt-mt323.dll
 0002:0000054c       __imp_?paste@QTextEdit@@UAEXXZ 1000754c     qt-mt323:qt-mt323.dll
 0002:00000550       __imp_?pasteSubType@QTextEdit@@UAEXABVQCString@@@Z 10007550     qt-mt323:qt-mt323.dll
 0002:00000554       __imp_?placeCursor@QTextEdit@@UAEXABVQPoint@@PAVQTextCursor@@@Z 10007554     qt-mt323:qt-mt323.dll
 0002:00000558       __imp_?polish@QTextEdit@@UAEXXZ 10007558     qt-mt323:qt-mt323.dll
 0002:0000055c       __imp_?qt_cast@QHBoxLayout@@UAEPAXPBD@Z 1000755c     qt-mt323:qt-mt323.dll
 0002:00000560       __imp_?qt_cast@QLabel@@UAEPAXPBD@Z 10007560     qt-mt323:qt-mt323.dll
 0002:00000564       __imp_?qt_cast@QTextEdit@@UAEPAXPBD@Z 10007564     qt-mt323:qt-mt323.dll
 0002:00000568       __imp_?qt_cast@QVBoxLayout@@UAEPAXPBD@Z 10007568     qt-mt323:qt-mt323.dll
 0002:0000056c       __imp_?qt_emit@QHBoxLayout@@UAE_NHPAUQUObject@@@Z 1000756c     qt-mt323:qt-mt323.dll
 0002:00000570       __imp_?qt_emit@QLabel@@UAE_NHPAUQUObject@@@Z 10007570     qt-mt323:qt-mt323.dll
 0002:00000574       __imp_?qt_emit@QTextEdit@@UAE_NHPAUQUObject@@@Z 10007574     qt-mt323:qt-mt323.dll
 0002:00000578       __imp_?qt_emit@QVBoxLayout@@UAE_NHPAUQUObject@@@Z 10007578     qt-mt323:qt-mt323.dll
 0002:0000057c       __imp_?qt_invoke@QHBoxLayout@@UAE_NHPAUQUObject@@@Z 1000757c     qt-mt323:qt-mt323.dll
 0002:00000580       __imp_?qt_invoke@QLabel@@UAE_NHPAUQUObject@@@Z 10007580     qt-mt323:qt-mt323.dll
 0002:00000584       __imp_?qt_invoke@QTextEdit@@UAE_NHPAUQUObject@@@Z 10007584     qt-mt323:qt-mt323.dll
 0002:00000588       __imp_?qt_invoke@QVBoxLayout@@UAE_NHPAUQUObject@@@Z 10007588     qt-mt323:qt-mt323.dll
 0002:0000058c       __imp_?qt_property@QHBoxLayout@@UAE_NHHPAVQVariant@@@Z 1000758c     qt-mt323:qt-mt323.dll
 0002:00000590       __imp_?qt_property@QLabel@@UAE_NHHPAVQVariant@@@Z 10007590     qt-mt323:qt-mt323.dll
 0002:00000594       __imp_?qt_property@QTextEdit@@UAE_NHHPAVQVariant@@@Z 10007594     qt-mt323:qt-mt323.dll
 0002:00000598       __imp_?qt_property@QVBoxLayout@@UAE_NHHPAVQVariant@@@Z 10007598     qt-mt323:qt-mt323.dll
 0002:0000059c       __imp_?redo@QTextEdit@@UAEXXZ 1000759c     qt-mt323:qt-mt323.dll
 0002:000005a0       __imp_?removeChild@QScrollView@@UAEXPAVQObject@@@Z 100075a0     qt-mt323:qt-mt323.dll
 0002:000005a4       __imp_?removeParagraph@QTextEdit@@UAEXH@Z 100075a4     qt-mt323:qt-mt323.dll
 0002:000005a8       __imp_?removeSelectedText@QTextEdit@@UAEXH@Z 100075a8     qt-mt323:qt-mt323.dll
 0002:000005ac       __imp_?removeSelection@QTextEdit@@UAEXH@Z 100075ac     qt-mt323:qt-mt323.dll
 0002:000005b0       __imp_?resetFormat@QTextEdit@@UAEXXZ 100075b0     qt-mt323:qt-mt323.dll
 0002:000005b4       __imp_?resize@QScrollView@@UAEXHH@Z 100075b4     qt-mt323:qt-mt323.dll
 0002:000005b8       __imp_?resizeContents@QScrollView@@UAEXHH@Z 100075b8     qt-mt323:qt-mt323.dll
 0002:000005bc       __imp_?resizeEvent@QLabel@@MAEXPAVQResizeEvent@@@Z 100075bc     qt-mt323:qt-mt323.dll
 0002:000005c0       __imp_?resizeEvent@QTextEdit@@MAEXPAVQResizeEvent@@@Z 100075c0     qt-mt323:qt-mt323.dll
 0002:000005c4       __imp_?scrollToAnchor@QTextEdit@@UAEXABVQString@@@Z 100075c4     qt-mt323:qt-mt323.dll
 0002:000005c8       __imp_?scrollToBottom@QTextEdit@@UAEXXZ 100075c8     qt-mt323:qt-mt323.dll
 0002:000005cc       __imp_?selectAll@QTextEdit@@UAEX_N@Z 100075cc     qt-mt323:qt-mt323.dll
 0002:000005d0       __imp_?setAlignment@QLabel@@UAEXH@Z 100075d0     qt-mt323:qt-mt323.dll
 0002:000005d4       __imp_?setAlignment@QLayoutItem@@UAEXH@Z 100075d4     qt-mt323:qt-mt323.dll
 0002:000005d8       __imp_?setAlignment@QTextEdit@@UAEXH@Z 100075d8     qt-mt323:qt-mt323.dll
 0002:000005dc       __imp_?setAutoAdd@QLayout@@UAEX_N@Z 100075dc     qt-mt323:qt-mt323.dll
 0002:000005e0       __imp_?setAutoResize@QLabel@@UAEX_N@Z 100075e0     qt-mt323:qt-mt323.dll
 0002:000005e4       __imp_?setBold@QTextEdit@@UAEX_N@Z 100075e4     qt-mt323:qt-mt323.dll
 0002:000005e8       __imp_?setBuddy@QLabel@@UAEXPAVQWidget@@@Z 100075e8     qt-mt323:qt-mt323.dll
 0002:000005ec       __imp_?setColor@QTextEdit@@UAEXABVQColor@@@Z 100075ec     qt-mt323:qt-mt323.dll
 0002:000005f0       __imp_?setContentsPos@QScrollView@@UAEXHH@Z 100075f0     qt-mt323:qt-mt323.dll
 0002:000005f4       __imp_?setCornerWidget@QScrollView@@UAEXPAVQWidget@@@Z 100075f4     qt-mt323:qt-mt323.dll
 0002:000005f8       __imp_?setCurrentFont@QTextEdit@@UAEXABVQFont@@@Z 100075f8     qt-mt323:qt-mt323.dll
 0002:000005fc       __imp_?setCursorPosition@QTextEdit@@UAEXHH@Z 100075fc     qt-mt323:qt-mt323.dll
 0002:00000600       __imp_?setDragAutoScroll@QScrollView@@UAEX_N@Z 10007600     qt-mt323:qt-mt323.dll
 0002:00000604       __imp_?setEnabled@QTextEdit@@UAEX_N@Z 10007604     qt-mt323:qt-mt323.dll
 0002:00000608       __imp_?setFamily@QTextEdit@@UAEXABVQString@@@Z 10007608     qt-mt323:qt-mt323.dll
 0002:0000060c       __imp_?setFont@QLabel@@UAEXABVQFont@@@Z 1000760c     qt-mt323:qt-mt323.dll
 0002:00000610       __imp_?setFont@QTextEdit@@UAEXABVQFont@@@Z 10007610     qt-mt323:qt-mt323.dll
 0002:00000614       __imp_?setFormat@QTextEdit@@UAEXPAVQTextFormat@@H@Z 10007614     qt-mt323:qt-mt323.dll
 0002:00000618       __imp_?setFrameRect@QFrame@@UAEXABVQRect@@@Z 10007618     qt-mt323:qt-mt323.dll
 0002:0000061c       __imp_?setFrameStyle@QFrame@@UAEXH@Z 1000761c     qt-mt323:qt-mt323.dll
 0002:00000620       __imp_?setGeometry@QBoxLayout@@UAEXABVQRect@@@Z 10007620     qt-mt323:qt-mt323.dll
 0002:00000624       __imp_?setGeometry@QSpacerItem@@UAEXABVQRect@@@Z 10007624     qt-mt323:qt-mt323.dll
 0002:00000628       __imp_?setHBarGeometry@QScrollView@@MAEXAAVQScrollBar@@HHHH@Z 10007628     qt-mt323:qt-mt323.dll
 0002:0000062c       __imp_?setHScrollBarMode@QScrollView@@UAEXW4ScrollBarMode@1@@Z 1000762c     qt-mt323:qt-mt323.dll
 0002:00000630       __imp_?setItalic@QTextEdit@@UAEX_N@Z 10007630     qt-mt323:qt-mt323.dll
 0002:00000634       __imp_?setLineWidth@QFrame@@UAEXH@Z 10007634     qt-mt323:qt-mt323.dll
 0002:00000638       __imp_?setLinkUnderline@QTextEdit@@UAEX_N@Z 10007638     qt-mt323:qt-mt323.dll
 0002:0000063c       __imp_?setMargin@QFrame@@UAEXH@Z 1000763c     qt-mt323:qt-mt323.dll
 0002:00000640       __imp_?setMargin@QLayout@@UAEXH@Z 10007640     qt-mt323:qt-mt323.dll
 0002:00000644       __imp_?setMargins@QScrollView@@MAEXHHHH@Z 10007644     qt-mt323:qt-mt323.dll
 0002:00000648       __imp_?setMenuBar@QLayout@@UAEXPAVQMenuBar@@@Z 10007648     qt-mt323:qt-mt323.dll
 0002:0000064c       __imp_?setMidLineWidth@QFrame@@UAEXH@Z 1000764c     qt-mt323:qt-mt323.dll
 0002:00000650       __imp_?setMimeSourceFactory@QTextEdit@@UAEXPAVQMimeSourceFactory@@@Z 10007650     qt-mt323:qt-mt323.dll
 0002:00000654       __imp_?setModified@QTextEdit@@UAEX_N@Z 10007654     qt-mt323:qt-mt323.dll
 0002:00000658       __imp_?setMovie@QLabel@@UAEXABVQMovie@@@Z 10007658     qt-mt323:qt-mt323.dll
 0002:0000065c       __imp_?setNum@QLabel@@UAEXH@Z 1000765c     qt-mt323:qt-mt323.dll
 0002:00000660       __imp_?setNum@QLabel@@UAEXN@Z 10007660     qt-mt323:qt-mt323.dll
 0002:00000664       __imp_?setOverwriteMode@QTextEdit@@UAEX_N@Z 10007664     qt-mt323:qt-mt323.dll
 0002:00000668       __imp_?setPalette@QTextEdit@@UAEXABVQPalette@@@Z 10007668     qt-mt323:qt-mt323.dll
 0002:0000066c       __imp_?setPaper@QTextEdit@@UAEXABVQBrush@@@Z 1000766c     qt-mt323:qt-mt323.dll
 0002:00000670       __imp_?setParagType@QTextEdit@@UAEXW4DisplayMode@QStyleSheetItem@@W4ListStyle@3@@Z 10007670     qt-mt323:qt-mt323.dll
 0002:00000674       __imp_?setParagraphBackgroundColor@QTextEdit@@UAEXHABVQColor@@@Z 10007674     qt-mt323:qt-mt323.dll
 0002:00000678       __imp_?setPicture@QLabel@@UAEXABVQPicture@@@Z 10007678     qt-mt323:qt-mt323.dll
 0002:0000067c       __imp_?setPixmap@QLabel@@UAEXABVQPixmap@@@Z 1000767c     qt-mt323:qt-mt323.dll
 0002:00000680       __imp_?setPointSize@QTextEdit@@UAEXH@Z 10007680     qt-mt323:qt-mt323.dll
 0002:00000684       __imp_?setReadOnly@QTextEdit@@UAEX_N@Z 10007684     qt-mt323:qt-mt323.dll
 0002:00000688       __imp_?setResizePolicy@QScrollView@@UAEXW4ResizePolicy@1@@Z 10007688     qt-mt323:qt-mt323.dll
 0002:0000068c       __imp_?setSelection@QTextEdit@@UAEXHHHHH@Z 1000768c     qt-mt323:qt-mt323.dll
 0002:00000690       __imp_?setSelectionAttributes@QTextEdit@@UAEXHABVQColor@@_N@Z 10007690     qt-mt323:qt-mt323.dll
 0002:00000694       __imp_?setSpacing@QLayout@@UAEXH@Z 10007694     qt-mt323:qt-mt323.dll
 0002:00000698       __imp_?setStyleSheet@QTextEdit@@UAEXPAVQStyleSheet@@@Z 10007698     qt-mt323:qt-mt323.dll
 0002:0000069c       __imp_?setTabStopWidth@QTextEdit@@UAEXH@Z 1000769c     qt-mt323:qt-mt323.dll
 0002:000006a0       __imp_?setText@QLabel@@UAEXABVQString@@@Z 100076a0     qt-mt323:qt-mt323.dll
 0002:000006a4       __imp_?setText@QTextEdit@@UAEXABVQString@@0@Z 100076a4     qt-mt323:qt-mt323.dll
 0002:000006a8       __imp_?setTextFormat@QTextEdit@@UAEXW4TextFormat@Qt@@@Z 100076a8     qt-mt323:qt-mt323.dll
 0002:000006ac       __imp_?setUnderline@QTextEdit@@UAEX_N@Z 100076ac     qt-mt323:qt-mt323.dll
 0002:000006b0       __imp_?setUndoDepth@QTextEdit@@UAEXH@Z 100076b0     qt-mt323:qt-mt323.dll
 0002:000006b4       __imp_?setUndoRedoEnabled@QTextEdit@@UAEX_N@Z 100076b4     qt-mt323:qt-mt323.dll
 0002:000006b8       __imp_?setVBarGeometry@QScrollView@@MAEXAAVQScrollBar@@HHHH@Z 100076b8     qt-mt323:qt-mt323.dll
 0002:000006bc       __imp_?setVScrollBarMode@QScrollView@@UAEXW4ScrollBarMode@1@@Z 100076bc     qt-mt323:qt-mt323.dll
 0002:000006c0       __imp_?setVerticalAlignment@QTextEdit@@UAEXW4VerticalAlignment@1@@Z 100076c0     qt-mt323:qt-mt323.dll
 0002:000006c4       __imp_?setWordWrap@QTextEdit@@UAEXW4WordWrap@1@@Z 100076c4     qt-mt323:qt-mt323.dll
 0002:000006c8       __imp_?setWrapColumnOrWidth@QTextEdit@@UAEXH@Z 100076c8     qt-mt323:qt-mt323.dll
 0002:000006cc       __imp_?setWrapPolicy@QTextEdit@@UAEXW4WrapPolicy@1@@Z 100076cc     qt-mt323:qt-mt323.dll
 0002:000006d0       __imp_?show@QScrollView@@UAEXXZ 100076d0     qt-mt323:qt-mt323.dll
 0002:000006d4       __imp_?sizeHint@QBoxLayout@@UBE?AVQSize@@XZ 100076d4     qt-mt323:qt-mt323.dll
 0002:000006d8       __imp_?sizeHint@QLabel@@UBE?AVQSize@@XZ 100076d8     qt-mt323:qt-mt323.dll
 0002:000006dc       __imp_?sizeHint@QSpacerItem@@UBE?AVQSize@@XZ 100076dc     qt-mt323:qt-mt323.dll
 0002:000006e0       __imp_?sizeHint@QTextEdit@@UBE?AVQSize@@XZ 100076e0     qt-mt323:qt-mt323.dll
 0002:000006e4       __imp_?spacerItem@QLayoutItem@@UAEPAVQSpacerItem@@XZ 100076e4     qt-mt323:qt-mt323.dll
 0002:000006e8       __imp_?spacerItem@QSpacerItem@@UAEPAV1@XZ 100076e8     qt-mt323:qt-mt323.dll
 0002:000006ec       __imp_?styleChange@QFrame@@MAEXAAVQStyle@@@Z 100076ec     qt-mt323:qt-mt323.dll
 0002:000006f0       __imp_?styleChange@QScrollView@@UAEXAAVQStyle@@@Z 100076f0     qt-mt323:qt-mt323.dll
 0002:000006f4       __imp_?sync@QTextEdit@@UAEXXZ 100076f4     qt-mt323:qt-mt323.dll
 0002:000006f8       __imp_?undo@QTextEdit@@UAEXXZ 100076f8     qt-mt323:qt-mt323.dll
 0002:000006fc       __imp_?viewportContextMenuEvent@QScrollView@@MAEXPAVQContextMenuEvent@@@Z 100076fc     qt-mt323:qt-mt323.dll
 0002:00000700       __imp_?viewportDragEnterEvent@QScrollView@@MAEXPAVQDragEnterEvent@@@Z 10007700     qt-mt323:qt-mt323.dll
 0002:00000704       __imp_?viewportDragLeaveEvent@QScrollView@@MAEXPAVQDragLeaveEvent@@@Z 10007704     qt-mt323:qt-mt323.dll
 0002:00000708       __imp_?viewportDragMoveEvent@QScrollView@@MAEXPAVQDragMoveEvent@@@Z 10007708     qt-mt323:qt-mt323.dll
 0002:0000070c       __imp_?viewportDropEvent@QScrollView@@MAEXPAVQDropEvent@@@Z 1000770c     qt-mt323:qt-mt323.dll
 0002:00000710       __imp_?viewportMouseDoubleClickEvent@QScrollView@@MAEXPAVQMouseEvent@@@Z 10007710     qt-mt323:qt-mt323.dll
 0002:00000714       __imp_?viewportMouseMoveEvent@QScrollView@@MAEXPAVQMouseEvent@@@Z 10007714     qt-mt323:qt-mt323.dll
 0002:00000718       __imp_?viewportMousePressEvent@QScrollView@@MAEXPAVQMouseEvent@@@Z 10007718     qt-mt323:qt-mt323.dll
 0002:0000071c       __imp_?viewportMouseReleaseEvent@QScrollView@@MAEXPAVQMouseEvent@@@Z 1000771c     qt-mt323:qt-mt323.dll
 0002:00000720       __imp_?viewportPaintEvent@QScrollView@@MAEXPAVQPaintEvent@@@Z 10007720     qt-mt323:qt-mt323.dll
 0002:00000724       __imp_?viewportResizeEvent@QTextEdit@@MAEXPAVQResizeEvent@@@Z 10007724     qt-mt323:qt-mt323.dll
 0002:00000728       __imp_?viewportWheelEvent@QScrollView@@MAEXPAVQWheelEvent@@@Z 10007728     qt-mt323:qt-mt323.dll
 0002:0000072c       __imp_?wheelEvent@QScrollView@@MAEXPAVQWheelEvent@@@Z 1000772c     qt-mt323:qt-mt323.dll
 0002:00000730       __imp_?widget@QLayoutItem@@UAEPAVQWidget@@XZ 10007730     qt-mt323:qt-mt323.dll
 0002:00000734       __imp_?windowActivationChange@QTextEdit@@MAEX_N@Z 10007734     qt-mt323:qt-mt323.dll
 0002:00000738       __imp_?zoomIn@QTextEdit@@UAEXH@Z 10007738     qt-mt323:qt-mt323.dll
 0002:0000073c       __imp_?zoomIn@QTextEdit@@UAEXXZ 1000773c     qt-mt323:qt-mt323.dll
 0002:00000740       __imp_?zoomOut@QTextEdit@@UAEXH@Z 10007740     qt-mt323:qt-mt323.dll
 0002:00000744       __imp_?zoomOut@QTextEdit@@UAEXXZ 10007744     qt-mt323:qt-mt323.dll
 0002:00000748       __imp_?zoomTo@QTextEdit@@UAEXH@Z 10007748     qt-mt323:qt-mt323.dll
 0002:0000074c       __imp_??0QPixmap@@QAE@QAPBD@Z 1000774c     qt-mt323:qt-mt323.dll
 0002:00000750       __imp_?null@QString@@2V1@A 10007750     qt-mt323:qt-mt323.dll
 0002:00000754       __imp_?close@QFile@@UAEXXZ 10007754     qt-mt323:qt-mt323.dll
 0002:00000758       __imp_?open@QFile@@UAE_NH@Z 10007758     qt-mt323:qt-mt323.dll
 0002:0000075c       __imp_??1QFile@@UAE@XZ     1000775c     qt-mt323:qt-mt323.dll
 0002:00000760       __imp_??0QFile@@QAE@ABVQString@@@Z 10007760     qt-mt323:qt-mt323.dll
 0002:00000764       __imp_?attribute@QDomElement@@QBE?AVQString@@ABV2@0@Z 10007764     qt-mt323:qt-mt323.dll
 0002:00000768       __imp_??1QDomElement@@UAE@XZ 10007768     qt-mt323:qt-mt323.dll
 0002:0000076c       __imp_?setContent@QDomDocument@@QAE_NPAVQIODevice@@PAVQString@@PAH2@Z 1000776c     qt-mt323:qt-mt323.dll
 0002:00000770       __imp_?documentElement@QDomDocument@@QBE?AVQDomElement@@XZ 10007770     qt-mt323:qt-mt323.dll
 0002:00000774       __imp_??1QDomDocument@@UAE@XZ 10007774     qt-mt323:qt-mt323.dll
 0002:00000778       __imp_??0QDomDocument@@QAE@XZ 10007778     qt-mt323:qt-mt323.dll
 0002:0000077c       __imp_?toElement@QDomNode@@QAE?AVQDomElement@@XZ 1000777c     qt-mt323:qt-mt323.dll
 0002:00000780       __imp_?isNull@QDomNode@@QBE_NXZ 10007780     qt-mt323:qt-mt323.dll
 0002:00000784       __imp_?nextSibling@QDomNode@@UBE?AV1@XZ 10007784     qt-mt323:qt-mt323.dll
 0002:00000788       __imp_?firstChild@QDomNode@@UBE?AV1@XZ 10007788     qt-mt323:qt-mt323.dll
 0002:0000078c       __imp_??1QDomNode@@UAE@XZ  1000778c     qt-mt323:qt-mt323.dll
 0002:00000790       __imp_??4QDomNode@@QAEAAV0@ABV0@@Z 10007790     qt-mt323:qt-mt323.dll
 0002:00000794       __imp_??1QStringList@@QAE@XZ 10007794     qt-mt323:qt-mt323.dll
 0002:00000798       __imp_??0QStringList@@QAE@ABV0@@Z 10007798     qt-mt323:qt-mt323.dll
 0002:0000079c       __imp_??0QStringList@@QAE@XZ 1000779c     qt-mt323:qt-mt323.dll
 0002:000007a0       __imp_??A?$QValueList@VQString@@@@QAEAAVQString@@I@Z 100077a0     qt-mt323:qt-mt323.dll
 0002:000007a4       __imp_?findIndex@?$QValueList@VQString@@@@QBEHABVQString@@@Z 100077a4     qt-mt323:qt-mt323.dll
 0002:000007a8       __imp_??Y?$QValueList@VQString@@@@QAEAAV0@ABV0@@Z 100077a8     qt-mt323:qt-mt323.dll
 0002:000007ac       __imp_??6?$QValueList@VQString@@@@QAEAAV0@ABVQString@@@Z 100077ac     qt-mt323:qt-mt323.dll
 0002:000007b0       __imp_??H@YA?BVQString@@ABV0@PBD@Z 100077b0     qt-mt323:qt-mt323.dll
 0002:000007b4       __imp_??8@YA_NABVQString@@0@Z 100077b4     qt-mt323:qt-mt323.dll
 0002:000007b8       __imp_??4QString@@QAEAAV0@ABV0@@Z 100077b8     qt-mt323:qt-mt323.dll
 0002:000007bc       __imp_??1QString@@QAE@XZ   100077bc     qt-mt323:qt-mt323.dll
 0002:000007c0       __imp_??0QString@@QAE@PBD@Z 100077c0     qt-mt323:qt-mt323.dll
 0002:000007c4       __imp_??0QString@@QAE@ABV0@@Z 100077c4     qt-mt323:qt-mt323.dll
 0002:000007c8       __imp_?addItem@QBoxLayout@@UAEXPAVQLayoutItem@@@Z 100077c8     qt-mt323:qt-mt323.dll
 0002:000007cc       __imp_??0QString@@QAE@XZ   100077cc     qt-mt323:qt-mt323.dll
 0002:000007d0       \177qt-mt323_NULL_THUNK_DATA 100077d0     qt-mt323:qt-mt323.dll
 0002:000007d4       ___xc_a                    100077d4     MSVCRT:cinitexe.obj
 0002:000007e4       ___xc_z                    100077e4     MSVCRT:cinitexe.obj
 0002:000007e8       ___xi_a                    100077e8     MSVCRT:cinitexe.obj
 0002:000007f4       ___xi_z                    100077f4     MSVCRT:cinitexe.obj
 0002:000007fc       ??_7config@@6B@            100077fc     config.obj
 0002:00000800       ??_C@_0CB@PAJCIMGI@Home?1User?5Interface?1Applications@ 10007800     config.obj
 0002:00000824       ??_C@_0DE@IHFGAIPG@Home?1System?1Workstation?5Update?1N@ 10007824     config.obj
 0002:00000858       ??_C@_0DG@OBIJJHND@Home?1System?1Workstation?5Update?1P@ 10007858     config.obj
 0002:00000890       ??_C@_0DF@KIHLMPK@Home?1System?1Workstation?5Update?1P@ 10007890     config.obj
 0002:000008c8       ??_C@_0CC@PEHOMNH@Home?1User?5Interface?1Panel?5Manage@ 100078c8     config.obj
 0002:000008ec       ??_C@_0CC@NFBKEABD@Home?1User?5Interface?1Type?5Handler@ 100078ec     config.obj
 0002:00000910       ??_C@_0BM@DDNKKIBO@Home?1System?1Object?1Settings?$AA@ 10007910     config.obj
 0002:0000092c       ??_C@_0CC@JBCIFMEP@Home?1System?1Workstations?1Setting@ 1000792c     config.obj
 0002:00000950       ??_C@_0BP@KBDBOBLL@Home?1User?5Interface?1Panel?5Sets?$AA@ 10007950     config.obj
 0002:00000970       ??_C@_0CH@DCOKFHME@Home?1User?5Interface?1Default?5Styl@ 10007970     config.obj
 0002:00000998       ??_C@_0CA@IDDAGIMM@Home?1Developer?1Vis?4?5Ed?4?5Buttons?$AA@ 10007998     config.obj
 0002:000009b8       ??_C@_0CK@ELPMFKLJ@Home?1Developer?1Generic?5config?5te@ 100079b8     config.obj
 0002:000009e4       ??_C@_0BH@FINFEFEI@Home?1System?1Log?5Delete?$AA@ 100079e4     config.obj
 0002:000009fc       ??_C@_0BA@DOLGMJC@UI?5Applications?$AA@ 100079fc     config.obj
 0002:00000a0c       ??_C@_0BJ@OPFECNJI@Batch?5file?5after?5no?9sync?$AA@ 10007a0c     config.obj
 0002:00000a28       ??_C@_0CC@CJFPGPFI@Batch?5file?5after?5sync?5with?5serve@ 10007a28     config.obj
 0002:00000a4c       ??_C@_0CD@DGKPGNNG@Batch?5file?5before?5sync?5with?5serv@ 10007a4c     config.obj
 0002:00000a70       ??_C@_0BM@KFMHFIDN@Panel?5Manager?5Configuration?$AA@ 10007a70     config.obj
 0002:00000a8c       ??_C@_0CI@BOLEANNC@Default?5User?5Interface?5for?5Devic@ 10007a8c     config.obj
 0002:00000ab4       ??_C@_0BG@HAELADPG@Misc?4?5Object?5Settings?$AA@ 10007ab4     config.obj
 0002:00000acc       ??_C@_0CA@JEDPHAPO@Individual?5Workstation?5Settings?$AA@ 10007acc     config.obj
 0002:00000aec       ??_C@_0DA@OBINNNOG@Panelman?5Application?5Configurati@ 10007aec     config.obj
 0002:00000b1c       ??_C@_0CE@JGKLCJJK@Default?5Stylesheet?5?$CIbncs_style?4x@ 10007b1c     config.obj
 0002:00000b40       ??_C@_0CD@NHNJMDBI@Visual?5Editor?5Button?5Configurati@ 10007b40     config.obj
 0002:00000b64       ??_C@_0DA@IHPEDEEE@Generic?5Configuration?5Text?5Edito@ 10007b64     config.obj
 0002:00000b94       ??_C@_0BG@JLLAPFDA@Deletion?5of?5old?5files?$AA@ 10007b94     config.obj
 0002:00000bac       ??_C@_0BI@CJELKHOM@config?1applications?4xml?$AA@ 10007bac     config.obj
 0002:00000bc4       ??_C@_0BH@NICNDPNG@windows?1bin?1nosync?4bat?$AA@ 10007bc4     config.obj
 0002:00000bdc       ??_C@_0BJ@EICPECHE@windows?1bin?1postsync?4bat?$AA@ 10007bdc     config.obj
 0002:00000bf8       ??_C@_0BI@CKNKBBEO@windows?1bin?1presync?4bat?$AA@ 10007bf8     config.obj
 0002:00000c10       ??_C@_0BE@PIBKGEME@config?1g_pnlman?4ini?$AA@ 10007c10     config.obj
 0002:00000c24       ??_C@_0BI@EHELLOIK@config?1typehandlers?4xml?$AA@ 10007c24     config.obj
 0002:00000c3c       ??_C@_0BL@LAFHKIHL@config?1object_settings?4xml?$AA@ 10007c3c     config.obj
 0002:00000c58       ??_C@_0CA@CGOJCLNG@config?1workstation_settings?4xml?$AA@ 10007c58     config.obj
 0002:00000c78       ??_C@_0BF@GGAPJNIF@config?1panelsets?4xml?$AA@ 10007c78     config.obj
 0002:00000c90       ??_C@_0CB@FEPFMKLB@config?1stylesheet?1bncs_style?4xml@ 10007c90     config.obj
 0002:00000cb4       ??_C@_0BJ@PHPALLJJ@config?1vised?1buttons?4xml?$AA@ 10007cb4     config.obj
 0002:00000cd0       ??_C@_0CE@EKIDLFAD@config?1plugins?1textPluginConfig?4@ 10007cd0     config.obj
 0002:00000cf4       ??_C@_0BF@NGGKJOMJ@config?1logdelete?4xml?$AA@ 10007cf4     config.obj
 0002:00000d0c       ??_C@_0DJ@CCFIKHF@Applications?5that?5can?5appear?5on?5@ 10007d0c     config.obj
 0002:00000d48       ??_C@_0KL@ELOJFOHM@The?5batch?5file?5that?5runs?5if?5this@ 10007d48     config.obj
 0002:00000df8       ??_C@_0OK@JBOFCOCC@The?5batch?5file?5that?5runs?5after?5t@ 10007df8     config.obj
 0002:00000ee8       ??_C@_0OE@LMLBNFKD@The?5batch?5file?5that?5runs?5before?5@ 10007ee8     config.obj
 0002:00000fcc       ??_C@_0BH@IJLNLCBP@Panelman?5configuration?$AA@ 10007fcc     config.obj
 0002:00000fe8       ??_C@_0EB@BIOJABDJ@What?5applications?5are?5default?5vi@ 10007fe8     config.obj
 0002:00001030       ??_C@_0EB@CNLMAKBN@Misc?4?5object?5settings?5?9?5a?5simple@ 10008030     config.obj
 0002:00001078       ??_C@_0EG@OGEBIPBP@Misc?4?5workstation?5settings?5?9?5a?5s@ 10008078     config.obj
 0002:000010c0       ??_C@_0EF@MEKHHFIP@Groups?5of?5panels?5as?5they?5appear?5@ 100080c0     config.obj
 0002:00001108       ??_C@_0BH@CJGPLCE@The?5default?5stylesheet?$AA@ 10008108     config.obj
 0002:00001120       ??_C@_0EP@OIMGINCG@The?5buttons?5as?5they?5appear?5in?5th@ 10008120     config.obj
 0002:00001170       ??_C@_0PG@KJOALGIM@File?5in?5the?5format?3?$DMpre?$DO?$CGlt?$DL?$DPxml@ 10008170     config.obj
 0002:00001268       ??_C@_0FN@LJJCBKPJ@Select?5what?5files?5are?5deleted?5wh@ 10008268     config.obj
 0002:000012c8       ??_C@_0CF@CIAIAFGJ@?1config?1plugins?1textPluginConfig@ 100082c8     config.obj
 0002:000012f0       ??_C@_03ICHNJLJF@key?$AA@  100082f0     config.obj
 0002:000012f4       ??_C@_0M@PPJNHBMP@description?$AA@ 100082f4     config.obj
 0002:00001300       ??_C@_08BABJIOEM@filename?$AA@ 10008300     config.obj
 0002:0000130c       ??_C@_04PCJFHION@help?$AA@ 1000830c     config.obj
 0002:00001311       ??_C@_00CNPNBAHC@?$AA@     10008311     config.obj
 0002:00001314       ??_C@_09FNFPFPED@14?514?53?51?$AA@ 10008314     plugindesc.obj
 0002:00001320       ??_C@_0M@KEPPNGJB@?$CD?5c?5?$CD000000?$AA@ 10008320     plugindesc.obj
 0002:0000132c       ??_C@_0M@HFCLKLOA@a?5c?5?$CD808080?$AA@ 1000832c     plugindesc.obj
 0002:00001338       ??_C@_0M@HNGHCCNN@?4?5c?5?$CDffffff?$AA@ 10008338     plugindesc.obj
 0002:00001344       ??_C@_0P@HFKAALMG@?4?4?4?4?4?4?4?4?4?4?4?4?4?4?$AA@ 10008344     plugindesc.obj
 0002:00001354       ??_C@_0P@MLHMKILI@?4?4?4?4?4?4?4?$CD?$CD?$CD?$CD?4?4?4?$AA@ 10008354     plugindesc.obj
 0002:00001364       ??_C@_0P@OHHKDNPB@?4?4?4?4?4?4?$CD?$CD?4?4?$CD?4?4?4?$AA@ 10008364     plugindesc.obj
 0002:00001374       ??_C@_0P@ODMLFBBG@?4?4?4?4?4?$CD?4?$CD?4?4?$CD?4?4?4?$AA@ 10008374     plugindesc.obj
 0002:00001384       ??_C@_0P@GPOCJCDB@?4?4?4?4?$CD?4?4?$CDa?4?$CD?4?4?4?$AA@ 10008384     plugindesc.obj
 0002:00001394       ??_C@_0P@EHLPPKKI@?4?4?4?$CD?$CD?$CD?$CD?$CD?4?4?$CD?4?4?4?$AA@ 10008394     plugindesc.obj
 0002:000013a4       ??_C@_0P@DPPLILLD@?4?4?4?$CD?4aaaa?4?$CD?4?4?4?$AA@ 100083a4     plugindesc.obj
 0002:000013b4       ??_C@_0P@BDJPMOJJ@?4?4?4?$CD?4?4?4?4?4?4?$CD?4?4?4?$AA@ 100083b4     plugindesc.obj
 0002:000013c4       ??_C@_0P@JKPGIILG@?4?4?4?$CD?$CD?$CD?$CD?$CD?$CD?$CD?$CD?4?4?4?$AA@ 100083c4     plugindesc.obj
 0002:000013d8       ??_7config_plugin_desc_base@@6B@ 100083d8     plugindesc.obj
 0002:000013ec       ??_7plugindesc@@6B@        100083ec     plugindesc.obj
 0002:00001400       ??_7text_highlighter@@6B@  10008400     text_highlighter.obj
 0002:00001408       ??_C@_05BIMBDNDC@black?$AA@ 10008408     text_highlighter.obj
 0002:00001410       ??_C@_02CBLDBPFN@?1?1?$AA@ 10008410     text_highlighter.obj
 0002:00001414       ??_C@_01ICJEACDI@?$DL?$AA@ 10008414     text_highlighter.obj
 0002:00001418       ??_C@_02GIPFHKNO@OK?$AA@   10008418     textPlugin.obj
 0002:00001424       ??_SQGuardedPtrPrivate@@6B@ 10008424     textPlugin.obj
 0002:00001478       ??_7QDockWindowList@@6B@   10008478     textPlugin.obj
 0002:0000149c       ??_7?$QPtrList@VQPopupMenu@@@@6B@ 1000849c     textPlugin.obj
 0002:000014c0       ??_7QPopupMenuList@@6B@    100084c0     textPlugin.obj
 0002:000014e0       ??_C@_04OOEBCMBF@FAIL?$AA@ 100084e0     textPlugin.obj
 0002:000014e8       ??_C@_08OBALAKLA@READONLY?$AA@ 100084e8     textPlugin.obj
 0002:000014f4       ??_C@_04KANDKFIK@DONE?$AA@ 100084f4     textPlugin.obj
 0002:000014fc       ??_C@_07NFANNNEC@UNKNOWN?$AA@ 100084fc     textPlugin.obj
 0002:00001508       ??_7config_plugin_base@@6BQObject@@@ 10008508     textPlugin.obj
 0002:000016e0       ??_7config_plugin_base@@6BQPaintDevice@@@ 100086e0     textPlugin.obj
 0002:00001700       ??_C@_0EB@GNDACMDJ@?$CC?5?9?5the?5author?5should?5have?5defin@ 10008700     textPlugin.obj
 0002:00001744       ??_C@_0CH@BDPDPLDP@This?5is?5the?5default?5?$CCAbout?$CC?5text@ 10008744     textPlugin.obj
 0002:00001770       ??_7?$QDict@VQAction@@@@6B@ 10008770     textPlugin.obj
 0002:00001790       ??_7textPlugin@@6BQObject@@@ 10008790     textPlugin.obj
 0002:00001968       ??_7textPlugin@@6BQPaintDevice@@@ 10008968     textPlugin.obj
 0002:00001988       ??_C@_0N@CMGAMHCH@textPlugin?3?5?$AA@ 10008988     textPlugin.obj
 0002:00001998       ??_C@_0M@LIJDBMP@?$DMh1?$DO?$CF1?$DM?1h1?$DO?$AA@ 10008998     textPlugin.obj
 0002:000019a4       ??_C@_0BN@CEGLABJP@2command?$CI?5QString?0?5QString?5?$CJ?$AA@ 100089a4     textPlugin.obj
 0002:000019c4       ??_C@_06BNCCALCL@unlock?$AA@ 100089c4     textPlugin.obj
 0002:000019cc       ??_C@_09JLEOPMAJ@?5?9?5error?$DN?$AA@ 100089cc     textPlugin.obj
 0002:000019d8       ??_C@_09LBCHCBIC@?5?9?5value?$DN?$AA@ 100089d8     textPlugin.obj
 0002:000019e4       ??_C@_0P@ELNNACEA@?5?9?5textStatus?$DN?$AA@ 100089e4     textPlugin.obj
 0002:000019f4       ??_C@_0L@LEAPMKGP@Reply?3?5op?$DN?$AA@ 100089f4     textPlugin.obj
 0002:00001a00       ??_C@_08HNIAHLMM@download?$AA@ 10008a00     textPlugin.obj
 0002:00001a0c       ??_C@_01KMDKNFGN@?1?$AA@   10008a0c     textPlugin.obj
 0002:00001a10       ??_C@_06KAOCKAGB@upload?$AA@ 10008a10     textPlugin.obj
 0002:00001a18       ??_C@_05CCAMFJOL@clean?$AA@ 10008a18     textPlugin.obj
 0002:00001a20       ??_C@_0IE@KAKGLGIF@?$DMp?$DO?$DMb?$DOFile?5not?5found?5and?5will?5be@ 10008a20     textPlugin.obj
 0002:00001aa4       ??_C@_0M@EBFEGAAI@Information?$AA@ 10008aa4     textPlugin.obj
 0002:00001ab0       ??_C@_05CFEJGMAI@dirty?$AA@ 10008ab0     textPlugin.obj
 0002:00001ab8       ??_C@_0CO@GKAEALGF@Being?5asked?5to?5navigate?5to?5?$CF1?5wi@ 10008ab8     textPlugin.obj
 0002:00001ae8       ??_C@_0N@EHHLDFOB@checkoutFile?$AA@ 10008ae8     textPlugin.obj
 0002:00001af8       ??_C@_04GNBLKAFA@?4XML?$AA@ 10008af8     textPlugin.obj
 0002:00001b00       ??_C@_0CI@KMJGKAMM@Error?5in?5XML?5?$CC?$CF1?$CC?5at?5line?5?$CF2?0?5co@ 10008b00     textPlugin.obj
 0002:00001b28       ??_C@_09GLNHIMFF@XML?5Error?$AA@ 10008b28     textPlugin.obj
 0002:00001b34       ??_C@_0L@CIKGEHEG@uploadFile?$AA@ 10008b34     textPlugin.obj
 0002:00001b40       ??_C@_0FC@LKHKDOLO@?$DMh3?$DOGeneric?5Text?5Configuration?5P@ 10008b40     textPlugin.obj
 0002:00001b94       ??_C@_08FIIOCAOP@13?324?350?$AA@ 10008b94     textPlugin.obj
 0002:00001ba0       ??_C@_0M@JEDEHNP@Sep?523?52021?$AA@ 10008ba0     textPlugin.obj
 0002:00001bb0       ??_7textPluginDlg@@6BQObject@@@ 10008bb0     textPlugindlgimpl.obj
 0002:00001d68       ??_7textPluginDlg@@6BQPaintDevice@@@ 10008d68     textPlugindlgimpl.obj
 0002:00001d88       ??_C@_0P@GFDCCPD@1textChanged?$CI?$CJ?$AA@ 10008d88     textPlugindlgimpl.obj
 0002:00001d98       ??_C@_0P@BHCOEIIK@2textChanged?$CI?$CJ?$AA@ 10008d98     textPlugindlgimpl.obj
 0002:00001da8       ?keywords@xml_highlighter@@0QBQBDB 10008da8     xml_highlighter.obj
 0002:00001dd8       ?delimiters@xml_highlighter@@0QBQBDB 10008dd8     xml_highlighter.obj
 0002:00001de4       ?quotes@xml_highlighter@@0QBQBDB 10008de4     xml_highlighter.obj
 0002:00001df8       ??_C@_01MNNFJEPP@?$DM?$AA@ 10008df8     xml_highlighter.obj
 0002:00001dfc       ??_C@_02HCGKDMEN@?1?$DO?$AA@ 10008dfc     xml_highlighter.obj
 0002:00001e00       ??_C@_01NEMOKFLO@?$DN?$AA@ 10008e00     xml_highlighter.obj
 0002:00001e04       ??_C@_02EGCJHIOB@id?$AA@   10008e04     xml_highlighter.obj
 0002:00001e08       ??_C@_07BANDPJOM@caption?$AA@ 10008e08     xml_highlighter.obj
 0002:00001e10       ??_C@_05PHLGJONK@title?$AA@ 10008e10     xml_highlighter.obj
 0002:00001e18       ??_C@_05LJDNNBIK@param?$AA@ 10008e18     xml_highlighter.obj
 0002:00001e20       ??_C@_04GPMDFGEJ@type?$AA@ 10008e20     xml_highlighter.obj
 0002:00001e28       ??_C@_05ENKANFLO@class?$AA@ 10008e28     xml_highlighter.obj
 0002:00001e30       ??_C@_04DMJJIPAH@icon?$AA@ 10008e30     xml_highlighter.obj
 0002:00001e38       ??_C@_07DLHCIBDH@default?$AA@ 10008e38     xml_highlighter.obj
 0002:00001e40       ??_C@_01GEODFPGF@?8?$AA@   10008e40     xml_highlighter.obj
 0002:00001e44       ??_C@_01BJJEKLCA@?$CC?$AA@ 10008e44     xml_highlighter.obj
 0002:00001e48       ??_C@_01OHGJGJJP@?$FL?$AA@ 10008e48     xml_highlighter.obj
 0002:00001e4c       ??_C@_01LBDDMOBJ@?$FN?$AA@ 10008e4c     xml_highlighter.obj
 0002:00001e50       ??_C@_01CLKCMJKC@?5?$AA@   10008e50     xml_highlighter.obj
 0002:00001e58       ??_7xml_highlighter@@6B@   10008e58     xml_highlighter.obj
 0002:00001e60       ??_C@_0BM@BJMCMKGI@XML?5highlighter?5destruction?$AA@ 10008e60     xml_highlighter.obj
 0002:00001e7c       ??_C@_09MHNMOMAI@darkgreen?$AA@ 10008e7c     xml_highlighter.obj
 0002:00001e88       ??_C@_04OBGPFBCN@blue?$AA@ 10008e88     xml_highlighter.obj
 0002:00001e90       ??_C@_07MFAOOMGP@darkred?$AA@ 10008e90     xml_highlighter.obj
 0002:00001e98       ??_C@_0L@PJHEGOOE@textPlugin?$AA@ 10008e98     moc_textPlugin.obj
 0002:00001eb0       ??_C@_07KMMNMMFF@command?$AA@ 10008eb0     moc_textPlugin.obj
 0002:00001ec4       ??_C@_0BJ@FEFNJDLM@command?$CIQString?0QString?$CJ?$AA@ 10008ec4     moc_textPlugin.obj
 0002:00001ee0       ??_C@_0BC@CJIJPEMM@textPluginDlgBase?$AA@ 10008ee0     moc_textPlugindlg.obj
 0002:00001f00       ??_C@_0P@DMEOIADN@languageChange?$AA@ 10008f00     moc_textPlugindlg.obj
 0002:00001f1c       ??_C@_0BB@PFEIHPGD@languageChange?$CI?$CJ?$AA@ 10008f1c     moc_textPlugindlg.obj
 0002:00001f30       ??_C@_0O@HNPKILMH@textPluginDlg?$AA@ 10008f30     moc_textPlugindlgimpl.obj
 0002:00001f4c       ??_C@_0M@NJKJFEFJ@textChanged?$AA@ 10008f4c     moc_textPlugindlgimpl.obj
 0002:00001f64       ??_C@_0O@HFGHCCOK@textChanged?$CI?$CJ?$AA@ 10008f64     moc_textPlugindlgimpl.obj
 0002:00001f90       ??_7textPluginDlgBase@@6BQObject@@@ 10008f90     textPlugindlg.obj
 0002:00002148       ??_7textPluginDlgBase@@6BQPaintDevice@@@ 10009148     textPlugindlg.obj
 0002:0000216c       ??_SQLabel@@6BQObject@@@   1000916c     textPlugindlg.obj
 0002:00002364       ??_SQLabel@@6BQPaintDevice@@@ 10009364     textPlugindlg.obj
 0002:0000238c       ??_SQTextEdit@@6BQObject@@@ 1000938c     textPlugindlg.obj
 0002:00002708       ??_SQTextEdit@@6BQPaintDevice@@@ 10009708     textPlugindlg.obj
 0002:0000272c       ??_SQSpacerItem@@6B@       1000972c     textPlugindlg.obj
 0002:00002774       ??_SQHBoxLayout@@6BQObject@@@ 10009774     textPlugindlg.obj
 0002:000027dc       ??_SQHBoxLayout@@6BQLayoutItem@@@ 100097dc     textPlugindlg.obj
 0002:00002824       ??_SQVBoxLayout@@6BQObject@@@ 10009824     textPlugindlg.obj
 0002:0000288c       ??_SQVBoxLayout@@6BQLayoutItem@@@ 1000988c     textPlugindlg.obj
 0002:000028cc       ??_C@_0BI@LCLOBMNM@textPluginDlgBaseLayout?$AA@ 100098cc     textPlugindlg.obj
 0002:000028e4       ??_C@_0N@CJBMCOMC@textLabel1_4?$AA@ 100098e4     textPlugindlg.obj
 0002:000028f4       ??_C@_09HCBNDNHI@textEdit1?$AA@ 100098f4     textPlugindlg.obj
 0002:00002900       ??_C@_07MOFDPJDG@layout1?$AA@ 10009900     textPlugindlg.obj
 0002:00002908       ??_C@_0L@INJINICK@textLabel2?$AA@ 10009908     textPlugindlg.obj
 0002:00002914       ??_C@_0O@DADHIOM@filenameLabel?$AA@ 10009914     textPlugindlg.obj
 0002:00002924       ??_C@_09BFIOMJJM@Filename?3?$AA@ 10009924     textPlugindlg.obj
 0002:00002934       ??_7type_info@@6B@         10009934     MSVCRT:ti_inst.obj
 0002:00002938       __pDefaultRawDllMain       10009938     MSVCRT:crtdll.obj
 0002:00002938       __pRawDllMain              10009938     MSVCRT:crtdll.obj
 0002:00002948       __load_config_used         10009948     MSVCRT:loadcfg.obj
 0002:00002990       ??_R4config@@6B@           10009990     config.obj
 0002:000029a4       ??_R3config@@8             100099a4     config.obj
 0002:000029b4       ??_R2config@@8             100099b4     config.obj
 0002:000029bc       ??_R1A@?0A@EA@config@@8    100099bc     config.obj
 0002:000029d8       ??_R4config_plugin_desc_base@@6B@ 100099d8     plugindesc.obj
 0002:000029ec       ??_R3config_plugin_desc_base@@8 100099ec     plugindesc.obj
 0002:000029fc       ??_R2config_plugin_desc_base@@8 100099fc     plugindesc.obj
 0002:00002a04       ??_R1A@?0A@EA@config_plugin_desc_base@@8 10009a04     plugindesc.obj
 0002:00002a20       ??_R4plugindesc@@6B@       10009a20     plugindesc.obj
 0002:00002a34       ??_R3plugindesc@@8         10009a34     plugindesc.obj
 0002:00002a44       ??_R2plugindesc@@8         10009a44     plugindesc.obj
 0002:00002a50       ??_R1A@?0A@EA@plugindesc@@8 10009a50     plugindesc.obj
 0002:00002a6c       ??_R4text_highlighter@@6B@ 10009a6c     text_highlighter.obj
 0002:00002a80       ??_R3text_highlighter@@8   10009a80     text_highlighter.obj
 0002:00002a90       ??_R2text_highlighter@@8   10009a90     text_highlighter.obj
 0002:00002aa0       ??_R1A@?0A@EA@text_highlighter@@8 10009aa0     text_highlighter.obj
 0002:00002abc       ??_R1A@?0A@EA@QSyntaxHighlighter@@8 10009abc     text_highlighter.obj
 0002:00002ad8       ??_R3QSyntaxHighlighter@@8 10009ad8     text_highlighter.obj
 0002:00002ae8       ??_R2QSyntaxHighlighter@@8 10009ae8     text_highlighter.obj
 0002:00002af4       ??_R13?0A@EA@Qt@@8         10009af4     text_highlighter.obj
 0002:00002b10       ??_R3Qt@@8                 10009b10     text_highlighter.obj
 0002:00002b20       ??_R2Qt@@8                 10009b20     text_highlighter.obj
 0002:00002b28       ??_R1A@?0A@EA@Qt@@8        10009b28     text_highlighter.obj
 0002:00002b44       ??_R3QShared@@8            10009b44     textPlugin.obj
 0002:00002b54       ??_R2QShared@@8            10009b54     textPlugin.obj
 0002:00002b5c       ??_R1A@?0A@EA@QShared@@8   10009b5c     textPlugin.obj
 0002:00002b78       ??_R1A@?0A@EA@QGList@@8    10009b78     textPlugin.obj
 0002:00002b94       ??_R3QGList@@8             10009b94     textPlugin.obj
 0002:00002ba4       ??_R2QGList@@8             10009ba4     textPlugin.obj
 0002:00002bb0       ??_R1A@?0A@EA@QPtrCollection@@8 10009bb0     textPlugin.obj
 0002:00002bcc       ??_R3QPtrCollection@@8     10009bcc     textPlugin.obj
 0002:00002bdc       ??_R2QPtrCollection@@8     10009bdc     textPlugin.obj
 0002:00002be4       ??_R4QGuardedPtrPrivate@@6B@ 10009be4     textPlugin.obj
 0002:00002bf8       ??_R3QGuardedPtrPrivate@@8 10009bf8     textPlugin.obj
 0002:00002c08       ??_R2QGuardedPtrPrivate@@8 10009c08     textPlugin.obj
 0002:00002c1c       ??_R1A@?0A@EA@QGuardedPtrPrivate@@8 10009c1c     textPlugin.obj
 0002:00002c38       ??_R1A@?0A@EA@QObject@@8   10009c38     textPlugin.obj
 0002:00002c54       ??_R3QObject@@8            10009c54     textPlugin.obj
 0002:00002c64       ??_R2QObject@@8            10009c64     textPlugin.obj
 0002:00002c70       ??_R1CI@?0A@EA@QShared@@8  10009c70     textPlugin.obj
 0002:00002c8c       ??_R4QDockWindowList@@6B@  10009c8c     textPlugin.obj
 0002:00002ca0       ??_R3QDockWindowList@@8    10009ca0     textPlugin.obj
 0002:00002cb0       ??_R2QDockWindowList@@8    10009cb0     textPlugin.obj
 0002:00002cc4       ??_R1A@?0A@EA@QDockWindowList@@8 10009cc4     textPlugin.obj
 0002:00002ce0       ??_R1A@?0A@EA@?$QPtrList@VQDockWindow@@@@8 10009ce0     textPlugin.obj
 0002:00002cfc       ??_R3?$QPtrList@VQDockWindow@@@@8 10009cfc     textPlugin.obj
 0002:00002d0c       ??_R2?$QPtrList@VQDockWindow@@@@8 10009d0c     textPlugin.obj
 0002:00002d1c       ??_R4QPopupMenuList@@6B@   10009d1c     textPlugin.obj
 0002:00002d30       ??_R3QPopupMenuList@@8     10009d30     textPlugin.obj
 0002:00002d40       ??_R2QPopupMenuList@@8     10009d40     textPlugin.obj
 0002:00002d54       ??_R1A@?0A@EA@QPopupMenuList@@8 10009d54     textPlugin.obj
 0002:00002d70       ??_R1A@?0A@EA@?$QPtrList@VQPopupMenu@@@@8 10009d70     textPlugin.obj
 0002:00002d8c       ??_R3?$QPtrList@VQPopupMenu@@@@8 10009d8c     textPlugin.obj
 0002:00002d9c       ??_R2?$QPtrList@VQPopupMenu@@@@8 10009d9c     textPlugin.obj
 0002:00002dac       ??_R4?$QPtrList@VQPopupMenu@@@@6B@ 10009dac     textPlugin.obj
 0002:00002dc0       ??_R4config_plugin_base@@6BQObject@@@ 10009dc0     textPlugin.obj
 0002:00002dd4       ??_R3config_plugin_base@@8 10009dd4     textPlugin.obj
 0002:00002de4       ??_R2config_plugin_base@@8 10009de4     textPlugin.obj
 0002:00002dfc       ??_R1A@?0A@EA@config_plugin_base@@8 10009dfc     textPlugin.obj
 0002:00002e18       ??_R1A@?0A@EA@QWidget@@8   10009e18     textPlugin.obj
 0002:00002e34       ??_R3QWidget@@8            10009e34     textPlugin.obj
 0002:00002e44       ??_R2QWidget@@8            10009e44     textPlugin.obj
 0002:00002e58       ??_R1CI@?0A@EA@QPaintDevice@@8 10009e58     textPlugin.obj
 0002:00002e74       ??_R3QPaintDevice@@8       10009e74     textPlugin.obj
 0002:00002e84       ??_R2QPaintDevice@@8       10009e84     textPlugin.obj
 0002:00002e8c       ??_R1A@?0A@EA@QPaintDevice@@8 10009e8c     textPlugin.obj
 0002:00002ea8       ??_R4config_plugin_base@@6BQPaintDevice@@@ 10009ea8     textPlugin.obj
 0002:00002ebc       ??_R1A@?0A@EA@QGDict@@8    10009ebc     textPlugin.obj
 0002:00002ed8       ??_R3QGDict@@8             10009ed8     textPlugin.obj
 0002:00002ee8       ??_R2QGDict@@8             10009ee8     textPlugin.obj
 0002:00002ef4       ??_R4textPlugin@@6BQObject@@@ 10009ef4     textPlugin.obj
 0002:00002f08       ??_R3textPlugin@@8         10009f08     textPlugin.obj
 0002:00002f18       ??_R2textPlugin@@8         10009f18     textPlugin.obj
 0002:00002f34       ??_R1A@?0A@EA@textPlugin@@8 10009f34     textPlugin.obj
 0002:00002f50       ??_R4textPlugin@@6BQPaintDevice@@@ 10009f50     textPlugin.obj
 0002:00002f64       ??_R4?$QDict@VQAction@@@@6B@ 10009f64     textPlugin.obj
 0002:00002f78       ??_R3?$QDict@VQAction@@@@8 10009f78     textPlugin.obj
 0002:00002f88       ??_R2?$QDict@VQAction@@@@8 10009f88     textPlugin.obj
 0002:00002f98       ??_R1A@?0A@EA@?$QDict@VQAction@@@@8 10009f98     textPlugin.obj
 0002:00002fb4       ??_R4textPluginDlg@@6BQObject@@@ 10009fb4     textPlugindlgimpl.obj
 0002:00002fc8       ??_R3textPluginDlg@@8      10009fc8     textPlugindlgimpl.obj
 0002:00002fd8       ??_R2textPluginDlg@@8      10009fd8     textPlugindlgimpl.obj
 0002:00002ff4       ??_R1A@?0A@EA@textPluginDlg@@8 10009ff4     textPlugindlgimpl.obj
 0002:00003010       ??_R1A@?0A@EA@textPluginDlgBase@@8 1000a010     textPlugindlgimpl.obj
 0002:0000302c       ??_R3textPluginDlgBase@@8  1000a02c     textPlugindlgimpl.obj
 0002:0000303c       ??_R2textPluginDlgBase@@8  1000a03c     textPlugindlgimpl.obj
 0002:00003054       ??_R4textPluginDlg@@6BQPaintDevice@@@ 1000a054     textPlugindlgimpl.obj
 0002:00003068       ??_R4xml_highlighter@@6B@  1000a068     xml_highlighter.obj
 0002:0000307c       ??_R3xml_highlighter@@8    1000a07c     xml_highlighter.obj
 0002:0000308c       ??_R2xml_highlighter@@8    1000a08c     xml_highlighter.obj
 0002:000030a0       ??_R1A@?0A@EA@xml_highlighter@@8 1000a0a0     xml_highlighter.obj
 0002:000030bc       ??_R4QVBoxLayout@@6BQObject@@@ 1000a0bc     textPlugindlg.obj
 0002:000030d0       ??_R3QVBoxLayout@@8        1000a0d0     textPlugindlg.obj
 0002:000030e0       ??_R2QVBoxLayout@@8        1000a0e0     textPlugindlg.obj
 0002:000030fc       ??_R1A@?0A@EA@QVBoxLayout@@8 1000a0fc     textPlugindlg.obj
 0002:00003118       ??_R1A@?0A@EA@QBoxLayout@@8 1000a118     textPlugindlg.obj
 0002:00003134       ??_R3QBoxLayout@@8         1000a134     textPlugindlg.obj
 0002:00003144       ??_R2QBoxLayout@@8         1000a144     textPlugindlg.obj
 0002:0000315c       ??_R1A@?0A@EA@QLayout@@8   1000a15c     textPlugindlg.obj
 0002:00003178       ??_R3QLayout@@8            1000a178     textPlugindlg.obj
 0002:00003188       ??_R2QLayout@@8            1000a188     textPlugindlg.obj
 0002:0000319c       ??_R1CI@?0A@EA@QLayoutItem@@8 1000a19c     textPlugindlg.obj
 0002:000031b8       ??_R3QLayoutItem@@8        1000a1b8     textPlugindlg.obj
 0002:000031c8       ??_R2QLayoutItem@@8        1000a1c8     textPlugindlg.obj
 0002:000031d0       ??_R1A@?0A@EA@QLayoutItem@@8 1000a1d0     textPlugindlg.obj
 0002:000031ec       ??_R4QVBoxLayout@@6BQLayoutItem@@@ 1000a1ec     textPlugindlg.obj
 0002:00003200       ??_R4QHBoxLayout@@6BQObject@@@ 1000a200     textPlugindlg.obj
 0002:00003214       ??_R3QHBoxLayout@@8        1000a214     textPlugindlg.obj
 0002:00003224       ??_R2QHBoxLayout@@8        1000a224     textPlugindlg.obj
 0002:00003240       ??_R1A@?0A@EA@QHBoxLayout@@8 1000a240     textPlugindlg.obj
 0002:0000325c       ??_R4QHBoxLayout@@6BQLayoutItem@@@ 1000a25c     textPlugindlg.obj
 0002:00003270       ??_R4QLabel@@6BQObject@@@  1000a270     textPlugindlg.obj
 0002:00003284       ??_R3QLabel@@8             1000a284     textPlugindlg.obj
 0002:00003294       ??_R2QLabel@@8             1000a294     textPlugindlg.obj
 0002:000032b0       ??_R1A@?0A@EA@QLabel@@8    1000a2b0     textPlugindlg.obj
 0002:000032cc       ??_R1A@?0A@EA@QFrame@@8    1000a2cc     textPlugindlg.obj
 0002:000032e8       ??_R3QFrame@@8             1000a2e8     textPlugindlg.obj
 0002:000032f8       ??_R2QFrame@@8             1000a2f8     textPlugindlg.obj
 0002:00003310       ??_R4QLabel@@6BQPaintDevice@@@ 1000a310     textPlugindlg.obj
 0002:00003324       ??_R4QTextEdit@@6BQObject@@@ 1000a324     textPlugindlg.obj
 0002:00003338       ??_R3QTextEdit@@8          1000a338     textPlugindlg.obj
 0002:00003348       ??_R2QTextEdit@@8          1000a348     textPlugindlg.obj
 0002:00003368       ??_R1A@?0A@EA@QTextEdit@@8 1000a368     textPlugindlg.obj
 0002:00003384       ??_R1A@?0A@EA@QScrollView@@8 1000a384     textPlugindlg.obj
 0002:000033a0       ??_R3QScrollView@@8        1000a3a0     textPlugindlg.obj
 0002:000033b0       ??_R2QScrollView@@8        1000a3b0     textPlugindlg.obj
 0002:000033cc       ??_R4QTextEdit@@6BQPaintDevice@@@ 1000a3cc     textPlugindlg.obj
 0002:000033e0       ??_R4textPluginDlgBase@@6BQObject@@@ 1000a3e0     textPlugindlg.obj
 0002:000033f4       ??_R4textPluginDlgBase@@6BQPaintDevice@@@ 1000a3f4     textPlugindlg.obj
 0002:00003408       ??_R4QSpacerItem@@6B@      1000a408     textPlugindlg.obj
 0002:0000341c       ??_R3QSpacerItem@@8        1000a41c     textPlugindlg.obj
 0002:0000342c       ??_R2QSpacerItem@@8        1000a42c     textPlugindlg.obj
 0002:00003438       ??_R1A@?0A@EA@QSpacerItem@@8 1000a438     textPlugindlg.obj
 0002:00003454       ??_R4type_info@@6B@        1000a454     MSVCRT:ti_inst.obj
 0002:00003468       ??_R3type_info@@8          1000a468     MSVCRT:ti_inst.obj
 0002:00003478       ??_R2type_info@@8          1000a478     MSVCRT:ti_inst.obj
 0002:00003480       ??_R1A@?0A@EA@type_info@@8 1000a480     MSVCRT:ti_inst.obj
 0002:0000349c       ___rtc_iaa                 1000a49c     MSVCRT:initsect.obj
 0002:000034a0       ___rtc_izz                 1000a4a0     MSVCRT:initsect.obj
 0002:000034a4       ___rtc_taa                 1000a4a4     MSVCRT:initsect.obj
 0002:000034a8       ___rtc_tzz                 1000a4a8     MSVCRT:initsect.obj
 0002:000041d0       __IMPORT_DESCRIPTOR_qt-mt323 1000b1d0     qt-mt323:qt-mt323.dll
 0002:000041e4       __IMPORT_DESCRIPTOR_MSVCR120 1000b1e4     MSVCRT:MSVCR120.dll
 0002:000041f8       __IMPORT_DESCRIPTOR_KERNEL32 1000b1f8     kernel32:KERNEL32.dll
 0002:0000420c       __NULL_IMPORT_DESCRIPTOR   1000b20c     qt-mt323:qt-mt323.dll
 0003:00000048       ___security_cookie         10011048     MSVCRT:gs_cookie.obj
 0003:0000004c       ___security_cookie_complement 1001104c     MSVCRT:gs_cookie.obj
 0003:00000050       ___native_dllmain_reason   10011050     MSVCRT:natstart.obj
 0003:00000054       ??_R0?AVconfig@@@8         10011054     config.obj
 0003:0000006c       ??_R0?AVconfig_plugin_desc_base@@@8 1001106c     plugindesc.obj
 0003:00000094       ??_R0?AVplugindesc@@@8     10011094     plugindesc.obj
 0003:000000b0       ??_R0?AVtext_highlighter@@@8 100110b0     text_highlighter.obj
 0003:000000d0       ??_R0?AVQSyntaxHighlighter@@@8 100110d0     text_highlighter.obj
 0003:000000f4       ??_R0?AVQt@@@8             100110f4     text_highlighter.obj
 0003:00000108       ??_R0?AUQShared@@@8        10011108     textPlugin.obj
 0003:00000120       ??_R0?AVQGList@@@8         10011120     textPlugin.obj
 0003:00000138       ??_R0?AVQPtrCollection@@@8 10011138     textPlugin.obj
 0003:00000158       ??_R0?AVQGuardedPtrPrivate@@@8 10011158     textPlugin.obj
 0003:0000017c       ??_R0?AVQObject@@@8        1001117c     textPlugin.obj
 0003:00000194       ??_R0?AVQDockWindowList@@@8 10011194     textPlugin.obj
 0003:000001b4       ??_R0?AV?$QPtrList@VQDockWindow@@@@@8 100111b4     textPlugin.obj
 0003:000001dc       ??_R0?AVQPopupMenuList@@@8 100111dc     textPlugin.obj
 0003:000001fc       ??_R0?AV?$QPtrList@VQPopupMenu@@@@@8 100111fc     textPlugin.obj
 0003:00000224       ??_R0?AVconfig_plugin_base@@@8 10011224     textPlugin.obj
 0003:00000248       ??_R0?AVQWidget@@@8        10011248     textPlugin.obj
 0003:00000260       ??_R0?AVQPaintDevice@@@8   10011260     textPlugin.obj
 0003:0000027c       ??_R0?AVQGDict@@@8         1001127c     textPlugin.obj
 0003:00000294       ??_R0?AVtextPlugin@@@8     10011294     textPlugin.obj
 0003:000002b0       ??_R0?AV?$QDict@VQAction@@@@@8 100112b0     textPlugin.obj
 0003:000002d4       ??_R0?AVtextPluginDlg@@@8  100112d4     textPlugindlgimpl.obj
 0003:000002f0       ??_R0?AVtextPluginDlgBase@@@8 100112f0     textPlugindlgimpl.obj
 0003:00000310       ??_R0?AVxml_highlighter@@@8 10011310     xml_highlighter.obj
 0003:00000330       ??_R0?AVQVBoxLayout@@@8    10011330     textPlugindlg.obj
 0003:0000034c       ??_R0?AVQBoxLayout@@@8     1001134c     textPlugindlg.obj
 0003:00000368       ??_R0?AVQLayout@@@8        10011368     textPlugindlg.obj
 0003:00000380       ??_R0?AVQLayoutItem@@@8    10011380     textPlugindlg.obj
 0003:0000039c       ??_R0?AVQHBoxLayout@@@8    1001139c     textPlugindlg.obj
 0003:000003b8       ??_R0?AVQLabel@@@8         100113b8     textPlugindlg.obj
 0003:000003d0       ??_R0?AVQFrame@@@8         100113d0     textPlugindlg.obj
 0003:000003e8       ??_R0?AVQTextEdit@@@8      100113e8     textPlugindlg.obj
 0003:00000400       ??_R0?AVQScrollView@@@8    10011400     textPlugindlg.obj
 0003:0000041c       ??_R0?AVQSpacerItem@@@8    1001141c     textPlugindlg.obj
 0003:00000438       ??_R0?AVtype_info@@@8      10011438     MSVCRT:ti_inst.obj
 0003:00000450       ?metaObj@textPlugin@@0PAVQMetaObject@@A 10011450     moc_textPlugin.obj
 0003:0000047c       ?metaObj@textPluginDlgBase@@0PAVQMetaObject@@A 1001147c     moc_textPlugindlg.obj
 0003:00000484       ?metaObj@textPluginDlg@@0PAVQMetaObject@@A 10011484     moc_textPlugindlgimpl.obj
 0003:000007d8       ?__type_info_root_node@@3U__type_info_node@@A 100117d8     MSVCRT:tncleanup.obj
 0003:000007e0       ___native_startup_lock     100117e0     <common>
 0003:000007e4       ___native_startup_state    100117e4     <common>
 0003:000007e8       ___dyn_tls_init_callback   100117e8     <common>
 0003:000007ec       ___onexitend               100117ec     <common>
 0003:000007f0       ___onexitbegin             100117f0     <common>

 entry point at        0001:000042de

 Static symbols

 0001:00000000       ??__EcleanUp_textPlugin@@YAXXZ 10001000 f   moc_textPlugin.obj
 0001:00000021       ??__EcleanUp_textPluginDlgBase@@YAXXZ 10001021 f   moc_textPlugindlg.obj
 0001:00000042       ??__EcleanUp_textPluginDlg@@YAXXZ 10001042 f   moc_textPlugindlgimpl.obj
 0001:0000409b       _pre_c_init                1000509b f   MSVCRT:crtdll.obj
 0001:00004301       ___DllMainCRTStartup       10005301 f   MSVCRT:crtdll.obj
 0001:00004580       $$000000                   10005580     MSVCRT:sehprolg4.obj
 0001:0000489c       __unwindfunclet$??0config@@QAE@ABVQString@@@Z$0 1000589c f   config.obj
 0001:000048a8       __unwindfunclet$??0config@@QAE@ABVQString@@@Z$1 100058a8 f   config.obj
 0001:000048b4       __unwindfunclet$??0config@@QAE@ABVQString@@@Z$2 100058b4 f   config.obj
 0001:000048c0       __unwindfunclet$??0config@@QAE@ABVQString@@@Z$3 100058c0 f   config.obj
 0001:000048cc       __unwindfunclet$??0config@@QAE@ABVQString@@@Z$4 100058cc f   config.obj
 0001:000048d8       __unwindfunclet$??0config@@QAE@ABVQString@@@Z$5 100058d8 f   config.obj
 0001:000048e1       __unwindfunclet$??0config@@QAE@ABVQString@@@Z$6 100058e1 f   config.obj
 0001:000048ea       __unwindfunclet$??0config@@QAE@ABVQString@@@Z$7 100058ea f   config.obj
 0001:000048f3       __unwindfunclet$??0config@@QAE@ABVQString@@@Z$8 100058f3 f   config.obj
 0001:000048fc       __unwindfunclet$??0config@@QAE@ABVQString@@@Z$9 100058fc f   config.obj
 0001:00004905       __unwindfunclet$??0config@@QAE@ABVQString@@@Z$10 10005905 f   config.obj
 0001:0000490e       __unwindfunclet$??0config@@QAE@ABVQString@@@Z$11 1000590e f   config.obj
 0001:00004917       __unwindfunclet$??0config@@QAE@ABVQString@@@Z$12 10005917 f   config.obj
 0001:00004920       __unwindfunclet$??0config@@QAE@ABVQString@@@Z$13 10005920 f   config.obj
 0001:00004929       __unwindfunclet$??0config@@QAE@ABVQString@@@Z$14 10005929 f   config.obj
 0001:00004932       __unwindfunclet$??0config@@QAE@ABVQString@@@Z$15 10005932 f   config.obj
 0001:0000493b       __unwindfunclet$??0config@@QAE@ABVQString@@@Z$16 1000593b f   config.obj
 0001:00004944       __unwindfunclet$??0config@@QAE@ABVQString@@@Z$17 10005944 f   config.obj
 0001:0000494d       __unwindfunclet$??0config@@QAE@ABVQString@@@Z$18 1000594d f   config.obj
 0001:00004956       __unwindfunclet$??0config@@QAE@ABVQString@@@Z$19 10005956 f   config.obj
 0001:0000495f       __unwindfunclet$??0config@@QAE@ABVQString@@@Z$20 1000595f f   config.obj
 0001:00004968       __unwindfunclet$??0config@@QAE@ABVQString@@@Z$21 10005968 f   config.obj
 0001:00004971       __unwindfunclet$??0config@@QAE@ABVQString@@@Z$22 10005971 f   config.obj
 0001:0000497a       __unwindfunclet$??0config@@QAE@ABVQString@@@Z$23 1000597a f   config.obj
 0001:00004983       __unwindfunclet$??0config@@QAE@ABVQString@@@Z$24 10005983 f   config.obj
 0001:0000498c       __unwindfunclet$??0config@@QAE@ABVQString@@@Z$25 1000598c f   config.obj
 0001:00004995       __unwindfunclet$??0config@@QAE@ABVQString@@@Z$26 10005995 f   config.obj
 0001:0000499e       __unwindfunclet$??0config@@QAE@ABVQString@@@Z$27 1000599e f   config.obj
 0001:000049a7       __unwindfunclet$??0config@@QAE@ABVQString@@@Z$28 100059a7 f   config.obj
 0001:000049b0       __unwindfunclet$??0config@@QAE@ABVQString@@@Z$29 100059b0 f   config.obj
 0001:000049b9       __unwindfunclet$??0config@@QAE@ABVQString@@@Z$30 100059b9 f   config.obj
 0001:000049c2       __unwindfunclet$??0config@@QAE@ABVQString@@@Z$31 100059c2 f   config.obj
 0001:000049cb       __unwindfunclet$??0config@@QAE@ABVQString@@@Z$32 100059cb f   config.obj
 0001:000049d4       __unwindfunclet$??0config@@QAE@ABVQString@@@Z$33 100059d4 f   config.obj
 0001:000049dd       __unwindfunclet$??0config@@QAE@ABVQString@@@Z$34 100059dd f   config.obj
 0001:000049e6       __unwindfunclet$??0config@@QAE@ABVQString@@@Z$35 100059e6 f   config.obj
 0001:000049ef       __unwindfunclet$??0config@@QAE@ABVQString@@@Z$36 100059ef f   config.obj
 0001:000049f8       __unwindfunclet$??0config@@QAE@ABVQString@@@Z$37 100059f8 f   config.obj
 0001:00004a01       __unwindfunclet$??0config@@QAE@ABVQString@@@Z$38 10005a01 f   config.obj
 0001:00004a0a       __unwindfunclet$??0config@@QAE@ABVQString@@@Z$39 10005a0a f   config.obj
 0001:00004a13       __unwindfunclet$??0config@@QAE@ABVQString@@@Z$40 10005a13 f   config.obj
 0001:00004a1c       __unwindfunclet$??0config@@QAE@ABVQString@@@Z$41 10005a1c f   config.obj
 0001:00004a25       __unwindfunclet$??0config@@QAE@ABVQString@@@Z$42 10005a25 f   config.obj
 0001:00004a2e       __unwindfunclet$??0config@@QAE@ABVQString@@@Z$43 10005a2e f   config.obj
 0001:00004a37       __unwindfunclet$??0config@@QAE@ABVQString@@@Z$44 10005a37 f   config.obj
 0001:00004a40       __unwindfunclet$??0config@@QAE@ABVQString@@@Z$45 10005a40 f   config.obj
 0001:00004a49       __unwindfunclet$??0config@@QAE@ABVQString@@@Z$46 10005a49 f   config.obj
 0001:00004a52       __unwindfunclet$??0config@@QAE@ABVQString@@@Z$47 10005a52 f   config.obj
 0001:00004a5b       __unwindfunclet$??0config@@QAE@ABVQString@@@Z$48 10005a5b f   config.obj
 0001:00004a64       __unwindfunclet$??0config@@QAE@ABVQString@@@Z$49 10005a64 f   config.obj
 0001:00004a6d       __unwindfunclet$??0config@@QAE@ABVQString@@@Z$50 10005a6d f   config.obj
 0001:00004a76       __unwindfunclet$??0config@@QAE@ABVQString@@@Z$51 10005a76 f   config.obj
 0001:00004a7f       __unwindfunclet$??0config@@QAE@ABVQString@@@Z$52 10005a7f f   config.obj
 0001:00004a88       __unwindfunclet$??0config@@QAE@ABVQString@@@Z$53 10005a88 f   config.obj
 0001:00004a91       __unwindfunclet$??0config@@QAE@ABVQString@@@Z$54 10005a91 f   config.obj
 0001:00004a9a       __unwindfunclet$??0config@@QAE@ABVQString@@@Z$55 10005a9a f   config.obj
 0001:00004aa3       __unwindfunclet$??0config@@QAE@ABVQString@@@Z$56 10005aa3 f   config.obj
 0001:00004aac       __ehhandler$??0config@@QAE@ABVQString@@@Z 10005aac f   config.obj
 0001:00004ac7       __unwindfunclet$??1config@@UAE@XZ$0 10005ac7 f   config.obj
 0001:00004ad3       __unwindfunclet$??1config@@UAE@XZ$1 10005ad3 f   config.obj
 0001:00004adf       __unwindfunclet$??1config@@UAE@XZ$2 10005adf f   config.obj
 0001:00004aeb       __unwindfunclet$??1config@@UAE@XZ$3 10005aeb f   config.obj
 0001:00004af7       __ehhandler$??1config@@UAE@XZ 10005af7 f   config.obj
 0001:00004b12       __unwindfunclet$?getDescFromKey@config@@QAE?AVQString@@ABV2@@Z$0 10005b12 f   config.obj
 0001:00004b12       __unwindfunclet$?getFilenameFromKey@config@@QAE?AVQString@@ABV2@@Z$0 10005b12 f   config.obj
 0001:00004b12       __unwindfunclet$?getHelpFromKey@config@@QAE?AVQString@@ABV2@@Z$0 10005b12 f   config.obj
 0001:00004b1b       __ehhandler$?getFilenameFromKey@config@@QAE?AVQString@@ABV2@@Z 10005b1b f   config.obj
 0001:00004b1b       __ehhandler$?getHelpFromKey@config@@QAE?AVQString@@ABV2@@Z 10005b1b f   config.obj
 0001:00004b1b       __ehhandler$?getDescFromKey@config@@QAE?AVQString@@ABV2@@Z 10005b1b f   config.obj
 0001:00004b36       __unwindfunclet$?getKeys@config@@QAE?AVQStringList@@XZ$0 10005b36 f   config.obj
 0001:00004b3f       __unwindfunclet$?getKeys@config@@QAE?AVQStringList@@XZ$1 10005b3f f   config.obj
 0001:00004b48       __unwindfunclet$?getKeys@config@@QAE?AVQStringList@@XZ$2 10005b48 f   config.obj
 0001:00004b51       __unwindfunclet$?getKeys@config@@QAE?AVQStringList@@XZ$3 10005b51 f   config.obj
 0001:00004b5a       __unwindfunclet$?getKeys@config@@QAE?AVQStringList@@XZ$4 10005b5a f   config.obj
 0001:00004b74       __unwindfunclet$?getKeys@config@@QAE?AVQStringList@@XZ$5 10005b74 f   config.obj
 0001:00004b7d       __unwindfunclet$?getKeys@config@@QAE?AVQStringList@@XZ$6 10005b7d f   config.obj
 0001:00004b86       __unwindfunclet$?getKeys@config@@QAE?AVQStringList@@XZ$7 10005b86 f   config.obj
 0001:00004b8f       __unwindfunclet$?getKeys@config@@QAE?AVQStringList@@XZ$8 10005b8f f   config.obj
 0001:00004b98       __unwindfunclet$?getKeys@config@@QAE?AVQStringList@@XZ$9 10005b98 f   config.obj
 0001:00004ba1       __unwindfunclet$?getKeys@config@@QAE?AVQStringList@@XZ$10 10005ba1 f   config.obj
 0001:00004baa       __ehhandler$?getKeys@config@@QAE?AVQStringList@@XZ 10005baa f   config.obj
 0001:00004bc5       __unwindfunclet$?getNamedAttribute@config@@AAE?AVQString@@ABV2@0@Z$0 10005bc5 f   config.obj
 0001:00004bce       __unwindfunclet$?getNamedAttribute@config@@AAE?AVQString@@ABV2@0@Z$1 10005bce f   config.obj
 0001:00004bd7       __unwindfunclet$?getNamedAttribute@config@@AAE?AVQString@@ABV2@0@Z$2 10005bd7 f   config.obj
 0001:00004be0       __unwindfunclet$?getNamedAttribute@config@@AAE?AVQString@@ABV2@0@Z$3 10005be0 f   config.obj
 0001:00004bfa       __unwindfunclet$?getNamedAttribute@config@@AAE?AVQString@@ABV2@0@Z$4 10005bfa f   config.obj
 0001:00004c03       __unwindfunclet$?getNamedAttribute@config@@AAE?AVQString@@ABV2@0@Z$5 10005c03 f   config.obj
 0001:00004c0c       __unwindfunclet$?getNamedAttribute@config@@AAE?AVQString@@ABV2@0@Z$6 10005c0c f   config.obj
 0001:00004c15       __unwindfunclet$?getNamedAttribute@config@@AAE?AVQString@@ABV2@0@Z$7 10005c15 f   config.obj
 0001:00004c1e       __unwindfunclet$?getNamedAttribute@config@@AAE?AVQString@@ABV2@0@Z$8 10005c1e f   config.obj
 0001:00004c27       __unwindfunclet$?getNamedAttribute@config@@AAE?AVQString@@ABV2@0@Z$9 10005c27 f   config.obj
 0001:00004c30       __ehhandler$?getNamedAttribute@config@@AAE?AVQString@@ABV2@0@Z 10005c30 f   config.obj
 0001:00004c4b       __unwindfunclet$?keys@plugindesc@@UAE?AVQStringList@@ABVQString@@0@Z$0 10005c4b f   plugindesc.obj
 0001:00004c53       __unwindfunclet$?keys@plugindesc@@UAE?AVQStringList@@ABVQString@@0@Z$1 10005c53 f   plugindesc.obj
 0001:00004c6d       __ehhandler$?keys@plugindesc@@UAE?AVQStringList@@ABVQString@@0@Z 10005c6d f   plugindesc.obj
 0001:00004c88       __unwindfunclet$??1text_highlighter@@UAE@XZ$0 10005c88 f   text_highlighter.obj
 0001:00004c88       __unwindfunclet$??0text_highlighter@@QAE@PAVQTextEdit@@@Z$0 10005c88 f   text_highlighter.obj
 0001:00004c91       __unwindfunclet$??0text_highlighter@@QAE@PAVQTextEdit@@@Z$1 10005c91 f   text_highlighter.obj
 0001:00004c91       __unwindfunclet$??1text_highlighter@@UAE@XZ$1 10005c91 f   text_highlighter.obj
 0001:00004c9d       __unwindfunclet$??0text_highlighter@@QAE@PAVQTextEdit@@@Z$2 10005c9d f   text_highlighter.obj
 0001:00004c9d       __unwindfunclet$??1text_highlighter@@UAE@XZ$2 10005c9d f   text_highlighter.obj
 0001:00004ca9       __ehhandler$??1text_highlighter@@UAE@XZ 10005ca9 f   text_highlighter.obj
 0001:00004ca9       __ehhandler$??0text_highlighter@@QAE@PAVQTextEdit@@@Z 10005ca9 f   text_highlighter.obj
 0001:00004cc4       __unwindfunclet$?highlightParagraph@text_highlighter@@UAEHABVQString@@H@Z$0 10005cc4 f   text_highlighter.obj
 0001:00004ccd       __unwindfunclet$?highlightParagraph@text_highlighter@@UAEHABVQString@@H@Z$1 10005ccd f   text_highlighter.obj
 0001:00004ce7       __unwindfunclet$?highlightParagraph@text_highlighter@@UAEHABVQString@@H@Z$2 10005ce7 f   text_highlighter.obj
 0001:00004d01       __unwindfunclet$?highlightParagraph@text_highlighter@@UAEHABVQString@@H@Z$3 10005d01 f   text_highlighter.obj
 0001:00004d0a       __unwindfunclet$?highlightParagraph@text_highlighter@@UAEHABVQString@@H@Z$4 10005d0a f   text_highlighter.obj
 0001:00004d13       __unwindfunclet$?highlightParagraph@text_highlighter@@UAEHABVQString@@H@Z$5 10005d13 f   text_highlighter.obj
 0001:00004d1c       __unwindfunclet$?highlightParagraph@text_highlighter@@UAEHABVQString@@H@Z$6 10005d1c f   text_highlighter.obj
 0001:00004d25       __unwindfunclet$?highlightParagraph@text_highlighter@@UAEHABVQString@@H@Z$8 10005d25 f   text_highlighter.obj
 0001:00004d2e       __unwindfunclet$?highlightParagraph@text_highlighter@@UAEHABVQString@@H@Z$9 10005d2e f   text_highlighter.obj
 0001:00004d37       __ehhandler$?highlightParagraph@text_highlighter@@UAEHABVQString@@H@Z 10005d37 f   text_highlighter.obj
 0001:00004d52       __unwindfunclet$??0?$QGuardedPtr@VQPopupMenu@@@@QAE@XZ$0 10005d52 f   textPlugin.obj
 0001:00004d52       __unwindfunclet$??0?$QGuardedPtr@VQDockWindow@@@@QAE@XZ$0 10005d52 f   textPlugin.obj
 0001:00004d52       __unwindfunclet$?create@plugindesc@@UAEPAVconfig_plugin_base@@ABVQString@@00@Z$0 10005d52 f   textPlugin.obj
 0001:00004d5c       __ehhandler$??0?$QGuardedPtr@VQDockWindow@@@@QAE@XZ 10005d5c f   textPlugin.obj
 0001:00004d5c       __ehhandler$?create@plugindesc@@UAEPAVconfig_plugin_base@@ABVQString@@00@Z 10005d5c f   textPlugin.obj
 0001:00004d5c       __ehhandler$??0?$QGuardedPtr@VQPopupMenu@@@@QAE@XZ 10005d5c f   textPlugin.obj
 0001:00004d77       __unwindfunclet$??0config_plugin_base@@QAE@ABVQString@@00@Z$0 10005d77 f   textPlugin.obj
 0001:00004d80       __unwindfunclet$??0config_plugin_base@@QAE@ABVQString@@00@Z$1 10005d80 f   textPlugin.obj
 0001:00004d8c       __unwindfunclet$??0config_plugin_base@@QAE@ABVQString@@00@Z$2 10005d8c f   textPlugin.obj
 0001:00004d98       __unwindfunclet$??0config_plugin_base@@QAE@ABVQString@@00@Z$3 10005d98 f   textPlugin.obj
 0001:00004da4       __ehhandler$??0config_plugin_base@@QAE@ABVQString@@00@Z 10005da4 f   textPlugin.obj
 0001:00004dbf       __unwindfunclet$??0textPlugin@@QAE@ABVQString@@00@Z$0 10005dbf f   textPlugin.obj
 0001:00004dc7       __unwindfunclet$??0textPlugin@@QAE@ABVQString@@00@Z$1 10005dc7 f   textPlugin.obj
 0001:00004dd2       __unwindfunclet$??0textPlugin@@QAE@ABVQString@@00@Z$2 10005dd2 f   textPlugin.obj
 0001:00004ddd       __unwindfunclet$??0textPlugin@@QAE@ABVQString@@00@Z$3 10005ddd f   textPlugin.obj
 0001:00004deb       __unwindfunclet$??0textPlugin@@QAE@ABVQString@@00@Z$4 10005deb f   textPlugin.obj
 0001:00004df9       __unwindfunclet$??0textPlugin@@QAE@ABVQString@@00@Z$5 10005df9 f   textPlugin.obj
 0001:00004e08       __unwindfunclet$??0textPlugin@@QAE@ABVQString@@00@Z$6 10005e08 f   textPlugin.obj
 0001:00004e12       __unwindfunclet$??0textPlugin@@QAE@ABVQString@@00@Z$7 10005e12 f   textPlugin.obj
 0001:00004e1a       __unwindfunclet$??0textPlugin@@QAE@ABVQString@@00@Z$8 10005e1a f   textPlugin.obj
 0001:00004e23       __unwindfunclet$??0textPlugin@@QAE@ABVQString@@00@Z$9 10005e23 f   textPlugin.obj
 0001:00004e2c       __unwindfunclet$??0textPlugin@@QAE@ABVQString@@00@Z$10 10005e2c f   textPlugin.obj
 0001:00004e35       __unwindfunclet$??0textPlugin@@QAE@ABVQString@@00@Z$11 10005e35 f   textPlugin.obj
 0001:00004e3e       __unwindfunclet$??0textPlugin@@QAE@ABVQString@@00@Z$12 10005e3e f   textPlugin.obj
 0001:00004e47       __unwindfunclet$??0textPlugin@@QAE@ABVQString@@00@Z$13 10005e47 f   textPlugin.obj
 0001:00004e51       __ehhandler$??0textPlugin@@QAE@ABVQString@@00@Z 10005e51 f   textPlugin.obj
 0001:00004e6c       __unwindfunclet$??1?$QDict@VQAction@@@@UAE@XZ$0 10005e6c f   textPlugin.obj
 0001:00004e75       __ehhandler$??1?$QDict@VQAction@@@@UAE@XZ 10005e75 f   textPlugin.obj
 0001:00004e90       __unwindfunclet$??1?$QPtrList@VQPopupMenu@@@@UAE@XZ$0 10005e90 f   textPlugin.obj
 0001:00004e99       __ehhandler$??1?$QPtrList@VQPopupMenu@@@@UAE@XZ 10005e99 f   textPlugin.obj
 0001:00004eb4       __unwindfunclet$??1QDockWindowList@@UAE@XZ$0 10005eb4 f   textPlugin.obj
 0001:00004ebd       __unwindfunclet$??1QDockWindowList@@UAE@XZ$1 10005ebd f   textPlugin.obj
 0001:00004ec6       __ehhandler$??1QDockWindowList@@UAE@XZ 10005ec6 f   textPlugin.obj
 0001:00004ee1       __unwindfunclet$??1QPopupMenuList@@UAE@XZ$0 10005ee1 f   textPlugin.obj
 0001:00004ee9       __ehhandler$??1QPopupMenuList@@UAE@XZ 10005ee9 f   textPlugin.obj
 0001:00004f04       __unwindfunclet$??1config_plugin_base@@UAE@XZ$0 10005f04 f   textPlugin.obj
 0001:00004f0d       __unwindfunclet$??1config_plugin_base@@UAE@XZ$1 10005f0d f   textPlugin.obj
 0001:00004f19       __unwindfunclet$??1config_plugin_base@@UAE@XZ$2 10005f19 f   textPlugin.obj
 0001:00004f25       __ehhandler$??1config_plugin_base@@UAE@XZ 10005f25 f   textPlugin.obj
 0001:00004f40       __unwindfunclet$??1textPlugin@@UAE@XZ$0 10005f40 f   textPlugin.obj
 0001:00004f48       __unwindfunclet$??1textPlugin@@UAE@XZ$1 10005f48 f   textPlugin.obj
 0001:00004f53       __unwindfunclet$??1textPlugin@@UAE@XZ$2 10005f53 f   textPlugin.obj
 0001:00004f5e       __unwindfunclet$??1textPlugin@@UAE@XZ$3 10005f5e f   textPlugin.obj
 0001:00004f6c       __unwindfunclet$??1textPlugin@@UAE@XZ$4 10005f6c f   textPlugin.obj
 0001:00004f7a       __unwindfunclet$??1textPlugin@@UAE@XZ$5 10005f7a f   textPlugin.obj
 0001:00004f89       __ehhandler$??1textPlugin@@UAE@XZ 10005f89 f   textPlugin.obj
 0001:00004fa4       __unwindfunclet$?about@config_plugin_base@@UAE?AVQString@@XZ$0 10005fa4 f   textPlugin.obj
 0001:00004fad       __unwindfunclet$?about@config_plugin_base@@UAE?AVQString@@XZ$1 10005fad f   textPlugin.obj
 0001:00004fc7       __ehhandler$?about@config_plugin_base@@UAE?AVQString@@XZ 10005fc7 f   textPlugin.obj
 0001:00004fe2       __unwindfunclet$?about@textPlugin@@UAE?AVQString@@XZ$0 10005fe2 f   textPlugin.obj
 0001:00004feb       __unwindfunclet$?about@textPlugin@@UAE?AVQString@@XZ$1 10005feb f   textPlugin.obj
 0001:00004ff4       __unwindfunclet$?about@textPlugin@@UAE?AVQString@@XZ$2 10005ff4 f   textPlugin.obj
 0001:00004ffd       __unwindfunclet$?about@textPlugin@@UAE?AVQString@@XZ$3 10005ffd f   textPlugin.obj
 0001:00005006       __unwindfunclet$?about@textPlugin@@UAE?AVQString@@XZ$4 10006006 f   textPlugin.obj
 0001:00005020       __ehhandler$?about@textPlugin@@UAE?AVQString@@XZ 10006020 f   textPlugin.obj
 0001:0000503b       __unwindfunclet$?activate@textPlugin@@UAEX_N@Z$0 1000603b f   textPlugin.obj
 0001:00005044       __unwindfunclet$?activate@textPlugin@@UAEX_N@Z$2 10006044 f   textPlugin.obj
 0001:0000504d       __unwindfunclet$?activate@textPlugin@@UAEX_N@Z$3 1000604d f   textPlugin.obj
 0001:00005056       __unwindfunclet$?activate@textPlugin@@UAEX_N@Z$4 10006056 f   textPlugin.obj
 0001:0000505f       __unwindfunclet$?activate@textPlugin@@UAEX_N@Z$5 1000605f f   textPlugin.obj
 0001:00005068       __unwindfunclet$?activate@textPlugin@@UAEX_N@Z$6 10006068 f   textPlugin.obj
 0001:00005071       __unwindfunclet$?activate@textPlugin@@UAEX_N@Z$7 10006071 f   textPlugin.obj
 0001:0000507a       __unwindfunclet$?activate@textPlugin@@UAEX_N@Z$8 1000607a f   textPlugin.obj
 0001:00005083       __unwindfunclet$?activate@textPlugin@@UAEX_N@Z$9 10006083 f   textPlugin.obj
 0001:0000508c       __unwindfunclet$?activate@textPlugin@@UAEX_N@Z$10 1000608c f   textPlugin.obj
 0001:00005095       __unwindfunclet$?activate@textPlugin@@UAEX_N@Z$11 10006095 f   textPlugin.obj
 0001:0000509e       __ehhandler$?activate@textPlugin@@UAEX_N@Z 1000609e f   textPlugin.obj
 0001:000050b9       __unwindfunclet$?apply@textPlugin@@UAEXXZ$0 100060b9 f   textPlugin.obj
 0001:000050c2       __unwindfunclet$?apply@textPlugin@@UAEXXZ$1 100060c2 f   textPlugin.obj
 0001:000050cb       __unwindfunclet$?apply@textPlugin@@UAEXXZ$2 100060cb f   textPlugin.obj
 0001:000050d4       __unwindfunclet$?apply@textPlugin@@UAEXXZ$3 100060d4 f   textPlugin.obj
 0001:000050dd       __unwindfunclet$?apply@textPlugin@@UAEXXZ$4 100060dd f   textPlugin.obj
 0001:000050e6       __unwindfunclet$?apply@textPlugin@@UAEXXZ$5 100060e6 f   textPlugin.obj
 0001:000050ef       __unwindfunclet$?apply@textPlugin@@UAEXXZ$6 100060ef f   textPlugin.obj
 0001:000050f8       __unwindfunclet$?apply@textPlugin@@UAEXXZ$7 100060f8 f   textPlugin.obj
 0001:00005101       __unwindfunclet$?apply@textPlugin@@UAEXXZ$8 10006101 f   textPlugin.obj
 0001:0000510a       __unwindfunclet$?apply@textPlugin@@UAEXXZ$9 1000610a f   textPlugin.obj
 0001:00005113       __unwindfunclet$?apply@textPlugin@@UAEXXZ$10 10006113 f   textPlugin.obj
 0001:0000511c       __unwindfunclet$?apply@textPlugin@@UAEXXZ$11 1000611c f   textPlugin.obj
 0001:00005125       __unwindfunclet$?apply@textPlugin@@UAEXXZ$12 10006125 f   textPlugin.obj
 0001:0000512e       __unwindfunclet$?apply@textPlugin@@UAEXXZ$13 1000612e f   textPlugin.obj
 0001:00005137       __unwindfunclet$?apply@textPlugin@@UAEXXZ$14 10006137 f   textPlugin.obj
 0001:00005140       __unwindfunclet$?apply@textPlugin@@UAEXXZ$16 10006140 f   textPlugin.obj
 0001:00005149       __ehhandler$?apply@textPlugin@@UAEXXZ 10006149 f   textPlugin.obj
 0001:00005164       __unwindfunclet$?textChanged@textPluginDlg@@QAEXXZ$0 10006164 f   textPlugin.obj
 0001:00005164       __unwindfunclet$?closeEvent@textPlugin@@UAEXPAVQCloseEvent@@@Z$0 10006164 f   textPlugin.obj
 0001:0000516d       __ehhandler$?closeEvent@textPlugin@@UAEXPAVQCloseEvent@@@Z 1000616d f   textPlugin.obj
 0001:0000516d       __ehhandler$?textChanged@textPluginDlg@@QAEXXZ 1000616d f   textPlugin.obj
 0001:00005188       __unwindfunclet$?db@@YAXABVQString@@@Z$0 10006188 f   textPlugin.obj
 0001:00005191       __ehhandler$?db@@YAXABVQString@@@Z 10006191 f   textPlugin.obj
 0001:000051ac       __unwindfunclet$?menus@textPlugin@@UAE?AVQPopupMenuList@@XZ$0 100061ac f   textPlugin.obj
 0001:000051c5       __ehhandler$?menus@textPlugin@@UAE?AVQPopupMenuList@@XZ 100061c5 f   textPlugin.obj
 0001:000051e0       __unwindfunclet$?navigate@textPlugin@@UAEXABVQString@@0@Z$0 100061e0 f   textPlugin.obj
 0001:000051e9       __unwindfunclet$?navigate@textPlugin@@UAEXABVQString@@0@Z$1 100061e9 f   textPlugin.obj
 0001:000051f2       __unwindfunclet$?navigate@textPlugin@@UAEXABVQString@@0@Z$2 100061f2 f   textPlugin.obj
 0001:000051fb       __ehhandler$?navigate@textPlugin@@UAEXABVQString@@0@Z 100061fb f   textPlugin.obj
 0001:00005216       __unwindfunclet$?reply@textPlugin@@UAEXPAVresponse@@@Z$0 10006216 f   textPlugin.obj
 0001:0000521f       __unwindfunclet$?reply@textPlugin@@UAEXPAVresponse@@@Z$1 1000621f f   textPlugin.obj
 0001:00005228       __unwindfunclet$?reply@textPlugin@@UAEXPAVresponse@@@Z$2 10006228 f   textPlugin.obj
 0001:00005231       __unwindfunclet$?reply@textPlugin@@UAEXPAVresponse@@@Z$3 10006231 f   textPlugin.obj
 0001:0000523a       __unwindfunclet$?reply@textPlugin@@UAEXPAVresponse@@@Z$4 1000623a f   textPlugin.obj
 0001:00005243       __unwindfunclet$?reply@textPlugin@@UAEXPAVresponse@@@Z$5 10006243 f   textPlugin.obj
 0001:0000524c       __unwindfunclet$?reply@textPlugin@@UAEXPAVresponse@@@Z$6 1000624c f   textPlugin.obj
 0001:00005255       __unwindfunclet$?reply@textPlugin@@UAEXPAVresponse@@@Z$7 10006255 f   textPlugin.obj
 0001:0000525e       __unwindfunclet$?reply@textPlugin@@UAEXPAVresponse@@@Z$8 1000625e f   textPlugin.obj
 0001:00005267       __unwindfunclet$?reply@textPlugin@@UAEXPAVresponse@@@Z$9 10006267 f   textPlugin.obj
 0001:00005270       __unwindfunclet$?reply@textPlugin@@UAEXPAVresponse@@@Z$10 10006270 f   textPlugin.obj
 0001:00005279       __unwindfunclet$?reply@textPlugin@@UAEXPAVresponse@@@Z$11 10006279 f   textPlugin.obj
 0001:00005282       __unwindfunclet$?reply@textPlugin@@UAEXPAVresponse@@@Z$12 10006282 f   textPlugin.obj
 0001:0000528b       __unwindfunclet$?reply@textPlugin@@UAEXPAVresponse@@@Z$13 1000628b f   textPlugin.obj
 0001:00005294       __unwindfunclet$?reply@textPlugin@@UAEXPAVresponse@@@Z$14 10006294 f   textPlugin.obj
 0001:0000529d       __unwindfunclet$?reply@textPlugin@@UAEXPAVresponse@@@Z$16 1000629d f   textPlugin.obj
 0001:000052a6       __unwindfunclet$?reply@textPlugin@@UAEXPAVresponse@@@Z$17 100062a6 f   textPlugin.obj
 0001:000052af       __unwindfunclet$?reply@textPlugin@@UAEXPAVresponse@@@Z$18 100062af f   textPlugin.obj
 0001:000052b8       __unwindfunclet$?reply@textPlugin@@UAEXPAVresponse@@@Z$20 100062b8 f   textPlugin.obj
 0001:000052c1       __ehhandler$?reply@textPlugin@@UAEXPAVresponse@@@Z 100062c1 f   textPlugin.obj
 0001:000052dc       __unwindfunclet$?toolbars@textPlugin@@UAE?AVQDockWindowList@@XZ$0 100062dc f   textPlugin.obj
 0001:000052f5       __ehhandler$?toolbars@textPlugin@@UAE?AVQDockWindowList@@XZ 100062f5 f   textPlugin.obj
 0001:00005310       __unwindfunclet$??0textPluginDlg@@QAE@ABVQString@@PAVQWidget@@PBDI@Z$0 10006310 f   textPlugindlgimpl.obj
 0001:00005318       __unwindfunclet$??0textPluginDlg@@QAE@ABVQString@@PAVQWidget@@PBDI@Z$1 10006318 f   textPlugindlgimpl.obj
 0001:00005327       __unwindfunclet$??0textPluginDlg@@QAE@ABVQString@@PAVQWidget@@PBDI@Z$2 10006327 f   textPlugindlgimpl.obj
 0001:00005336       __ehhandler$??0textPluginDlg@@QAE@ABVQString@@PAVQWidget@@PBDI@Z 10006336 f   textPlugindlgimpl.obj
 0001:00005351       __unwindfunclet$??1textPluginDlg@@UAE@XZ$0 10006351 f   textPlugindlgimpl.obj
 0001:00005359       __unwindfunclet$??1textPluginDlg@@UAE@XZ$1 10006359 f   textPlugindlgimpl.obj
 0001:00005368       __ehhandler$??1textPluginDlg@@UAE@XZ 10006368 f   textPlugindlgimpl.obj
 0001:00005383       __unwindfunclet$?load@textPluginDlg@@QAE_NABVQString@@@Z$0 10006383 f   textPlugindlgimpl.obj
 0001:00005383       __unwindfunclet$?save@textPluginDlg@@QAEXABVQString@@@Z$0 10006383 f   textPlugindlgimpl.obj
 0001:0000538c       __unwindfunclet$?save@textPluginDlg@@QAEXABVQString@@@Z$1 1000638c f   textPlugindlgimpl.obj
 0001:0000538c       __unwindfunclet$?load@textPluginDlg@@QAE_NABVQString@@@Z$1 1000638c f   textPlugindlgimpl.obj
 0001:00005395       __unwindfunclet$?load@textPluginDlg@@QAE_NABVQString@@@Z$2 10006395 f   textPlugindlgimpl.obj
 0001:00005395       __unwindfunclet$?save@textPluginDlg@@QAEXABVQString@@@Z$2 10006395 f   textPlugindlgimpl.obj
 0001:0000539e       __ehhandler$?save@textPluginDlg@@QAEXABVQString@@@Z 1000639e f   textPlugindlgimpl.obj
 0001:0000539e       __ehhandler$?load@textPluginDlg@@QAE_NABVQString@@@Z 1000639e f   textPlugindlgimpl.obj
 0001:000053b9       __unwindfunclet$??0xml_highlighter@@QAE@PAVQTextEdit@@@Z$0 100063b9 f   xml_highlighter.obj
 0001:000053c1       __unwindfunclet$??0xml_highlighter@@QAE@PAVQTextEdit@@@Z$1 100063c1 f   xml_highlighter.obj
 0001:000053ca       __unwindfunclet$??0xml_highlighter@@QAE@PAVQTextEdit@@@Z$2 100063ca f   xml_highlighter.obj
 0001:000053d3       __unwindfunclet$??0xml_highlighter@@QAE@PAVQTextEdit@@@Z$3 100063d3 f   xml_highlighter.obj
 0001:000053dc       __ehhandler$??0xml_highlighter@@QAE@PAVQTextEdit@@@Z 100063dc f   xml_highlighter.obj
 0001:000053f7       __unwindfunclet$??1xml_highlighter@@UAE@XZ$0 100063f7 f   xml_highlighter.obj
 0001:000053ff       __ehhandler$??1xml_highlighter@@UAE@XZ 100063ff f   xml_highlighter.obj
 0001:0000541a       __unwindfunclet$?qt_emit@textPluginDlg@@UAE_NHPAUQUObject@@@Z$0 1000641a f   moc_textPlugin.obj
 0001:0000541a       __unwindfunclet$?qt_emit@textPlugin@@UAE_NHPAUQUObject@@@Z$0 1000641a f   moc_textPlugin.obj
 0001:00005423       __ehhandler$?qt_emit@textPlugin@@UAE_NHPAUQUObject@@@Z 10006423 f   moc_textPlugin.obj
 0001:00005423       __ehhandler$?qt_emit@textPluginDlg@@UAE_NHPAUQUObject@@@Z 10006423 f   moc_textPlugin.obj
 0001:0000543e       __unwindfunclet$?command@textPlugin@@IAEXVQString@@0@Z$0 1000643e f   moc_textPlugindlgimpl.obj
 0001:0000543e       __unwindfunclet$?command@textPluginDlg@@IAEXVQString@@0@Z$0 1000643e f   moc_textPlugindlgimpl.obj
 0001:00005447       __unwindfunclet$?command@textPlugin@@IAEXVQString@@0@Z$1 10006447 f   moc_textPlugindlgimpl.obj
 0001:00005447       __unwindfunclet$?command@textPluginDlg@@IAEXVQString@@0@Z$1 10006447 f   moc_textPlugindlgimpl.obj
 0001:00005450       __unwindfunclet$?command@textPluginDlg@@IAEXVQString@@0@Z$2 10006450 f   moc_textPlugindlgimpl.obj
 0001:00005450       __unwindfunclet$?command@textPlugin@@IAEXVQString@@0@Z$2 10006450 f   moc_textPlugindlgimpl.obj
 0001:00005464       __ehhandler$?command@textPluginDlg@@IAEXVQString@@0@Z 10006464 f   moc_textPlugindlgimpl.obj
 0001:00005464       __ehhandler$?command@textPlugin@@IAEXVQString@@0@Z 10006464 f   moc_textPlugindlgimpl.obj
 0001:00005489       __unwindfunclet$??0textPluginDlgBase@@QAE@PAVQWidget@@PBDI@Z$0 10006489 f   textPlugindlg.obj
 0001:00005492       __unwindfunclet$??0textPluginDlgBase@@QAE@PAVQWidget@@PBDI@Z$1 10006492 f   textPlugindlg.obj
 0001:0000549c       __unwindfunclet$??0textPluginDlgBase@@QAE@PAVQWidget@@PBDI@Z$2 1000649c f   textPlugindlg.obj
 0001:000054a6       __unwindfunclet$??0textPluginDlgBase@@QAE@PAVQWidget@@PBDI@Z$3 100064a6 f   textPlugindlg.obj
 0001:000054b0       __unwindfunclet$??0textPluginDlgBase@@QAE@PAVQWidget@@PBDI@Z$4 100064b0 f   textPlugindlg.obj
 0001:000054ba       __unwindfunclet$??0textPluginDlgBase@@QAE@PAVQWidget@@PBDI@Z$5 100064ba f   textPlugindlg.obj
 0001:000054c4       __unwindfunclet$??0textPluginDlgBase@@QAE@PAVQWidget@@PBDI@Z$6 100064c4 f   textPlugindlg.obj
 0001:000054ce       __unwindfunclet$??0textPluginDlgBase@@QAE@PAVQWidget@@PBDI@Z$7 100064ce f   textPlugindlg.obj
 0001:000054d8       __ehhandler$??0textPluginDlgBase@@QAE@PAVQWidget@@PBDI@Z 100064d8 f   textPlugindlg.obj
 0001:000054f3       __unwindfunclet$?languageChange@textPluginDlgBase@@MAEXXZ$0 100064f3 f   textPlugindlg.obj
 0001:000054fc       __unwindfunclet$?languageChange@textPluginDlgBase@@MAEXXZ$1 100064fc f   textPlugindlg.obj
 0001:00005505       __ehhandler$?languageChange@textPluginDlgBase@@MAEXXZ 10006505 f   textPlugindlg.obj
 0001:00005520       ??__FcleanUp_textPlugin@@YAXXZ 10006520 f   moc_textPlugin.obj
 0001:0000552b       ??__FcleanUp_textPluginDlgBase@@YAXXZ 1000652b f   moc_textPlugindlg.obj
 0001:00005536       ??__FcleanUp_textPluginDlg@@YAXXZ 10006536 f   moc_textPlugindlgimpl.obj
 0002:000007d8       _cleanUp_textPlugin$initializer$ 100077d8     moc_textPlugin.obj
 0002:000007dc       _cleanUp_textPluginDlgBase$initializer$ 100077dc     moc_textPlugindlg.obj
 0002:000007e0       _cleanUp_textPluginDlg$initializer$ 100077e0     moc_textPlugindlgimpl.obj
 0002:000007ec       _pcinit                    100077ec     MSVCRT:crtdll.obj
 0002:000007f0       _pinit                     100077f0     MSVCRT:atonexit.obj
 0002:00001ea4       ?signal_0@?3??staticMetaObject@textPlugin@@SAPAVQMetaObject@@XZ@4UQUMethod@@B 10008ea4     moc_textPlugin.obj
 0002:00001eb8       ?signal_tbl@?3??staticMetaObject@textPlugin@@SAPAVQMetaObject@@XZ@4QBUQMetaData@@B 10008eb8     moc_textPlugin.obj
 0002:00001ef4       ?slot_0@?3??staticMetaObject@textPluginDlgBase@@SAPAVQMetaObject@@XZ@4UQUMethod@@B 10008ef4     moc_textPlugindlg.obj
 0002:00001f10       ?slot_tbl@?3??staticMetaObject@textPluginDlgBase@@SAPAVQMetaObject@@XZ@4QBUQMetaData@@B 10008f10     moc_textPlugindlg.obj
 0002:00001f40       ?slot_0@?3??staticMetaObject@textPluginDlg@@SAPAVQMetaObject@@XZ@4UQUMethod@@B 10008f40     moc_textPlugindlgimpl.obj
 0002:00001f58       ?slot_tbl@?3??staticMetaObject@textPluginDlg@@SAPAVQMetaObject@@XZ@4QBUQMetaData@@B 10008f58     moc_textPlugindlgimpl.obj
 0002:00001f74       ?signal_0@?3??staticMetaObject@textPluginDlg@@SAPAVQMetaObject@@XZ@4UQUMethod@@B 10008f74     moc_textPlugindlgimpl.obj
 0002:00001f80       ?signal_tbl@?3??staticMetaObject@textPluginDlg@@SAPAVQMetaObject@@XZ@4QBUQMetaData@@B 10008f80     moc_textPlugindlgimpl.obj
 0002:0000293c       _GS_ExceptionPointers      1000993c     MSVCRT:gs_report.obj
 0002:000034b0       __ehfuncinfo$??0config@@QAE@ABVQString@@@Z 1000a4b0     config.obj
 0002:000034d4       __unwindtable$??0config@@QAE@ABVQString@@@Z 1000a4d4     config.obj
 0002:0000369c       __unwindtable$??1config@@UAE@XZ 1000a69c     config.obj
 0002:000036bc       __ehfuncinfo$??1config@@UAE@XZ 1000a6bc     config.obj
 0002:000036e0       __ehfuncinfo$?getKeys@config@@QAE?AVQStringList@@XZ 1000a6e0     config.obj
 0002:00003704       __unwindtable$?getKeys@config@@QAE?AVQStringList@@XZ 1000a704     config.obj
 0002:00003764       __unwindtable$?getFilenameFromKey@config@@QAE?AVQString@@ABV2@@Z 1000a764     config.obj
 0002:00003764       __unwindtable$?getHelpFromKey@config@@QAE?AVQString@@ABV2@@Z 1000a764     config.obj
 0002:00003764       __unwindtable$?getDescFromKey@config@@QAE?AVQString@@ABV2@@Z 1000a764     config.obj
 0002:0000376c       __ehfuncinfo$?getFilenameFromKey@config@@QAE?AVQString@@ABV2@@Z 1000a76c     config.obj
 0002:0000376c       __ehfuncinfo$?getHelpFromKey@config@@QAE?AVQString@@ABV2@@Z 1000a76c     config.obj
 0002:0000376c       __ehfuncinfo$?getDescFromKey@config@@QAE?AVQString@@ABV2@@Z 1000a76c     config.obj
 0002:00003790       __ehfuncinfo$?getNamedAttribute@config@@AAE?AVQString@@ABV2@0@Z 1000a790     config.obj
 0002:000037b4       __unwindtable$?getNamedAttribute@config@@AAE?AVQString@@ABV2@0@Z 1000a7b4     config.obj
 0002:0000380c       __unwindtable$?keys@plugindesc@@UAE?AVQStringList@@ABVQString@@0@Z 1000a80c     plugindesc.obj
 0002:0000381c       __ehfuncinfo$?keys@plugindesc@@UAE?AVQStringList@@ABVQString@@0@Z 1000a81c     plugindesc.obj
 0002:00003840       __ehfuncinfo$?highlightParagraph@text_highlighter@@UAEHABVQString@@H@Z 1000a840     text_highlighter.obj
 0002:00003864       __unwindtable$?highlightParagraph@text_highlighter@@UAEHABVQString@@H@Z 1000a864     text_highlighter.obj
 0002:000038ac       __unwindtable$??1text_highlighter@@UAE@XZ 1000a8ac     text_highlighter.obj
 0002:000038ac       __unwindtable$??0text_highlighter@@QAE@PAVQTextEdit@@@Z 1000a8ac     text_highlighter.obj
 0002:000038c4       __ehfuncinfo$??1text_highlighter@@UAE@XZ 1000a8c4     text_highlighter.obj
 0002:000038c4       __ehfuncinfo$??0text_highlighter@@QAE@PAVQTextEdit@@@Z 1000a8c4     text_highlighter.obj
 0002:000038e8       __unwindtable$??1QDockWindowList@@UAE@XZ 1000a8e8     textPlugin.obj
 0002:000038f8       __ehfuncinfo$??1QDockWindowList@@UAE@XZ 1000a8f8     textPlugin.obj
 0002:0000391c       __unwindtable$??1?$QPtrList@VQPopupMenu@@@@UAE@XZ 1000a91c     textPlugin.obj
 0002:00003924       __ehfuncinfo$??1?$QPtrList@VQPopupMenu@@@@UAE@XZ 1000a924     textPlugin.obj
 0002:00003948       __unwindtable$??1QPopupMenuList@@UAE@XZ 1000a948     textPlugin.obj
 0002:00003950       __ehfuncinfo$??1QPopupMenuList@@UAE@XZ 1000a950     textPlugin.obj
 0002:00003974       __unwindtable$??0config_plugin_base@@QAE@ABVQString@@00@Z 1000a974     textPlugin.obj
 0002:00003994       __ehfuncinfo$??0config_plugin_base@@QAE@ABVQString@@00@Z 1000a994     textPlugin.obj
 0002:000039b8       __unwindtable$??1config_plugin_base@@UAE@XZ 1000a9b8     textPlugin.obj
 0002:000039d0       __ehfuncinfo$??1config_plugin_base@@UAE@XZ 1000a9d0     textPlugin.obj
 0002:000039f4       __unwindtable$?about@config_plugin_base@@UAE?AVQString@@XZ 1000a9f4     textPlugin.obj
 0002:00003a04       __ehfuncinfo$?about@config_plugin_base@@UAE?AVQString@@XZ 1000aa04     textPlugin.obj
 0002:00003a28       __ehfuncinfo$??0textPlugin@@QAE@ABVQString@@00@Z 1000aa28     textPlugin.obj
 0002:00003a4c       __unwindtable$??0textPlugin@@QAE@ABVQString@@00@Z 1000aa4c     textPlugin.obj
 0002:00003abc       __ehfuncinfo$??1textPlugin@@UAE@XZ 1000aabc     textPlugin.obj
 0002:00003ae0       __unwindtable$??1textPlugin@@UAE@XZ 1000aae0     textPlugin.obj
 0002:00003b10       __unwindtable$?toolbars@textPlugin@@UAE?AVQDockWindowList@@XZ 1000ab10     textPlugin.obj
 0002:00003b18       __ehfuncinfo$?toolbars@textPlugin@@UAE?AVQDockWindowList@@XZ 1000ab18     textPlugin.obj
 0002:00003b3c       __unwindtable$?menus@textPlugin@@UAE?AVQPopupMenuList@@XZ 1000ab3c     textPlugin.obj
 0002:00003b44       __ehfuncinfo$?menus@textPlugin@@UAE?AVQPopupMenuList@@XZ 1000ab44     textPlugin.obj
 0002:00003b68       __ehfuncinfo$?reply@textPlugin@@UAEXPAVresponse@@@Z 1000ab68     textPlugin.obj
 0002:00003b8c       __unwindtable$?reply@textPlugin@@UAEXPAVresponse@@@Z 1000ab8c     textPlugin.obj
 0002:00003c24       __unwindtable$?navigate@textPlugin@@UAEXABVQString@@0@Z 1000ac24     textPlugin.obj
 0002:00003c3c       __ehfuncinfo$?navigate@textPlugin@@UAEXABVQString@@0@Z 1000ac3c     textPlugin.obj
 0002:00003c60       __ehfuncinfo$?activate@textPlugin@@UAEX_N@Z 1000ac60     textPlugin.obj
 0002:00003c84       __unwindtable$?activate@textPlugin@@UAEX_N@Z 1000ac84     textPlugin.obj
 0002:00003cdc       __unwindtable$?closeEvent@textPlugin@@UAEXPAVQCloseEvent@@@Z 1000acdc     textPlugin.obj
 0002:00003cdc       __unwindtable$?textChanged@textPluginDlg@@QAEXXZ 1000acdc     textPlugin.obj
 0002:00003ce4       __ehfuncinfo$?closeEvent@textPlugin@@UAEXPAVQCloseEvent@@@Z 1000ace4     textPlugin.obj
 0002:00003ce4       __ehfuncinfo$?textChanged@textPluginDlg@@QAEXXZ 1000ace4     textPlugin.obj
 0002:00003d08       __ehfuncinfo$?apply@textPlugin@@UAEXXZ 1000ad08     textPlugin.obj
 0002:00003d2c       __unwindtable$?apply@textPlugin@@UAEXXZ 1000ad2c     textPlugin.obj
 0002:00003dbc       __ehfuncinfo$?about@textPlugin@@UAE?AVQString@@XZ 1000adbc     textPlugin.obj
 0002:00003de0       __unwindtable$?about@textPlugin@@UAE?AVQString@@XZ 1000ade0     textPlugin.obj
 0002:00003e08       __unwindtable$?create@plugindesc@@UAEPAVconfig_plugin_base@@ABVQString@@00@Z 1000ae08     textPlugin.obj
 0002:00003e08       __unwindtable$??0?$QGuardedPtr@VQPopupMenu@@@@QAE@XZ 1000ae08     textPlugin.obj
 0002:00003e08       __unwindtable$??0?$QGuardedPtr@VQDockWindow@@@@QAE@XZ 1000ae08     textPlugin.obj
 0002:00003e10       __ehfuncinfo$??0?$QGuardedPtr@VQPopupMenu@@@@QAE@XZ 1000ae10     textPlugin.obj
 0002:00003e10       __ehfuncinfo$?create@plugindesc@@UAEPAVconfig_plugin_base@@ABVQString@@00@Z 1000ae10     textPlugin.obj
 0002:00003e10       __ehfuncinfo$??0?$QGuardedPtr@VQDockWindow@@@@QAE@XZ 1000ae10     textPlugin.obj
 0002:00003e34       __unwindtable$??1?$QDict@VQAction@@@@UAE@XZ 1000ae34     textPlugin.obj
 0002:00003e3c       __ehfuncinfo$??1?$QDict@VQAction@@@@UAE@XZ 1000ae3c     textPlugin.obj
 0002:00003e60       __unwindtable$?db@@YAXABVQString@@@Z 1000ae60     textPlugin.obj
 0002:00003e68       __ehfuncinfo$?db@@YAXABVQString@@@Z 1000ae68     textPlugin.obj
 0002:00003e8c       __unwindtable$??0textPluginDlg@@QAE@ABVQString@@PAVQWidget@@PBDI@Z 1000ae8c     textPlugindlgimpl.obj
 0002:00003ea4       __ehfuncinfo$??0textPluginDlg@@QAE@ABVQString@@PAVQWidget@@PBDI@Z 1000aea4     textPlugindlgimpl.obj
 0002:00003ec8       __unwindtable$??1textPluginDlg@@UAE@XZ 1000aec8     textPlugindlgimpl.obj
 0002:00003ed8       __ehfuncinfo$??1textPluginDlg@@UAE@XZ 1000aed8     textPlugindlgimpl.obj
 0002:00003efc       __unwindtable$?load@textPluginDlg@@QAE_NABVQString@@@Z 1000aefc     textPlugindlgimpl.obj
 0002:00003efc       __unwindtable$?save@textPluginDlg@@QAEXABVQString@@@Z 1000aefc     textPlugindlgimpl.obj
 0002:00003f14       __ehfuncinfo$?save@textPluginDlg@@QAEXABVQString@@@Z 1000af14     textPlugindlgimpl.obj
 0002:00003f14       __ehfuncinfo$?load@textPluginDlg@@QAE_NABVQString@@@Z 1000af14     textPlugindlgimpl.obj
 0002:00003f38       __unwindtable$??0xml_highlighter@@QAE@PAVQTextEdit@@@Z 1000af38     xml_highlighter.obj
 0002:00003f58       __ehfuncinfo$??0xml_highlighter@@QAE@PAVQTextEdit@@@Z 1000af58     xml_highlighter.obj
 0002:00003f7c       __unwindtable$??1xml_highlighter@@UAE@XZ 1000af7c     xml_highlighter.obj
 0002:00003f84       __ehfuncinfo$??1xml_highlighter@@UAE@XZ 1000af84     xml_highlighter.obj
 0002:00003fa8       __unwindtable$?qt_emit@textPluginDlg@@UAE_NHPAUQUObject@@@Z 1000afa8     moc_textPlugin.obj
 0002:00003fa8       __unwindtable$?qt_emit@textPlugin@@UAE_NHPAUQUObject@@@Z 1000afa8     moc_textPlugin.obj
 0002:00003fb0       __ehfuncinfo$?qt_emit@textPluginDlg@@UAE_NHPAUQUObject@@@Z 1000afb0     moc_textPlugin.obj
 0002:00003fb0       __ehfuncinfo$?qt_emit@textPlugin@@UAE_NHPAUQUObject@@@Z 1000afb0     moc_textPlugin.obj
 0002:00003fd4       __unwindtable$?command@textPluginDlg@@IAEXVQString@@0@Z 1000afd4     moc_textPlugindlgimpl.obj
 0002:00003fd4       __unwindtable$?command@textPlugin@@IAEXVQString@@0@Z 1000afd4     moc_textPlugindlgimpl.obj
 0002:00003fec       __ehfuncinfo$?command@textPlugin@@IAEXVQString@@0@Z 1000afec     moc_textPlugindlgimpl.obj
 0002:00003fec       __ehfuncinfo$?command@textPluginDlg@@IAEXVQString@@0@Z 1000afec     moc_textPlugindlgimpl.obj
 0002:00004010       __ehfuncinfo$??0textPluginDlgBase@@QAE@PAVQWidget@@PBDI@Z 1000b010     textPlugindlg.obj
 0002:00004034       __unwindtable$??0textPluginDlgBase@@QAE@PAVQWidget@@PBDI@Z 1000b034     textPlugindlg.obj
 0002:00004074       __unwindtable$?languageChange@textPluginDlgBase@@MAEXXZ 1000b074     textPlugindlg.obj
 0002:00004084       __ehfuncinfo$?languageChange@textPluginDlgBase@@MAEXXZ 1000b084     textPlugindlg.obj
 0002:000040a8       __sehtable$??_L@YGXPAXIHP6EX0@Z1@Z 1000b0a8     MSVCRT:ehvecctr.obj
 0002:000040c8       __sehtable$??_M@YGXPAXIHP6EX0@Z@Z 1000b0c8     MSVCRT:ehvecdtr.obj
 0002:000040e8       __sehtable$?__ArrayUnwind@@YGXPAXIHP6EX0@Z@Z 1000b0e8     MSVCRT:ehvecdtr.obj
 0002:00004108       __sehtable$__onexit        1000b108     MSVCRT:atonexit.obj
 0002:00004128       __sehtable$___DllMainCRTStartup 1000b128     MSVCRT:crtdll.obj
 0002:00004150       __sehtable$__IsNonwritableInCurrentImage 1000b150     MSVCRT:pesect.obj
 0002:00004170       .edata                     1000b170     textPlugin.exp
 0002:00004198       rgpv                       1000b198     textPlugin.exp
 0002:0000419c       rgszName                   1000b19c     textPlugin.exp
 0002:000041a0       rgwOrd                     1000b1a0     textPlugin.exp
 0002:000041a2       szName                     1000b1a2     textPlugin.exp
 0002:000041b1       $N00001                    1000b1b1     textPlugin.exp
 0002:0000977c       .idata$6                   1001077c     qt-mt323:qt-mt323.dll
 0002:000097cc       .idata$6                   100107cc     MSVCRT:MSVCR120.dll
 0002:000099e0       .idata$6                   100109e0     kernel32:KERNEL32.dll
 0003:00000000       _textPlugin_XPM            10011000     plugindesc.obj
 0003:00000454       _cleanUp_textPlugin        10011454     moc_textPlugin.obj
 0003:00000458       ?param_signal_0@?3??staticMetaObject@textPlugin@@SAPAVQMetaObject@@XZ@4QBUQUParameter@@B 10011458     moc_textPlugin.obj
 0003:00000478       ?$S1@?3??staticMetaObject@textPlugin@@SAPAVQMetaObject@@XZ@4IA 10011478     moc_textPlugin.obj
 0003:00000480       _cleanUp_textPluginDlgBase 10011480     moc_textPlugindlg.obj
 0003:00000488       _cleanUp_textPluginDlg     10011488     moc_textPlugindlgimpl.obj
 0003:0000048c       ?param_signal_0@?3??staticMetaObject@textPluginDlg@@SAPAVQMetaObject@@XZ@4QBUQUParameter@@B 1001148c     moc_textPlugindlgimpl.obj
 0003:000004ac       ?$S1@?3??staticMetaObject@textPluginDlg@@SAPAVQMetaObject@@XZ@4IA 100114ac     moc_textPlugindlgimpl.obj
 0003:000004b0       ___proc_attached           100114b0     MSVCRT:crtdll.obj
 0003:000004b8       _GS_ExceptionRecord        100114b8     MSVCRT:gs_report.obj
 0003:00000508       _GS_ContextRecord          10011508     MSVCRT:gs_report.obj
 0003:000007d4       _DebuggerWasPresent        100117d4     MSVCRT:gs_report.obj
 0004:000000a0       $R000000                   100120a0     Script1.res
 0004:00000528       $R000488                   10012528     Script1.res
